:100000000C94A5130C94D6130C94D6130C94D613FD
:100010000C94D6130C94D6130C94D6130C94D613BC
:100020000C94D6130C94D6130C94D6130C94D613AC
:100030000C94D6130C94D6130C94D6130C94D6139C
:100040000C94D6130C94BDB00C94D6130C94D61308
:100050000C94D6130C94D6130C9486B80C94907D03
:100060000C94D6130C9442370C94D6130C94D613DC
:100070000C94D6130C94D6130C94D6130C94D6135C
:100080000C94D6130C94D6130C94D6130C94D6134C
:100090000C94D6130C94D6130C94D6130C94D6133C
:1000A0000C94D6130C94D6130C94D6130C94D6132C
:1000B0000C94D6130C94D6130C94D6130C94D6131C
:1000C0000C94D6130C94D6130C94D6130C94D6130C
:1000D0000C94D6130C94D6130C94D6130C94D613FC
:1000E0000C94D613CC7BCF7BBE7BC27BC87B067CBB
:1000F000D37BD77BDD7BE17BE57BEB7BEF7BF37B0E
:10010000067CF97BFD7B017CAC7CB17CB67CC07C41
:10011000CA7C437DD47CDC7CE47CEE7CF87C027D74
:10012000117D1B7D437D257D2F7D397DEAB8FAB891
:1001300019B929B944B949B94CB951B954B959B9DE
:100140005CB961B96BB9084AD73B3BCE016E84BC40
:10015000BFFDC12F3D6C74319ABD56833DDA3D0021
:10016000C77F11BED9E4BB4C3E916BAAAABE00006A
:1001700000803F05A84CCDB2D44EB93836A9020C48
:1001800050B9918688083CA6AAAA2ABE0000008021
:100190003F00434F4D4D554E49434154494F4E004A
:1001A00044525952554E004552524F525300494EF7
:1001B000464F004543484F0047322F473320626186
:1001C0006420706172616D65746572730A00536CAE
:1001D0006565702E2E2E00473239206E6577205AC5
:1001E0005F6F66667365743A0028422961636B002D
:1001F000284629726F6E7400285229696768740056
:10020000284C296566740052756E6E696E672069A8
:100210006E204452592D52554E206D6F64650A0070
:10022000473239204175746F20426564204C6576F1
:10023000656C696E670A003F2856296572626F73A4
:1002400065204C6576656C20697320696D706C6102
:10025000757369626C652028302D34292E0A004799
:100260003330206E6577205A5F6F66667365743A27
:1002700000506C6561736520736574205A5F6F660A
:10028000667365743A00205A5F4D41585F504F5372
:100290003A2000206C6576656C5F6265645F763A33
:1002A0002000205A3A200020593A2000426564205C
:1002B000583A200047323800416E796375626963AD
:1002C0002072656164792E00526573756D696E6781
:1002D000207072696E74005761697420666F7220B5
:1002E000757365722E2E2E004E6F206D6F76652E03
:1002F00000456E642066696C65206C6973740A0041
:10030000426567696E2066696C65206C6973740A62
:10031000005344207072696E74696E67206279744C
:100320006520004E6F74205344207072696E7469AA
:100330006E670A00506C6561736520736574205A9E
:100340005F6F66667365743A0048656174696E67CD
:100350002E2E2E00416E796375626963207265618D
:1003600064792E00B301AE01A701A00192016F666E
:10037000660044454255473A004B494C4C45442E93
:1003800020006F6B0048656174696E6720646F6E52
:10039000652E003F0A0020573A0048656174696E77
:1003A000672E2E2E00416E79637562696320726537
:1003B0006164792E00416E796375626963204F66CE
:1003C000662E007A5F6D61783A20007A5F6D696E03
:1003D0003A2000795F6D61783A2000785F6D61782E
:1003E0003A20005265706F7274696E6720656E64A2
:1003F00073746F70207374617475730A004D3134B7
:100400003520533C696E6465783E206F7574206FAB
:10041000662072616E67652028302D31290A0053ED
:10042000657474696E672054726176656C204163EF
:1004300063656C65726174696F6E3A200053657410
:1004400074696E67205265747261637420416363DE
:10045000656C65726174696F6E3A200053657474DF
:10046000696E67205072696E7420416363656C65C4
:10047000726174696F6E3A200053657474696E67B7
:10048000205072696E7420616E64205472617665CA
:100490006C20416363656C65726174696F6E3A20AC
:1004A00000205A00205900580020204D61783A2041
:1004B00000205A00205900580020204D696E3A2033
:1004C000004F666600536F667420656E6473746FC8
:1004D00070733A200020643A0020693A0020703A94
:1004E0000043290A0061626C656420286D696E20F2
:1004F00074656D702000436F6C642065787472754C
:1005000064657320617265200023646566696E65A9
:10051000202044454641554C545F4B6420002364E1
:100520006566696E65202044454641554C545F4BD5
:1005300069200023646566696E6520204445464154
:10054000554C545F4B702000504944204175746FE6
:1005500074756E652066696E6973686564212050E4
:10056000757420746865206C617374204B702C2046
:100570004B6920616E64204B6420636F6E737461FD
:100580006E74732066726F6D2062656C6F77206980
:100590006E746F20436F6E66696775726174696F00
:1005A0006E2E680A00504944204175746F74756E50
:1005B00065206661696C6564212074696D656F757D
:1005C000740A00504944204175746F74756E65203B
:1005D0006661696C6564212054656D706572617433
:1005E00075726520746F6F20686967680A00204B18
:1005F000643A2000204B693A2000204B703A2000DA
:100600000A20436C617373696320504944200A00D7
:100610002054753A2000204B753A2000206D6178F7
:100620003A2000206D696E3A200020643A200020B4
:10063000626961733A200042696C696E656172207B
:1006400047726964206E6F742079657420637265E7
:10065000617465640A00426564204C6576656C6966
:100660006E6720004661696C656420746F20656E5A
:1006700061626C6520426564204C6576656C696ECC
:10068000670A004F666673657473206170706C69E9
:100690006564004572723A20546F6F206661722162
:1006A00000546F6F206661722066726F6D207265F4
:1006B000666572656E636520706F696E740A00000E
:1006C00000000000000000000087434E6F206361BF
:1006D0007365206C696768740A00416374697665A4
:1006E0002045787472756465723A2000556E6B6EA1
:1006F0006F776E20636F6D6D616E643A2022004EDD
:100700006F204C696E65204E756D62657220776949
:10071000746820636865636B73756D2C204C61731E
:1007200074204C696E653A20004B494C4C45442E70
:10073000200053544F505045442E20005072696E93
:100740007465722073746F707065642064756520C1
:10075000746F206572726F72732E204669782074F0
:100760006865206572726F7220616E6420757365B2
:10077000204D39393920746F207265737461727439
:100780002E202854656D70657261747572652069DC
:10079000732072657365742E20536574206974200C
:1007A00061667465722072657374617274696E67D4
:1007B000290A004E6F20436865636B73756D20775F
:1007C000697468206C696E65206E756D6265722C47
:1007D000204C617374204C696E653A200063686533
:1007E000636B73756D206D69736D617463682C2024
:1007F0004C617374204C696E653A20004C696E65DB
:10080000204E756D626572206973206E6F74204C86
:10081000617374204C696E65204E756D6265722B34
:10082000312C204C617374204C696E653A20004D68
:10083000313130004D3331004D38342058205920AB
:100840005A20450053442072656164206572726FBE
:10085000720A00446F6E65207072696E74696E670B
:100860002066696C650A0020496E76616C696420B7
:10087000657874727564657220004572726F7220BB
:1008800077726974696E6720746F20454550524FC6
:100890004D210A00206279746573290A005365743A
:1008A00074696E67732053746F7265642028004505
:1008B0004550524F4D20636865636B73756D206DB5
:1008C00069736D617463680A0020627974657329C5
:1008D0000A002073746F7265642073657474696EA6
:1008E00067732072657472696576656420280050AC
:1008F00072656865617420504C4120426564005007
:1009000072656865617420504C4100507265706179
:100910007265004D3530300053746F7265004D388C
:1009200035372046005A202D20302E31004D3835E5
:10093000372041005A202B20302E31005072657034
:10094000617265204C6576656C696E670047333669
:10095000004D656173757265205A20506F73004DAC
:1009600061696E004733330053746F7265005A201B
:100970004F6666736574005A204F6666736574002F
:100980004E6577205A204F6666736574004E657712
:10099000205A204F66667365740047333500426500
:1009A00067696E204C6576656C696E670041757489
:1009B0006F204C6576656C696E67204265640050F7
:1009C000726568656174204142532042656400503D
:1009D00072656865617420414253005072657061B0
:1009E000726500436F6F6C646F776E00507265685C
:1009F00065617420414253005072656865617420DE
:100A0000504C41004D38340044697361626C65207C
:100A10007374657070657273004D6F7665206178D0
:100A2000697300473238004175746F20686F6D65D7
:100A3000004D61696E004D6F76652058004D6F76F0
:100A4000652059004D6F7665205A0045787472759F
:100A5000646572004578747275646572004D6F76D6
:100A600065205A004D6F76652059004D6F766520E0
:100A700058004D6F766520617869730043616E6E32
:100A80006F7420656E746572207375626469723A62
:100A90002000052E2E004D61696E004361726420B6
:100AA00072656D6F766564004361726420696E7370
:100AB0006572746564006F6B0020746F6F206C6FDB
:100AC0006E6720657874727573696F6E20707265D9
:100AD00076656E7465640A0020636F6C64206578C7
:100AE00074727573696F6E2070726576656E746569
:100AF000640A004B494C4C45442E20004B494C4C59
:100B000045442E2000506C656173652072657365E5
:100B100074005052494E5445522048414C5445446B
:100B2000005072696E7465722068616C7465642E21
:100B3000206B696C6C28292063616C6C6564210AE8
:100B400000656E7175657565696E67202200576175
:100B5000726E696E673A20486F6D696E67204275E4
:100B60006D702044697669736F72203C20310A00F1
:100B70000000A0400000A0400000A0400000524340
:100B800000005243000087430101010000200023C0
:100B900000260029002C002F003200000100000375
:100BA00001060109010505050507050808080802F1
:100BB0000202020A0A0808040404040101010101F6
:100BC0000101010303030303030303040707070CE5
:100BD0000C0C0C0C0C0C0C0202020206060606069B
:100BE0000606060B0B0B0B0B0B0B0B010210202048
:100BF0000808102040102040800201020108040271
:100C000001010204081020408080402010080402E6
:100C1000018004020180402010080402010804023F
:100C20000101020408102040800102040810204045
:100C30008000000A0B02090C0D0E080703040100D6
:100C400000000000000000000000000000000000A4
:100C50000000000000000000000000000012111061
:100C60000000000000000000000000000000000084
:100C7000000000000000004B494C4C45442E200071
:100C8000202D20496E76616C6964206578747275D8
:100C9000646572206E756D62657220210A00414E96
:100CA000594355424943204B4F5353454C005765D8
:100CB0006C636F6D650057656C636F6D6500203107
:100CC0002E312E30002020506C616E6E65724275A0
:100CD0006666657242797465733A200020467265D3
:100CE00065204D656D6F72793A2000436F6D7069B4
:100CF0006C65643A204E6F762031332032303137C4
:100D00000A00207C20417574686F723A2028414E99
:100D1000594355424943204B4F5353454C2C2032A5
:100D20003031372F392F3138290A00323031362D02
:100D300031322D30362031323A303000204C617360
:100D40007420557064617465643A2000312E312E30
:100D5000300A004D61726C696E0020536F667477C3
:100D60006172652052657365740A0020576174636F
:100D700068646F672052657365740A002042726F61
:100D8000776E206F75742052657365740A00204574
:100D9000787465726E616C2052657365740A0050D8
:100DA0006F77657255700A0073746172740A004738
:100DB00031205A2B323000473931006572726F7220
:100DC0002077726974696E6720746F2066696C653C
:100DD0000A00456E6473746F707320256320256369
:100DE00020256320256300205A3A0020593A00202C
:100DF000583A00656E6473746F7073206869743A52
:100E00002000446F6E6520736176696E67206669A5
:100E10006C652E0A004D3239004D6F766520302EFC
:100E2000316D6D004D6F766520316D6D004D6F76C3
:100E3000652031306D6D00507265706172650052D1
:100E40006573746F7265206661696C7361666500B5
:100E50004C6F6164206D656D6F72790053746F72B1
:100E600065206D656D6F72790046696C616D656EA8
:100E700074004D6F74696F6E0054656D70657261BA
:100E800074757265004D61696E00507265686561C8
:100E9000742041425320636F6E660050726568652E
:100EA000617420504C4120636F6E66005049442DA0
:100EB00044005049442D44005049442D49005049B4
:100EC000442D49005049442D50005049442D5000B4
:100ED0002002204661637400200220466163740092
:100EE0002002204D6178002002204D617800200210
:100EF000204D696E002002204D696E004F6666002D
:100F00004F6E20004175746F74656D700046616EA0
:100F10002073706565640046616E2073706565645A
:100F20000042656400426564004E6F7A7A6C650029
:100F30004E6F7A7A6C6500436F6E74726F6C0053FB
:100F4000746F7265206D656D6F7279004265640023
:100F5000426564004E6F7A7A6C65004E6F7A7A6CE7
:100F6000650046616E2073706565640046616E20A1
:100F700073706565640054656D7065726174757237
:100F8000650025753A2530327500253032753A25D1
:100F9000303275002D2D2D005344005A0059005851
:100FA000000120000120007061757365004E6F2004
:100FB00053442063617264005072696E74206672DB
:100FC0006F6D2053440053746F70207072696E749B
:100FD00000526573756D65207072696E74005061A2
:100FE000757365207072696E7400436F6E74726FF2
:100FF0006C004175746F204C6576656C696E672076
:1010000042656400507265706172650054756E656A
:1010100000496E666F2073637265656E00466C6F83
:101020007700466C6F770046616E2073706565646B
:101030000046616E2073706565640042656400421D
:101040006564004E6F7A7A6C65004E6F7A7A6C65D3
:10105000005370656564005370656564004D616997
:101060006E0000002110422063308440A550C6600D
:10107000E770088129914AA16BB18CC1ADD1CEE155
:10108000EFF13112100273325222B5529442F772CC
:10109000D662399318837BB35AA3BDD39CC3FFF3A5
:1010A000DEE36224433420040114E664C774A444DC
:1010B00085546AA54BB528850995EEE5CFF5ACC5F5
:1010C0008DD55336722611163006D776F6669556AC
:1010D000B4465BB77AA719973887DFF7FEE79DD745
:1010E000BCC7C448E5588668A7784008611802283C
:1010F0002338CCC9EDD98EE9AFF9488969990AA995
:101100002BB9F55AD44AB77A966A711A500A333A0B
:10111000122AFDDBDCCBBFFB9EEB799B588B3BBBE4
:101120001AABA66C877CE44CC55C222C033C600C9B
:10113000411CAEED8FFDECCDCDDD2AAD0BBD688D34
:10114000499D977EB66ED55EF44E133E322E511EEB
:10115000700E9FFFBEEFDDDFFCCF1BBF3AAF599F84
:10116000788F8891A981CAB1EBA10CD12DC14EF124
:101170006FE18010A100C230E3200450254046708A
:101180006760B9839893FBA3DAB33DC31CD37FE3B5
:101190005EF3B1029012F322D232354214527762DA
:1011A0005672EAB5CBA5A89589856EF54FE52CD585
:1011B0000DC5E234C324A01481046674476424542A
:1011C0000544DBA7FAB79987B8975FE77EF71DC795
:1011D0003CD7D326F2369106B0165766767615467A
:1011E00034564CD96DC90EF92FE9C899E9898AB9E5
:1011F000ABA94458654806782768C018E1088238CA
:10120000A3287DCB5CDB3FEB1EFBF98BD89BBBABF4
:101210009ABB754A545A376A167AF10AD01AB32A19
:10122000923A2EFD0FED6CDD4DCDAABD8BADE89D44
:10123000C98D267C076C645C454CA23C832CE01C69
:10124000C10C1FEF3EFF5DCF7CDF9BAFBABFD98FD4
:10125000F89F176E367E554E745E932EB23ED10EB9
:10126000F01E7C3C3E5E2B3D3F2F5B5D3B2C2A22DB
:101270005C0000002100240027002A002D0030001F
:10128000330001010000040107010A0100002200EF
:10129000250028002B002E00310034000201000040
:1012A000050108010B014573746570732F6D6D00A6
:1012B0004573746570732F6D6D005A737465707328
:1012C0002F6D6D005A73746570732F6D6D005973B7
:1012D000746570732F6D6D005973746570732F6D25
:1012E0006D005873746570732F6D6D00587374655D
:1012F00070732F6D6D00412D74726176656C0041C5
:101300002D74726176656C00412D72657472616333
:101310007400412D7265747261637400416D61786F
:10132000204500416D6178204500416D6178205A6B
:1013300000416D6178205A00416D6178205900416B
:101340006D6178205900416D6178205800416D61D0
:10135000782058005654726176206D696E0056549C
:10136000726176206D696E00566D696E00566D690A
:101370006E00566D6178204500566D6178204500FD
:10138000566D6178205A00566D6178205A00566D6E
:101390006178205900566D6178205900566D61784A
:1013A000205800566D617820580056652D6A657288
:1013B0006B0056652D6A65726B00567A2D6A6572F0
:1013C0006B00567A2D6A65726B0056792D6A6572CC
:1013D0006B0056792D6A65726B0056782D6A6572BE
:1013E0006B0056782D6A65726B00416363656C0013
:1013F000416363656C005A204F6666736574005ADA
:10140000204F666673657400436F6E74726F6C0074
:1014100046696C2E204469612E0046696C2E20447A
:1014200069612E004F6666004F6E20004520696E90
:10143000206D6D3300436F6E74726F6C0020746F9B
:101440006F206C6F6E6720657874727573696F6E4C
:101450002070726576656E7465640A0020636F6C37
:101460006420657874727573696F6E20707265762A
:10147000656E7465640A000000D2420000D242002A
:101480000087430000D2C20000D2C200000000204A
:1014900064667361663A2000205A3A200020593A67
:1014A000200042656420583A2000203D3D3D3D002B
:1014B000202020200042696C696E656172204C65B5
:1014C00076656C696E6720477269643A0A2000206D
:1014D0006C6576656C5F6265645F76616C75653AB4
:1014E0000020453A00205A3A0020593A00583A0064
:1014F0006175746F25692E67004D3234004D3233AB
:101500002025730057726974696E6720746F2066B6
:10151000696C653A20006F70656E206661696C6564
:10152000642C2046696C653A20006F70656E2066F9
:1015300061696C65642C2046696C653A20004669D7
:101540006C652073656C65637465640A002053697B
:101550007A653A200046696C65206F70656E656437
:101560003A20006F70656E206661696C65642C209E
:1015700046696C653A20002066696C653A20004E29
:101580006F7720002220706F7300222070617265D7
:101590006E743A2200535542524F5554494E4520DD
:1015A00043414C4C207461726765743A22004B4988
:1015B0004C4C45442E2000747279696E6720746F1C
:1015C0002063616C6C207375622D67636F646520A6
:1015D00066696C6573207769746820746F6F206D1D
:1015E000616E79206C6576656C732E204D415820B4
:1015F0006C6576656C2069733A004572726F723A59
:101600000043616E6E6F74206F70656E207375623B
:101610006469722000473930004731205A2D32303A
:101620000070012C0190012701B0012201C0011DB1
:1016300001F00118011002130130020E01600209CD
:101640000190020401C002FF000003FA004003F50C
:10165000008003F000D003EB002004E6007004E1FA
:1016600000E004DC004005D700C005D2004006CDF4
:1016700000D006C8008007C3003008BE00F008B9DB
:1016800000C009B400B00AAF00B00BAA00D00CA58E
:1016900000000EA000500F9B00C010960050129149
:1016A0000000148C00C0158700B0178200B0197DAF
:1016B00000D01B7800001E730040206E009022694D
:1016C00000F024640040275F0090295A00E02B5569
:1016D00000102E500020304B0010324600E0334105
:1016E0000090353C001037370070383200A0392D9B
:1016F00000B03A2800A03B2300603C1E00103D19BA
:1017000000903D1400103E0F00703E0A00C03E05E0
:1017100000003F000073746F70002066697273747C
:10172000005A0059005800486F6D65200020666916
:101730007273740A005A0059005800486F6D652092
:10174000006563686F3A0072657365740073746155
:1017500072740053442063617264206F6B0A006FDF
:1017600070656E526F6F74206661696C65640A0003
:10177000766F6C756D652E696E6974206661696C33
:1017800065640A00534420696E6974206661696C5F
:101790000A0024F4D43050C38E20C2A24017828B9A
:1017A0007011127A910D816CD90AA861E108C758AD
:1017B0006607615143061E4B5D05C145A7041A41EA
:1017C0001104093D9803713931034036DB0265335A
:1017D0009102D4305402802E1D02632CEE01752A32
:1017E000C501B028A001102781018F2564012B2499
:1017F0004B01E0223401AC211F018D200D01801F1F
:10180000FC00841EED00971DDF00B81CD200E61B13
:10181000C600201BBC00641AB200B219A8000A1945
:10182000A0006A189900D117910040178B00B516D7
:10183000840031167E00B31579003A157300C71481
:101840006F0058146A00EE136600881363002513B6
:101850005E00C7125B006C12570015125400C111D4
:10186000510070114F0021114B00D61049008D100E
:1018700047004610440002104200C00F4000800F95
:101880003E00420F3C00060F3B00CB0E3800930E8B
:1018900037005C0E3500270E3400F30D3200C10D09
:1018A0003100900D3000600D2E00320D2D00050D21
:1018B0002C00D90C2B00AE0C2900850C29005C0CE7
:1018C0002700350C27000E0C2600E80B2400C40B63
:1018D0002400A00B23007D0B23005A0B2100390BA1
:1018E0002100180B2000F80A1F00D90A1E00BB0AAD
:1018F0001E009D0A1D00800A1D00630A1C00470A85
:101900001B002C0A1B00110A1A00F7091A00DD0936
:101910001900C4091900AB091900920917007B09C5
:101920001800630917004C09160036091600200933
:1019300016000A091500F5081500E0081400CC0887
:101940001400B8081400A4081400900813007D08BF
:1019500012006B08130058081200460812003408E1
:101960001100230811001208110001081100F007EE
:101970001000E0071000D0071000C0071000B007EB
:101980000F00A107100091070E0083070F007407D6
:101990000F0065070E0057070E0049070E003B07B2
:1019A0000D002E070E0020070D0013070D0006077F
:1019B0000D00F9060C00ED060D00E0060C00D40643
:1019C0000C00C8060C00BC060C00B0060C00A406F7
:1019D0000B0099060C008D060B0082060B007706A3
:1019E0000B006C060B0061060A0057060B004C0644
:1019F0000A0042060A0038060A002E060A002406DB
:101A00000A001A060A001006090007060A00FD056A
:101A10000900F4050900EB050900E2050900D905F4
:101A20000900D0050900C7050900BE050900B50574
:101A30000800AD050800A50509009C0508009405EF
:101A400008008C050800840508007C050800740562
:101A500008006C050700650508005D0507005605D0
:101A600008004E0507004705070040050800380537
:101A70000700310507002A050700230507001C059C
:101A80000600160507000F050700080506000205F9
:101A90000700FB040600F5040700EE040600E80456
:101AA0000600E2040700DB040600D5040600CF04AC
:101AB0000600C9040600C3040600BD040600B704FE
:101AC0000600B1040500AC040600A6040600A0044C
:101AD00005009B04060095040500900406008A0496
:101AE000050085040500800406007A0405007504DD
:101AF0000500700405006B04050066040500610420
:101B000005005C04050057040500520405004D045F
:101B1000050048040500430405003E0404003A049F
:101B2000050035040500300404002C0405002704DA
:101B30000400230405001E0404001A040400160413
:101B40000500110404000D04040009040500040448
:101B5000040000040400FC030400F8030400F40380
:101B60000400F0030400EC030400E8030400E403B1
:101B70000400E0030400DC030400D8030400D403E1
:101B80000400D0030400CC030400C8030300C50311
:101B9000030024F404D9201BC40C5C0E9804C4096F
:101BA0005F0265077101F405F900FB04B300480406
:101BB0008700C10369005803550003034500BE02B6
:101BC0003A008402310053022A002902250004024F
:101BD0002000E4011C00C8011900AF0117009801A2
:101BE0001400840113007101100061011000510103
:101BF0000E0043010D0036010B002B010B002001EC
:101C00000B00150109000C01090003010800FB008D
:101C10000800F3000800EB000700E4000600DE0007
:101C20000600D8000600D2000600CC000500C70060
:101C30000500C2000500BD000400B9000400B500A5
:101C40000400B1000400AD000400A9000400A500D8
:101C50000300A20003009F0004009B000300980003
:101C600003009500020093000300900003008D0024
:101C700002008B000300880002008600020084003E
:101C80000300810002007F0002007D0002007B0053
:101C90000200790002007700010076000200740063
:101CA000020072000100710002006F0002006D006E
:101CB00001006C0002006A00010069000200670078
:101CC000010066000100650001006400020062007E
:101CD000010061000100600001005F0002005D0082
:101CE00001005C0001005B0001005A000100590086
:101CF0000100580001005700010056000100550086
:101D00000100540001005300000053000100520084
:101D1000010051000100500001004F0001004E0081
:101D200000004E0001004D0001004C0001004B007E
:101D300000004B0001004A0001004900010048007A
:101D40000000480001004700010046000000460076
:101D5000010045000000450001004400010043006F
:101D60000000430001004200000042000100410069
:101D7000000041000100400001003F0000003F0062
:101D800001003E0000003E0001003D0000003D005B
:101D900001003C0000003C0000003C0001003B0052
:101DA00000003B0001003A0000003A000100390049
:101DB0000000390001003800000038000000380041
:101DC0000100370000003700010036000000360037
:101DD000000036000100350000003500000035002D
:101DE0000100340000003400000034000100330022
:101DF0000000330000003300010032000000320018
:101E0000000032000100310000003100000031000C
:101E100001003000000030000000300001002F0001
:101E200000002F0000002F0000002F0001002E00F6
:101E300000002E0000002E0001002D0000002D00EB
:101E400000002D0000002D0001002C0000002C00DF
:101E500000002C0000002C0001002B0000002B00D3
:101E600000002B0000002B0001002A0000002A00C7
:101E700000002A0000002A000100290000002900BB
:101E800000002900000029000000290001002800AE
:101E900000002800000028000000280000002800A2
:101EA0000100270000002700000027000000270095
:101EB0000000270001002600000026000000260088
:101EC000000026000000260001002500000025007B
:101ED000000025000000250000002500000025006E
:101EE0000100240000002400000024000000240061
:101EF0000000240001002300000023000000230054
:101F00000000230000002300000023000000230045
:101F10000100220000002200000022000000220038
:101F2000000022000000220001002100000021002A
:101F3000000021000000210000002100000021001D
:101F4000000021000100200000002000000020000F
:101F50000000200000002000000020000000200001
:101F60000000200001001F0000001F0000001F00F3
:101F700000001F0000001F0000001F0000001F00E5
:101F800001001E0000001E0000001E0000001E00D8
:101F900000004D383420582059205A204500205A3E
:101FA0003A0020593A0020436F756E7420583A2049
:101FB0000028290A0053746F7077617463683A3A95
:101FC000006265640A002C2073797374656D207358
:101FD000746F7070656421204865617465725F4933
:101FE000443A20004572723A204D494E54454D50B6
:101FF000004D494E54454D502074726967676572B3
:102000006564004572723A204D415854454D502048
:10201000424544004572723A204D415854454D5056
:10202000004D415854454D50207472696767657280
:1020300065640020706F736974696F6E206F7574CA
:10204000206F662072616E67652E0A003F50726FC6
:10205000626520004733300047323800473238008D
:1020600047323900473238004D3838380047323867
:1020700000473239004732380046696C6520646594
:102080006C657465643A0044656C6574696F6E20B4
:102090006661696C65642C2046696C653A20006F46
:1020A00070656E206661696C65642C2046696C659C
:1020B0003A20002569730025696D20256973002584
:1020C00069682025696D20256973002569642025CC
:1020D00069682025696D20256973002569792025A7
:1020E0006964202569682025696D20256973005081
:1020F00072696E742074696D653A200050726F7455
:1021000065637465642050696E0A002042403A009D
:1021100020403A00202F0020423A00202F00205477
:102120003A0042656420646F6E652E003F0A00200D
:10213000573A004265642048656174696E672E00F5
:1021400020453A00205A3A0020593A00583A0046B1
:1021500049524D574152455F4E414D453A4D61728E
:102160006C696E20312E312E30416E796375626953
:102170006320534F555243455F434F44455F55528B
:102180004C3A2050524F544F434F4C5F5645525398
:10219000494F4E3A312E30204D414348494E455F1C
:1021A000545950453A416E796375626963204558C8
:1021B0005452554445525F434F554E543A31205581
:1021C0005549443A63656465326132662D34316144
:1021D000322D343734382D396231322D6335356341
:1021E00036326633363766660A003A20007A5F6D0B
:1021F00061783A20007A5F6D696E3A20005A204F6C
:102200006666736574005374616E64617264204421
:102210006576696174696F6E3A20002052616E675D
:10222000653A2000204D61783A2000204D696E3AD1
:1022300020004D65616E3A200046696E69736865DD
:102240006421002072616E67653A2000206D61781C
:102250003A2000206D696E3A2000207369676D6135
:102260003A2000206D65616E3A20003A207A3A20CB
:1022700000206F662000205A002059002058004797
:102280006F696E6720746F3A002C200050756C6C7B
:10229000696E6720706F696E7420746F7761726405
:1022A000732063656E7465723A00436C6F636B777D
:1022B0006973650A00436F756E7465722D00204462
:1022C0006972656374696F6E3A2000202020616E28
:1022D000676C653A20005374617274696E6720728E
:1022E00061646975733A2000506F736974696F6E29
:1022F000696E67207468652070726F62652E2E2E7D
:102300000A003F4E756D626572206F66206C6567CE
:102310007320696E206D6F76656D656E74206E6FCB
:102320007420706C61757369626C652028302D3182
:1023300035292E0A003F2028582C5929206C6F631C
:102340006174696F6E206F757473696465206F6660
:102350002070726F626561626C652072616469757C
:10236000732E0A003F53616D706C652073697A6546
:10237000206E6F7420706C61757369626C652028C3
:10238000342D3530292E0A004D3438205A2D507204
:102390006F6265205265706561746162696C697411
:1023A0007920546573740A003F566572626F7365D5
:1023B000204C6576656C206E6F7420706C6175734F
:1023C00069626C652028302D34292E0A004861721C
:1023D00064636F6465642044656661756C74205342
:1023E000657474696E6773204C6F616465640A007C
:1023F00020204D383531205A005A2D50726F6265B9
:10240000204F666673657420286D6D293A0A002096
:10241000204D3230302044300A0020204D32303000
:102420002044002044697361626C65640A00466957
:102430006C616D656E742073657474696E67733A50
:102440000020440020490020204D3330312050002E
:102450005049442073657474696E67733A0A0020AA
:10246000460020420020480020204D3134352053C2
:10247000004D6174657269616C2068656174757086
:1024800020706172616D65746572733A0A00204351
:102490000020420020410020530020520020204D07
:1024A000363635204C0044656C7461207365747455
:1024B000696E67733A204C3D646961676F6E616C49
:1024C0005F726F642C20523D7261646975732C20B9
:1024D000533D7365676D656E74735F7065725F738E
:1024E00065636F6E642C204142433D646961676F90
:1024F0006E616C5F726F645F7472696D5F746F7729
:1025000065725F5B3132335D0A00205A002059004A
:1025100020204D363636205800456E6473746F7037
:102520002061646A7573746D656E7420286D6D2901
:102530003A0A0020204D3432302053004175746F28
:1025400020426564204C6576656C696E673A0A00C6
:10255000205A0020590020204D32303620580048A3
:102560006F6D65206F666673657420286D6D290A2E
:1025700000204500205A0020590020580020420029
:1025800020540020204D32303520530041647661C4
:102590006E636564207661726961626C65733A206E
:1025A000533D4D696E2066656564726174652028CF
:1025B0006D6D2F73292C20543D4D696E207472610E
:1025C00076656C20666565647261746520286D6D42
:1025D0002F73292C20423D6D696E696D756D2073D6
:1025E00065676D656E742074696D6520286D73294B
:1025F0002C20583D6D6178696D756D205859206AA1
:1026000065726B20286D6D2F73292C20205A3D6D2B
:102610006178696D756D205A206A65726B20286D2E
:102620006D2F73292C2020453D6D6178696D756D86
:102630002045206A65726B20286D6D2F73290A0072
:1026400020540020520020204D32303420500041D0
:102650006363656C65726174696F6E733A20503D97
:102660007072696E74696E672C20523D7265747267
:1026700061637420616E6420543D74726176656C90
:102680000A00204500205A0020590020204D3230F9
:10269000312058004D6178696D756D204163636527
:1026A0006C65726174696F6E20286D6D2F733229AD
:1026B0003A0A00204500205A0020590020204D32BF
:1026C00030332058004D6178696D756D2066656501
:1026D00064726174657320286D6D2F73293A0A0046
:1026E000204500205A0020590020204D3932205822
:1026F0000053746570732070657220756E69743A4A
:102700000A00526573656E643A20004E414E494E90
:10271000495459494E46CDCCCC3D0AD7233C17B736
:10272000D13877CC2B329595E6241FB14F0A0000A3
:1027300020410000C84200401C4620BCBE4CCA1BC1
:102740000E5AAEC59D7472E119DA11241FBECFEF87
:10275000D1E2DEBFCDBF00E00CBF14E0A0E0B2E0EC
:10276000E8E4F3EE01E00BBF02C007900D92A43B3A
:10277000B107D9F725E1A4EBB4E001C01D92A13E59
:10278000B207E1F713E1C4EAD3E100E006C0219704
:102790000109802FFE010E9450E5C33AD10780E075
:1027A0000807A9F70E94A3DA0C9492F10C94000098
:1027B0002F923F924F925F926F927F928F929F9251
:1027C000AF92BF92CF92DF92EF92FF920F931F933F
:1027D000CF93DF93CDB7DEB7C257D1090FB6F894C8
:1027E000DEBF0FBECDBF0091730820E6029F8001BF
:1027F00011240D50194F1093C3040093C20480910B
:10280000E41380FF18C0E1E4F7E184917F013FEF1A
:10281000E31AF30A882321F00E94A832F701F5CFCA
:10282000D8018D918D01882319F00E94A832F8CF2C
:102830008AE00E94A8322091C2043091C304F901B9
:1028400080812F5F3F4F8032D1F3F093C304E09338
:10285000C2048E3469F0F090C204E090C3046AE2CE
:1028600070E08F2D9E2D0E9485E80097D1F420C046
:10287000818190ED980F9A3010F08D3261F7329689
:10288000DF0131962C9120532A30D0F3CD01FC0189
:10289000019620812032D9F3F093C304E093C2045F
:1028A000DACFFC0131968291803231F08A3221F008
:1028B000AF2DBE2D9D9102C01082F5CFFD0180810C
:1028C00011968032D9F380538A3010F00C94FA2F8D
:1028D00020E030E06AE0629FA001639F500D112468
:1028E0009A01205331098191280F311D87FD3A95B6
:1028F000808180538A3078F38F013196D8018C9192
:102900008032D1F31093C0040093BF049D3411F4BE
:102910000C94971E943511F40C944D2E973411F0AD
:102920000C94FA2F2E31310509F4F0C7B0F424309D
:10293000310538F48091AB022230310508F444C0EF
:102940004DC02C31310509F42BC208F035C22430BA
:10295000310509F4E3C10C946C2E2832310509F4D9
:102960001BC2B8F42332310509F41EC224323105EA
:1029700009F41EC22132310511F00C946C2E84EB47
:1029800092E09093930B8093920B0E94AB310C9446
:102990006C2E2A35310511F40C94E81D48F42932C7
:1029A000310511F00C946C2E0E94EA6C0C946C2E84
:1029B0002B35310511F40C94EC1D2C35310511F437
:1029C0000C94F11D0C946C2E882311F40C946C2E35
:1029D0000E94F8950E947F600C946C2E882311F45D
:1029E0000C946C2E11E02230310509F010E00E94A9
:1029F000F89519821A821B821C821D821E821F82F8
:102A0000188682E50E94C030882309F438C10E94EC
:102A10005D316B017C012091FF0E3091000F4091E0
:102A2000010F5091020F2AA73BA74CA75DA78090EA
:102A3000030F9090040FA090050FB090060F8091A7
:102A4000EF0E9091F00EA091F10EB091F20E8EABC0
:102A50009FABA8AFB9AF2091F30E3091F40E409127
:102A6000F50E5091F60E2AAB3BAB4CAB5DAB20E0C4
:102A700030E0A901C701B6010E945AED882309F48C
:102A800014C12AA53BA54CA55DA56EA97FA988AD5B
:102A900099AD0E945AED81110BC0A50194016AA95C
:102AA0007BA98CA99DA90E945AED882309F4FDC039
:102AB00020E030E0A901C701B6010E945AED881F4D
:102AC0008827881F18130BC080E090E0A0E8BFE3C0
:102AD00026968CAF9DAFAEAFBFAF26970AC020E061
:102AE00030E040E85FEB26962CAF3DAF4EAF5FAFD6
:102AF00026972AA53BA54CA55DA56EA97FA988AD03
:102B000099AD0E9458E522966CAF7DAF8EAF9FAF16
:102B10002297A50194016AA97BA98CA99DA90E946D
:102B200058E56AAF7BAF8CAF9DAF22962CAD3DAD23
:102B30004EAD5FAD2297CA01B9010E94BFED2B01D6
:102B40003C012AAD3BAD4CAD5DADCA01B9010E945F
:102B5000BFED9B01AC01C301B2010E9459E50E9487
:102B6000EAE76EA77FA788AB99AB20E030E040E0B2
:102B70005FE30E94BFED2B013C01A7019601C70155
:102B8000B6010E94BFED6B017C01A3019201C3015C
:102B9000B2010E94BFED9B01AC01C701B6010E94CA
:102BA00058E50E94EAE79B01AC0126966CAD7DAD2D
:102BB0008EAD9FAD26970E94BFED6B017C012EA9C3
:102BC0003FA948AD59AD6AA57BA58CA59DA50E94DE
:102BD00059E520E030E040E05FE30E94BFED2B01CB
:102BE0003C016AAD7BAD8CAD9DAD90582EA53FA547
:102BF00048A959A90E9445E69B01AC01C701B6014D
:102C00000E94BFED9B01AC01C301B2010E9459E5D6
:102C10002AA53BA54CA55DA50E9458E569837A834A
:102C20008B839C832AA93BA94CA95DA9C501B4014A
:102C30000E9459E520E030E040E05FE30E94BFEDF4
:102C40002B013C012EA53FA548A959A922966CADA0
:102C50007DAD8EAD9FAD22970E9445E69B01AC01F4
:102C6000C701B6010E94BFED9B01AC01C301B201D7
:102C70000E9459E5A50194010E9458E512C089E41B
:102C80000E94C030882331F00E945D3169837A83CD
:102C90008B839C838AE40E94C030882331F00E9499
:102CA0005D316D837E838F83988720E030E0A901BA
:102CB00069817A818B819C810E945AED81110BC0C0
:102CC00020E030E0A9016D817E818F8198850E948E
:102CD0005AED882349F0612FCE0101960E940BAC7A
:102CE0000E949D320C946C2EEAEFF5E184918F01E5
:102CF0000F5F1F4F882321F00E94A832F801F6CF02
:102D0000E8EBF1E084918F010F5F1F4F882311F4EE
:102D10000C946C2E0E94A832F801F4CF80E50E943A
:102D2000C030882329F00E9452316B017C0103C01E
:102D3000C12CD12C760183E50E94C030882321F07C
:102D40000E9486316B017C010E9479B00E949D3205
:102D50008091A2069091A306A091A406B091A50629
:102D6000C80ED91EEA1EFB1E80915802811105C0B3
:102D700060E08EEC91E00E9426820E94847DDC015E
:102D8000CB018C199D09AE09BF09B7FD02C00C9497
:102D90006C2E0E949B56F1CF0E94EE6C0C946C2E10
:102DA0000E94DE9C0C946C2E0E9445C20C946C2EEA
:102DB0000E949BC00C946C2E81E08093BE040E9404
:102DC000E6A5811148C486E50E94C030882329F019
:102DD0000E943A319FAF8EAF04C041E050E05FAF38
:102DE0004EAF8EAD9FAD059768F0E7E3F2E08491BA
:102DF0008F010F5F1F4F882309F42DC40E94A83252
:102E0000F801F5CF84E40E94C0308EAB85E40E94C7
:102E1000C03060968FAF6097AEADBFADAB2BD9F031
:102E2000E0E2F2E084918F010F5F1F4F882321F0D1
:102E30000E94A832F801F6CFBEA9BB2361F0E7E0FB
:102E4000F2E084918F010F5F1F4F882321F00E94D1
:102E5000A832F801F6CF83E50E94C030882349F0FC
:102E60000E945D3120E030E040E752E40E9445E6F8
:102E700004C060E070E088EC92E46093000270931C
:102E8000010280930202909303028CE40E94C030FE
:102E9000882319F00E945D3118C020E030E04CEB2F
:102EA00052E46091E20E7091E30E8091E40E9091F5
:102EB000E50E0E9458E52091D60E3091D70E409134
:102EC000D80E5091D90E0E9459E50E94B6E67BA714
:102ED0006AA782E50E94C030882319F00E945D3104
:102EE00018C020E030E04CEC52E46091E20E7091AA
:102EF000E30E8091E40E9091E50E0E9459E5209139
:102F0000D60E3091D70E4091D80E5091D90E0E9416
:102F100059E50E94B6E68B0186E40E94C030882302
:102F200019F00E945D3118C020E030E04EEA52E412
:102F30006091E60E7091E70E8091E80E9091E90E97
:102F40000E9458E52091DA0E3091DB0E4091DC0EA4
:102F50005091DD0E0E9459E50E94B6E61B0182E405
:102F60000E94C030882319F00E945D3118C020E013
:102F700030E042EB52E46091E60E7091E70E8091F2
:102F8000E80E9091E90E0E9459E52091DA0E3091F9
:102F9000DB0E4091DC0E5091DD0E0E9459E50E943F
:102FA000B6E67BAB6AABEAA5FBA5BF01FF0F880BBA
:102FB000990B0E9460ED26966CAF7DAF8EAF9FAFF0
:102FC00026978090E20E9090E30EA090E40EB090D1
:102FD000E50EC090D60ED090D70EE090D80EF090AF
:102FE000D90E20E030E042ED52E4C501B4010E9468
:102FF00058E5A70196010E9459E59B01AC01269670
:103000006CAD7DAD8EAD9FAD26970E945AED87FDCC
:103010000FC0F1E02796FFAF2797C80143972AA575
:103020003BA52817390744F427961FAE279704C0FD
:1030300031E027963FAF2797B801012E000C880B8F
:10304000990B0E9460ED2B013C0120E030E042ED45
:1030500052E4C501B4010E9459E5A70196010E94FE
:1030600059E59B01AC01C301B2010E94A1E718160A
:1030700054F041E04EA78AA59BA54396801791077F
:1030800024F41EA602C051E05EA7B101032C000C7F
:10309000880B990B0E9460ED2B966CAF7DAF8EAFC5
:1030A0009FAF2B978090E60E9090E70EA090E80ED1
:1030B000B090E90EC090DA0ED090DB0EE090DC0EFE
:1030C000F090DD0E20E030E042ED52E4C501B401A5
:1030D0000E9458E5A70196010E9459E59B01AC01A9
:1030E0002B966CAD7DAD8EAD9FAD2B970E945AEDAA
:1030F00087FD0AC081E08AAF8AA99BA94397281659
:10310000390624F41AAE02C091E09AAFAAA9BBA96D
:10311000BD01BB0F880B990B0E9460ED2B013C0198
:1031200020E030E042ED52E4C501B4010E9459E5CF
:10313000A70196010E9459E59B01AC01C301B201B0
:103140000E94A1E7FF24F394181644F0C1014396AE
:10315000EAA9FBA98E179F070CF4F12C2796FFAD67
:103160002797F1110EC02EA5222329F088EF91E0B8
:103170000E94F0E40DC03AAD31110AC0F1100FC049
:1031800016C080E092E00E94F0E44EA54111EECF1F
:103190005AAD552321F080EF91E00E94F0E4FF202A
:1031A00009F459C289EE91E00E94F0E454C20E94F1
:1031B00079B080914E098EA710924E099EA9911167
:1031C0000AC00E94DE588AEA96E00E94E0950E94BA
:1031D00035550E940E320E942E9881E00E94D799A8
:1031E000882321F0AEA5A0934E0935C21CA21DA2D2
:1031F0001EA21FA218A219A21AA21BA2EAA5FBA531
:103200000E1B1F0B17FF02C0095F1F4F83E01595B0
:1032100007958A95E1F7B801012E000C880B990BF0
:103220000E9460ED2F966CAF7DAF8EAF9FAF2F9752
:10323000EAA8FBA8E218F308F7FE03C0F7E0EF0ED8
:10324000F11CB3E0F594E794BA95E1F7B7010F2CC0
:10325000000C880B990B0E9460ED2B013C018AE564
:103260000E94C03081110E945D316091770670919B
:103270007806072E000C880B990B0E9460ED9B01CD
:10328000AC012F966CAD7DAD8EAD9FAD2F970E949A
:103290005AED811123C06091790670917A06072E4C
:1032A000000C880B990B0E9460ED9B01AC01C301DF
:1032B000B2010E945AED811111C080917306909164
:1032C00074062AA53BA52817390741F48091750695
:1032D000909176062816390609F44EC03EA5309323
:1032E0004E090E94DD971093780600937706F092BE
:1032F0007A06E09279062091E20E3091E30E409139
:10330000E40E5091E50E26966CAD7DAD8EAD9FAD71
:1033100026970E9458E52091D60E3091D70E409105
:10332000D80E5091D90E0E9458E50E94B6E67093CF
:103330007406609373062091E60E3091E70E40917B
:10334000E80E5091E90E2B966CAD7DAD8EAD9FAD24
:103350002B970E9458E52091DA0E3091DB0E4091B8
:10336000DC0E5091DD0E0E9458E50E94B6E6709387
:103370007606609375061EA641E04AAB1BA61AA608
:1033800051E05AAF89E027968FAF2797312CDE01A5
:103390001196B9A7A8A781E04AA948274AAB8AA5F0
:1033A0009BA5092E000CAA0BBB0B64968CAF9DAF9E
:1033B000AEAFBFAF649727962FAD2797321609F4AB
:1033C000CEC0632D032C000C770B880B990B0E9449
:1033D00060ED9B01AC012F966CAD7DAD8EAD9FADC8
:1033E0002F970E94BFED9B01AC0126966CAD7DAD81
:1033F0008EAD9FAD26970E9459E56B017C016496C6
:103400006CAD7DAD8EAD9FAD64970E9460ED9B016C
:10341000AC01C301B2010E94BFED9B01AC012B9630
:103420006CAD7DAD8EAD9FAD2B970E9459E54B01E4
:103430005C0120E030E0A901C701B6010E945AED0D
:1034400087FD05C020E030E040E05FE303C020E0FE
:1034500030E0A901C701B6010E9459E50E94EBE6E0
:103460006B017C016CA37DA38EA39FA320E030E0C1
:10347000A901C501B4010E945AED87FD05C020E0F5
:1034800030E040E05FE303C020E030E0A901C50187
:10349000B4010E9459E50E94EBE668A379A38AA3D0
:1034A0009BA3A8A5B9A5ECE01D92EA95E9F7C9820E
:1034B000DA82EB82FC826D837E838F839887CE01D4
:1034C00001960E94A2AB882309F446C02EAD3FAD01
:1034D00060964FAD6097BE01605E7F4FCE018496CF
:1034E0000E94209A29E0332D3203800111244AA53D
:1034F0005BA5040F151F000F111F000F111F015DA9
:103500001A4F209144023091450240914602509159
:1035100047020E9459E5D8016D937D938D939C934A
:10352000139707ED11E0F8018491882329F00F5FCC
:103530001F4F0E94A832F7CF60914402709145025C
:10354000809146029091470242E00E949B368AE0B9
:103550000E94A8320E949B56FAAD3F0E2CCF4AA57E
:103560005BA54F5F5F4F5BA74AA749305105A1F0AC
:10357000BAA9B11109C0EFEFEAAFFFEF2796FFAF8D
:103580002797A8E03A2E07CF21E02AAF39E0279607
:103590003FAF2797312CFFCE80E00E94D799882338
:1035A00021F05EA550934E0956C00E9414988EA932
:1035B000811124C014E0E8E0EE2E04E0FE2CF11AA4
:1035C000DE2CD01A21E041E0602F812F0E94EADF3B
:1035D00021E04FEF602F8F2D0E94EADF2FEF41E0B7
:1035E0006D2D812F0E94EADF2FEF4FEF6D2D8F2D74
:1035F0000E94EADF015020F71150F8F60E9406976A
:103600009EA991111BC081E080932E058FEF9EE053
:103610000E94A75E9B01AC016091070F7091080F9B
:103620008091090F90910A0F0E9458E56093070F4F
:103630007093080F8093090F90930A0F0E94B7C7E9
:10364000AEA9AA2311F08EA501C081E080934E0996
:1036500081110E940E3281E08093441580903705DD
:1036600090903805A0903905B0903A0520913B051F
:1036700030913C0540913D0550913E05C501B40196
:103680000E9458E59B01AC01C501B4010E9459E5B7
:103690006B017C016093330570933405809335058D
:1036A00090933605A50194010E9458E59B01AC0159
:1036B000C701B6010E9459E560932F05709330054C
:1036C000809331059093320580904705909048058E
:1036D000A0904905B0904A052091430530914405DA
:1036E0004091450550914605C501B4010E9458E539
:1036F0009B01AC01C501B4010E9459E56B017C013D
:1037000060934B0570934C0580934D0590934E0547
:10371000A50194010E9458E59B01AC01C701B601C7
:103720000E9459E560934F057093500580935105B1
:1037300090935205C0905705D0905805E0905905D8
:10374000F0905A0520915B0530915C0540915D0534
:1037500050915E05C701B6010E9458E59B01AC017E
:10376000C701B6010E9459E5609353057093540553
:103770008093550590935605C0906F05D0907005C5
:10378000E0907105F090720520916B0530916C0509
:1037900040916D0550916E05C701B6010E9458E534
:1037A0009B01AC01C701B6010E9459E56093730506
:1037B000709374058093750590937605C0902F06DD
:1037C000D0903006E0903106F0903206209133061A
:1037D000309134064091350650913606C701B60146
:1037E0000E9458E59B01AC01C701B6010E9459E552
:1037F00060932B0670932C0680932D0690932E06D3
:103800008090570690905806A0905906B0905A069E
:1038100020915B0630915C0640915D0650915E06FA
:10382000C501B4010E9458E59B01AC01C501B4017A
:103830000E9459E56B017C01609353067093540616
:103840008093550690935606A50194010E9458E571
:103850009B01AC01C701B6010E9459E560934F0678
:10386000709350068093510690935206809067069D
:1038700090906806A0906906B0906A062091630651
:10388000309164064091650650916606C501B40109
:103890000E9458E59B01AC01C501B4010E9459E5A5
:1038A0006B017C0160936B0670936C0680936D06D0
:1038B00090936E06A50194010E9458E59B01AC010E
:1038C000C701B6010E9459E560936F0670937006B8
:1038D00080937106909372060E94FE3764EF71E048
:1038E00080E090E00E944C7D0E9462D464E670E02B
:1038F00080E090E00E944C7D0E94643A64E670E0B3
:1039000080E090E00E944C7D0C946C2E88E50E9433
:10391000C030882319F00E945D310DC020E030E0F6
:10392000A9016091FF0E7091000F8091010F90919D
:10393000020F0E9459E56CA37DA38EA39FA389E586
:103940000E94C030882319F00E945D310DC020E034
:1039500030E0A9016091030F7091040F8091050F71
:103960009091060F0E9459E568A379A38AA39BA3AF
:103970000CA11DA12EA13FA109831A832B833C8397
:103980006D837E838F83988720E030E0A90160916A
:10399000EA0E7091EB0E8091EC0E9091ED0E0E946C
:1039A00059E52091DE0E3091DF0E4091E00E5091EE
:1039B000E10E0E9459E569877A878B879C87CE0143
:1039C00001960E94A2AB882311F40C946C2E83E51F
:1039D0000E94C030882321F00E940231482F01C08C
:1039E00041E080E0E3964FAFE3970E94AC970E94DE
:1039F0002E9821E030E0E3964FADE397BE01605E84
:103A00007F4FCE0184960E94209A6B017C010E9418
:103A1000B7C7ECEAF2E084918F010F5F1F4F882354
:103A200021F00E94A832F801F6CF27E137EB41EDF3
:103A300058E36CA17DA18EA19FA10E9459E542E0AF
:103A40000E949B36E7EAF2E084918F010F5F1F4FDF
:103A5000882321F00E94A832F801F6CF27E137EB46
:103A600041ED58E368A179A18AA19BA10E9459E583
:103A700042E00E949B36E2EAF2E084918F010F5F00
:103A80001F4F882321F00E94A832F801F6CF27E1CA
:103A900037EB41ED58E3C701B6010E9459E542E01A
:103AA0000E949B368AE00E94A832E3E9F2E084910A
:103AB0008F010F5F1F4F882321F00E94A832F80169
:103AC000F6CF8090B4049090B504A090B604B09066
:103AD000B70427E137EB41ED58E3C501B4010E947B
:103AE00059E542E00E949B368AE00E94A832E6E84F
:103AF000F2E084918F010F5F1F4F882321F00E9415
:103B0000A832F801F6CF42E063E070E087E893E482
:103B10000E949B368AE00E94A83220E030E047E80D
:103B200053E4C501B4010E9458E5A70196010E9423
:103B300059E527E137EB41ED58E30E9459E59B0138
:103B4000AC0160E070E0CB010E9458E560937F0615
:103B5000709380068093810690938206E1E7F2E0FD
:103B600084918F010F5F1F4F882321F00E94A8329C
:103B7000F801F6CF60917F067091800680918106F2
:103B80009091820642E00E949B368AE00E94A83211
:103B9000EFE5F2E084918F010F5F1F4F882321F042
:103BA0000E94A832F801F6CF60914402709145025C
:103BB000809146029091470242E00E949B368AE043
:103BC0000E94A8320E9414980E94B7C70C946C2ED1
:103BD0001092BD040C946C2E81E08093BD040C9473
:103BE0006C2E85E40E94C030B82E811102C00E9464
:103BF00079B05DEF852E52E0952E6FEFC62E6EE008
:103C0000D62E76EDE72E7EE0F72E00E010E0A12C18
:103C1000F40181914F010E94C0308823E1F1D60167
:103C20002D913D914D915C91E0962FAFE097E196FB
:103C30003FAFE197E3964FAFE397E2965FAFE2972E
:103C40000E945D31F6016083718382839383E096E5
:103C50002FADE097E1963FADE197E3964FADE39747
:103C6000E2965FADE29703301105A9F00E9458E596
:103C70009B01AC01D7016D917D918D919C910E942A
:103C800059E5F7016083718382839383C8010E94A1
:103C9000CD9BAA24A3940F5F1F4FF4E0CF0ED11C3D
:103CA00024E0E20EF11C0430110509F0B1CFAA2086
:103CB00019F00E940E3237C0BB20A9F1C0900B0F43
:103CC000D0900C0FE0900D0FF0900E0F2091030993
:103CD000309104094091050950910609C701B601C8
:103CE0000E94BFED0E94ACE76093D00B7093D10BA4
:103CF0008093D20B9093D30BC701B6010E94B6E616
:103D00002FB7F8946093E0137093E1138093E2135C
:103D10009093E3132FBF1092C00B1092C10B10921F
:103D2000C20B1092C30B0E94B7C70C946C2E2537A0
:103D3000310509F47FC608F0C8C02B34310509F4F9
:103D4000F7C208F06DC02831310509F47EC2E8F5EC
:103D50002231310509F4CAC5D8F42230310508F4FE
:103D6000B3C12131310511F00C946C2E60E088EE66
:103D700092E00E9426825F988A989FB7F89480917B
:103D800008018E7F809308019FBF12980C946C2EBF
:103D90002531310509F44FC240F42431310511F0C9
:103DA0000C946C2EE0E0F3E003C22631310509F4F7
:103DB00046C22731310511F00C946C2E40E061E0D1
:103DC000C8010E941EA10C946C2E2E31310509F4FD
:103DD00095C298F42A31310509F446C208F43BC271
:103DE0002B31310509F44EC22C31310511F00C9400
:103DF0006C2E0E9493C00C946C2E2032310509F475
:103E000081C208F48DC22A32310509F48DC22033F3
:103E1000310511F00C946C2E0E94BBCA0C946C2ED0
:103E20002936310509F496C340F52335310509F4E7
:103E300058C598F42D34310509F49CC208F47CC2AD
:103E40002135310509F434C52235310511F00C94C2
:103E50006C2E1092BC040C946C2E2535310509F49F
:103E600049C508F443C52C35310509F456C5283633
:103E7000310509F48FC20C946C2E2E36310509F4ED
:103E8000CBC280F42B36310509F40EC508F408C501
:103E90002C36310509F43FC32D36310509F474C3BE
:103EA0000C946C2E2037310509F439C308F4C7C2CD
:103EB0002237310509F4BAC52337310511F00C94C6
:103EC0006C2E0E94A7C70C946C2E2E3241E0340752
:103ED00011F40C94D42908F06BC02B3C310509F483
:103EE00018C798F52C38310509F41DC380F428371C
:103EF000310509F427C62937310509F42AC62737C1
:103F0000310511F00C946C2EE3EEF3E099C52E3BD5
:103F1000310509F4C1C430F42139310509F41FC653
:103F20000C946C2E283C310509F490C6293C3105CF
:103F300011F00C946C2E6FE0E62E69E0F62E0DEF7A
:103F400012E074E0D72ED00ECCC62C3D310511F412
:103F50000C94CA2898F42D3C310509F461C708F483
:103F6000F5C62E3C310509F4C6C7233D310511F0D5
:103F70000C946C2EE1E4F7E10C944428223E3105C8
:103F800011F40C94EE2838F42D3D310511F40C9405
:103F9000D6280C946C2E2C3281E0380711F40C9446
:103FA00017292D32314011F40C943B290C946C2EBE
:103FB000253FA1E03A0711F40C94152E08F044C0F7
:103FC0002239E1E03E0711F40C94B02CF0F42336D2
:103FD00041E0340711F40C94232E38F42F32314091
:103FE00011F40C94412A0C946C2E203991E039077D
:103FF00011F40C94AD2C2139314011F00C946C2E3D
:1040000081E00E94D7990C946C2E243AB1E03B07D2
:1040100011F40C94B42C48F42A39314011F00C946A
:104020006C2E0E947EC70C946C2E2C3A41E0340713
:1040300011F40C941A2D243F314011F00C946C2E85
:104040000E94FE370C946C2E233583E0380711F460
:104050000C94202EE8F4273FA1E03A0711F40C94C9
:104060001D2E10F40C941A2E2939E2E03E0709F4B3
:1040700089C72A39324011F00C946C2E15E4E12ED8
:1040800015E1F12E0DEF12E083E0D82ED00EEDC732
:10409000283743E0340711F40C943A2E48F42935BC
:1040A000334011F00C946C2E0E9432C60C946C2E8E
:1040B000203A93E0390709F429C1273E334011F42F
:1040C0000C943F2E0C946C2E80E50E94C030882307
:1040D00061F00E9452316B017C01BB24B394672BC9
:1040E000682B692B31F4B12C04C0B12CC12CD12C1C
:1040F000760183E50E94C030882399F00E948631C2
:104100006B017C01B1100FC0672B682B692B59F430
:10411000F8018081882339F061E0C8010E943B8268
:1041200007C0BB20A9F360E087ED92E00E942682E1
:1041300081E0809396060E9479B00E949D32C1145E
:10414000D104E104F104E9F08091A2069091A30664
:10415000A091A406B091A506C80ED91EEA1EFB1EAA
:104160000E94847DDC01CB018C199D09AE09BF0939
:10417000B7FF1AC0809196068823B1F00E949B5623
:10418000EFCF80919606882319F00E949B56F9CFB5
:104190008091300C60E0882319F088EC92E002C036
:1041A00088EB92E00E942682109296060C946C2E68
:1041B00084918F010F5F1F4F882321F00E94A83246
:1041C000F801F6CF1092B60E1092B50E40E050E016
:1041D000BA0181E69CE00E94D6738BE1E1E6FCE047
:1041E000DE01159601900D928A95E1F780915F0CA2
:1041F0009091600C9C838B838FED93E09A838983ED
:1042000040E050E0BE016F5F7F4F83EB94E00E947F
:10421000E99ECE0101960E944056E1EFF2E08491C2
:104220008F010F5F1F4F882311F40C946C2E0E9496
:10423000A832F801F4CF0E94D0A80C946C2E1092F2
:10424000300C1092310C0C946C2E0E94CB9E0E946C
:104250008AAA0C946C2E81E0809374088093940B4E
:104260001092300C0C946C2E8091310C882311F438
:104270000C946C2E83E50E94C03081110C946F2E3B
:104280000C946C2E8091310C882351F1E1E1F3E024
:1042900084918F010F5F1F4F882321F00E94A83265
:1042A000F801F6CF6091AC0E7091AD0E8091AE0E1C
:1042B0009091AF0E4AE00E94D5328FE20E94A83260
:1042C0006091A80E7091A90E8091AA0E9091AB0EEC
:1042D0004AE00E94D5328AE00E94A8320C946C2EEB
:1042E000E3E2F3E084918F010F5F1F4F882311F405
:1042F0000C946C2E0E94A832F801F4CF0E9454BF97
:104300000C946C2E0E940FBE0C946C2E81E0809356
:104310002F0C40E060E0C8010E941EA10C946C2E9E
:104320000E9465BE0C946C2E0E94B5BD0C946C2E40
:104330000E948AAA0C946C2E80917508843010F02B
:104340000C946C2E8091C10491E0980F9093C1045D
:10435000913061F4909374089093940B8E5F8093E6
:10436000C1040E94A8328AE00E94A8321092740808
:104370000C946C2EE4E3F3E084918F010F5F1F4FE8
:10438000882321F00E94A832F801F6CF0E94D1A71D
:104390000C946C2E88E690E00E94633681110C9498
:1043A0006C2E8091E41383FF02C00C946C2E83E585
:1043B0000E94C030882361F10E945D310E94B6E600
:1043C00070938108609380080E945D3120E030E0A6
:1043D0004AEA52E40E945AED18163CF00E94D1A716
:1043E00060E084E593E00E9426820E945D31209186
:1043F0009E0830919F084091A0085091A1080E940A
:10440000A1E718162CF460E089E493E00E9426826C
:104410000E94BADF0C946C2E8EE40E94C030882378
:1044200011F40C946C2E0E9447316093D715709351
:10443000D8158093D9159093DA150C946C2E83E5DA
:104440000E94C030882319F00E94D33001C080E060
:104450008093E413E1E4F7E184918F010F5F1F4F34
:10446000882321F00E94A832F801F6CFE2E7F3E0BA
:1044700084918F010F5F1F4F882321F00E94A83283
:10448000F801F6CF8091E4138823A1F144E6C42E0D
:1044900043E0D42EE12CF12C20E08091E41390E055
:1044A0000E2C02C0959587950A94E2F780FF17C0FD
:1044B000BB24B394B20E222319F08CE20E94A832DE
:1044C000F60125913491F901849189010F5F1F4F05
:1044D000882321F00E94A8329801F5CF2B2DFFEF01
:1044E000EF1AFF0A32E0C30ED11C45E0E416F104D6
:1044F000A1F60CC0EEE6F3E084918F010F5F1F4F31
:10450000882321F00E94A832F801F6CF8AE00E94A9
:10451000A8320C946C2E10921C020C946C2E89E71D
:1045200093E00E9459568091E41383FF02C00C94DB
:104530006C2E83E50E94C030882311F40C946C2EFD
:104540000E945D310E94B6E670937F0860937E08FA
:104550000C946C2E89E690E00E94633681110C94D5
:104560002E30E2E8F3E084918F010F5F1F4F882324
:1045700021F00E94A832F801F6CF0E949BC88AE081
:104580000E94A8320C942E308DE690E00E94633693
:1045900081110C946C2E8091E41383FF02C00C9463
:1045A0006C2E83E50E94C0308AAB811105C082E584
:1045B0000E94C0308823B1F10E945D310E94B6E6AE
:1045C00070938108609380080E945D3120E030E0A4
:1045D0004AEA52E40E945AED181614F40C947F2E05
:1045E0000E94D1A760E085EA93E00E942682609154
:1045F000800870918108072E000C880B990B0E948F
:1046000060ED20919E0830919F084091A008509144
:10461000A1080E94A1E718162CF460E08AE993E053
:104620000E9426820E94BADF81E080931C021EAAAB
:104630001FAA18AE19AE1EA61FA618AA19AA1AA656
:104640001EAE5CE35AAF8CE123968FAF239796E4BE
:1046500028969FAF2897C12CD12C20E8E22E3FEB63
:10466000F32E812C912C5401609180087091810867
:10467000072E000C880B990B0E9460ED162F072F58
:10468000782E692E262F372F482F592FB601C701B4
:104690000E945AED882321F120919E0830919F08B5
:1046A0004091A0085091A108612F702F872D962D61
:1046B0000E945AED881F8827881F8AA7AAA9AA23C3
:1046C00099F0882389F080911C02882311F40C94BE
:1046D0006C2E60E085E893E00E9426820C946C2E9C
:1046E0001C2D0D2D7E2C6F2C0E94847D6B017C0176
:1046F000DC01CB012EA53FA548A959A9821B930B2C
:10470000A40BB50BB7FD45C0D701C60188519C4F1E
:10471000AF4FBF4F8EA79FA7A8ABB9AB0E949BC856
:10472000E6E9F3E084912F019FEF491A590A8823A3
:1047300021F00E94A832F201F5CF81149104A10466
:10474000B104D1F0D501C401805F984DAF4FBF4F88
:10475000BC01CD016C197D098E099F0928EE33E05B
:1047600040E050E00E9435F1CA01B9010E94563381
:104770008AE00E94A8320DC0E3E9F3E084912F01A2
:10478000AFEF4A1A5A0A882321F00E94A832F20198
:10479000F5CF0E949B560E949D3220909E0830903B
:1047A0009F084090A0085090A1089101A201612F9C
:1047B000702F872D962D0E9458E59F7781149104C4
:1047C000A104B10449F420E030E040E85FE30E9436
:1047D0005AED87FF0BC008C020E030E040E450E411
:1047E0000E94A1E7181614F446015701BAA5BB238D
:1047F000B9F12EA93FA948AD59AD211531054105A3
:10480000510541F0D701C601821B930BA40BB50BD8
:10481000B7FD26C09101A2016EAD7AAD23968FAD92
:10482000239728969FAD28970E9458E520E030E016
:1048300040EC5FE30E945AED87FD45CFD701C601EA
:10484000805A9541AF4FBF4F8EAB9FABA8AFB9AF6A
:104850002EAE3AAE23964FAE239728965FAE28979A
:1048600080911C02882309F42ECF81149104A104A5
:10487000B10429F4C12ED02EE72CF62CF5CE90E110
:10488000C91A97E2D90AE108F108C818D908EA0854
:10489000FB08F7FE18CFEECF0E9423C90C946C2EB4
:1048A0000E9475C80C946C2E0E9466C80C946C2EE5
:1048B0000E94F9B70E9479B00E94485610927D0874
:1048C00010927C0868EE73E080E090E00E944C7DDE
:1048D00060E085EB93E00E9426820E9479520C945E
:1048E0006C2E81E08093BC040C946C2E0E9415C841
:1048F0000C946C2E83E50E94C030882311F40C9434
:104900006C2E0E9486316093A6067093A706809352
:10491000A8069093A9060C946C2E8DEFC82E82E009
:10492000D82E97EFE92E98E0F92E10E0D6018D9160
:104930006D010E94C030882309F46DC0133009F066
:1049400063C00E945D314B015C0120E030E040EA31
:1049500051E40E945AED87FF4EC0A5019401609179
:1049600003097091040980910509909106090E943C
:1049700045E62B013C019B01AC016091430970911C
:10498000440980914509909146090E94BFED6093CA
:104990004309709344098093450990934609A30104
:1049A0009201609133097091340980913509909199
:1049B00036090E94BFED60933309709334098093E8
:1049C00035099093360960915C0970915D09809179
:1049D0005E0990915F090E945EEDA30192010E9421
:1049E000BFED0E94BCE660935C0970935D09809303
:1049F0005E0990935F098092030990920409A09246
:104A00000509B092060907C00E945D31F701608375
:104A10007183828393831F5FF4E0EF0EF11C1430E7
:104A200009F084CF0E94E0880C946C2E0E94B7C7D6
:104A30000C946C2E60E0C8010E943B820C946C2E9A
:104A400084918F010F5F1F4F882321F00E94A832AD
:104A5000F801F6CFEBEDF3E084918F010F5F1F4F6C
:104A6000882321F00E94A832F801F6CF649903C090
:104A70000BE114E002C000E214E0D8018D918D0139
:104A8000882319F00E94A832F8CF8AE00E94A83249
:104A9000E3EDF3E084918F010F5F1F4F882321F036
:104AA0000E94A832F801F6CF8091030180FD03C077
:104AB0000BE114E002C000E214E0F80181918F01E3
:104AC000882319F00E94A832F8CF8AE00E94A83209
:104AD000EBECF3E084918F010F5F1F4F882321F0EF
:104AE0000E94A832F801F6CF4B9903C00BE114E005
:104AF00002C000E214E0D8018D918D01882319F0E5
:104B00000E94A832F8CF8AE00E94A832E3ECF3E0DA
:104B100084918F010F5F1F4F882321F00E94A832DC
:104B2000F801F6CF4A9903C00BE114E002C000E29D
:104B300014E0F80181918F01882309F4E7CC0E94E9
:104B4000A832F7CF81E080932902809343150C941B
:104B50006C2E10922902109243150C946C2E83E552
:104B60000E94C0308823F9F00E943A31182F823019
:104B7000D8F0EAEFF5E184918F010F5F1F4F882392
:104B800021F00E94A832F801F6CFEDEFF3E0849116
:104B90008F010F5F1F4F882311F40C946C2E0E941D
:104BA000A832F801F4CF10E088E40E94C0308823D6
:104BB000B1F00E943A31E12FF0E08A3A91053CF0E1
:104BC000853021E092072CF084E091E002C08AEA6F
:104BD00090E0EE0FFF1FEA57F74F9183808386E442
:104BE0000E94C0308823A1F00E943A31E12FF0E00A
:104BF000EE0FFF1FE657F74F8F3F910519F014F0A6
:104C00008FEF90E097FF02C080E090E09183808377
:104C100082E40E94C030882311F40C946C2E0E9410
:104C20003A31E12FF0E08530910534F08838910574
:104C30002CF087E890E002C085E090E0EE0FFF1FC7
:104C4000EE57F74F918380830C946C2E88EC90E0A4
:104C50000E94633681110C946C2E84E40E94C03053
:104C6000882311F40C946C2E0E945D3111E020E039
:104C700030E0A9010E945AED811101C010E01093AB
:104C80004B09112359F10091B80410E00E945D31E5
:104C9000000F111F000F111FF801E85BFD4F60832B
:104CA00071838283938320E030E0A9016091480200
:104CB0007091490280914A0290914B020E945AEDF4
:104CC00081110CC080E090E0A0E4B0E48093480241
:104CD00090934902A0934A02B0934B020E94E3547E
:104CE000FBC7D8018D918D010E94C030882349F007
:104CF0000E945D310E94BCE6F7016083718382836C
:104D00009383F4E0EF0EF11CD012EBCF0E94768873
:104D1000E3C747E2E42E49E0F42E0DEF12E054E041
:104D2000D52ED00ED8018D918D010E94C0308823E0
:104D300039F00E945D31F701608371838283938330
:104D4000F4E0EF0EF11CD012EDCFC6C783E50E9450
:104D5000C0308823D9F00E945D31AB01BC01409383
:104D60004709509348096093490970934A09409351
:104D70000709509308096093090970930A0989E7A4
:104D800094E00E9427378AE00E94A83280E50E94C2
:104D9000C030882399F00E945D31AB01BC01409383
:104DA0004709509348096093490970934A098CE573
:104DB00094E00E9427378AE00E94A83282E50E9490
:104DC000C030882399F00E945D31AB01BC01409353
:104DD0000B0950930C0960930D0970930E098DE334
:104DE00094E00E9427378AE00E94A83284E50E945E
:104DF000C030882309F470C70E945D31AB01BC014B
:104E000040930709509308096093090970930A09B0
:104E10008FE194E00E9427378AE00E94A8325CC7A5
:104E200083E50E94C030882351F00E945D31609379
:104E3000230970932409809325099093260984E51A
:104E40000E94C030882351F00E945D3160931F0999
:104E500070932009809321099093220982E40E9493
:104E6000C030882351F00E945231609351157093E5
:104E70005215809353159093541588E50E94C030C5
:104E8000882351F00E945D3160933709709338098F
:104E90008093390990933A0989E50E94C0308823AC
:104EA00051F00E945D3160933B0970933C098093FF
:104EB0003D0990933E098AE50E94C030882351F055
:104EC0000E945D3160933F097093400980934109CE
:104ED0009093420985E40E94C030882309F4FCC6FF
:104EE0000E945D31609343097093440980934509A2
:104EF00090934609F1C69DEFA92E92E0B92E2FEFAF
:104F0000C22E2EE0D22E32EEE32E3EE0F32E00E053
:104F100010E0D5018D915D010E94C030882311F110
:104F20000E945D312B013C01F701208131814281DA
:104F300053810E9458E59B01AC01D6016D917D9192
:104F40008D919C910E9459E5F60160837183828363
:104F50009383D7014D925D926D927C921397C80115
:104F60000E94CD9B0F5F1F4FB4E0CB0ED11CE4E03D
:104F7000EE0EF11C0330110561F60E940E320E9404
:104F8000B7C7AAC68CE40E94C030882351F00E94A3
:104F90005D3160939502709396028093970290938F
:104FA000980282E50E94C030882351F00E945D3152
:104FB0006093990270939A0280939B0290939C0253
:104FC00083E50E94C030882351F00E945D316093D8
:104FD000EF027093F0028093F1029093F20281E469
:104FE0000E94C030882351F00E945D316093EA0B2B
:104FF0007093EB0B8093EC0B9093ED0B82E40E948B
:10500000C030882351F00E945D316093E20B7093B1
:10501000E30B8093E40B9093E50B83E40E94C03094
:10502000882351F00E945D316093DA0B7093DB0BA3
:105030008093DC0B9093DD0B2091950230919602CA
:1050400040919702509198026091990270919A0252
:1050500080919B0290919C020E94F55D3DC6F4E018
:10506000EF0EF11CD01609F437C6D8018D918D01D1
:105070000E94C030882399F30E945D31F70160835C
:10508000718382839383EBCF84918F010F5F1F4FD6
:10509000882321F00E94A832F801F6CFE5ECF4E075
:1050A00084918F010F5F1F4F882321F00E94A83247
:1050B000F801F6CFE1ECF4E084918F010F5F1F4F10
:1050C000882321F00E94A832F801F6CFE9EBF4E042
:1050D00084918F010F5F1F4F882321F00E94A83217
:1050E000F801F6CF40911002509111026091120226
:1050F0007091130287EB94E00E94273740911402CD
:1051000050911502609116027091170284EB94E0A1
:105110000E942737409118025091190260911A029B
:1051200070911B0281EB94E00E942737E9EAF4E0DA
:1051300084918F010F5F1F4F882321F00E94A832B6
:10514000F801F6CF409104025091050260910602E9
:105150007091070287EA94E00E9427374091080285
:105160005091090260910A0270910B0284EA94E066
:105170000E94273740910C0250910D0260910E025F
:1051800070910F0281EA94E00E9427378AE00E9422
:10519000A832A2C583E5F4D7882309F49DC50E94EF
:1051A0003A319093A1028093A00296C58DED90E0D4
:1051B0000E946336811190C583E5E2D7882309F404
:1051C0008BC50091B80410E00E943A31000F111F06
:1051D000F801EE5BFD4F918380837EC580E5D0D7DB
:1051E000882309F479C50E943A318C0183E5C8D738
:1051F000882321F00E943A317C0103C0EE24EA9416
:10520000FE2CC7010196039708F066C517FD64C51B
:10521000E1E0F3E0C801992721913191281739077E
:1052200009F45AC523E0E135F207B1F7EFC683E58B
:10523000A7D7882319F00E942D3102C084E091E0A5
:1052400099A388A380E59CD7882349F00E942D313B
:10525000893833E1930728F088E893E102C088EEAB
:1052600093E09A838983BE01605E7F4FCE010196F1
:105270000E9417AA31C585E483D781110FC080E54C
:105280007FD7882391F00E945D3160932A0270934A
:105290002B0280932C0290932D0207C0EBD7181697
:1052A00019066CF7EAEFF5E16EC089E469D7882347
:1052B00081F00E945D312CE933E549E45EE30E9410
:1052C000BFED609332027093330280933402909367
:1052D000350284E455D7882379F0EFD72CE933E5FC
:1052E00049E45EE30E9445E660932E0270932F022C
:1052F0008093300290933102E1E4F7E184918F01D1
:105300000F5F1F4F882321F00E94A832F801F6CFCB
:1053100040912A0250912B0260912C0270912D0233
:105320008DED94E00E9427372CE933E549E45EE3F4
:105330006091320270913302809134029091350273
:105340000E9445E6AB01BC0189ED94E00E940C3758
:105350002CE933E549E45EE360912E0270912F025F
:1053600080913002909131020E94BFEDAB01BC01EF
:1053700085ED94E00E940C378AE00E94A832ACC40C
:105380000E94A832F80184918F010F5F1F4F811195
:10539000F7CF06E314E0D8018D918D01882309F43D
:1053A000B5C80E94A832F7CF83E5EAD6082F882334
:1053B00099F083D760934C0270934D0280934E0214
:1053C00090934F0211E020E030E0A9010E945AEDD5
:1053D000811110E010934F0980E5D2D6182F882351
:1053E000A1F020E030E0A90160914C0270914D02E3
:1053F00080914E0290914F020E945AED882311F045
:1054000001D7182F10934F0967C4011165C4E1E457
:10541000F7E184918F010F5F1F4F882321F00E94D5
:10542000A832F801F6CF80914F09811103C06AE2DA
:1054300074E002C06DE174E086EF94E00E94AF3248
:1054400020E030E040E05FE360914C0270914D025B
:1054500080914E0290914F020E9459E50E94B6E65B
:1054600085EE94E00E944C36E1EEF4E084918F01E9
:105470000F5F1F4F882309F42FC40E94A832F80140
:10548000F5CF85E47DD6882319F0F4D67C0102C0DF
:10549000E12CF12C83E474D6882331F0EBD6AA9664
:1054A0009FAF8EAFAA9706C0E5E0F0E0AA96FFAFE7
:1054B000EEAFAA9785E564D6882329F0A3D6AB96EC
:1054C0008FAFAB9703C0AB961FAEAB9783E558D6B3
:1054D000882331F0F2D66AAB7EA78EAF9AAF08C0B0
:1054E0001AAA1EA6F7FC0AC0F6E1FEAF23E42AAF13
:1054F000E114F10439F41092B80404C03CE83EAF62
:1055000042E44AAF0E94847D4B015C01EF2819F40C
:1055100007E414E00CC00AE514E0D8018D918D0178
:10552000882311F40C9486220E94A832F6CFF80149
:1055300081918F01882319F00E94A832F8CF8AE068
:105540000E94A8320E94F9B78FE78093E71381E0A9
:1055500080931C02A4968CAE9DAEAEAEBFAEA49757
:10556000AF968CAE9DAEAEAEBFAEAF9728961FAED7
:105570002897F0E42796FFAF27972CE12C962FAFC2
:105580002C9736E460963FAF609761961FAE6197A7
:1055900065961FAE659766961FAE669767961FAEB7
:1055A00067976F961CAE1DAE1EAE1FAE6F976B96C3
:1055B0001CAE1DAE1EAE1FAE6B97C12CD12C76015A
:1055C000FFE74F2E512C612C712C8FE790E0A0E06B
:1055D000B0E08EAB9FABA8AFB9AFA8961CAE1DAE26
:1055E0001EAE1FAEA89791E0A0969FAFA0972496FD
:1055F0001FAE1EAE249710E000E0312C212C8091CC
:105600001C02882309F4A2C10E94847D6AA77BA79B
:105610008CA79DA78091E513882309F4B9C00E9447
:10562000C3BA10919E0800919F083090A008209066
:10563000A108212F302F432D522D61966FAD619718
:1056400065967FAD659766968FAD669767969FADB9
:1056500067970E945AED87FF0CC061961FAF619754
:1056600065960FAF659766963FAE669767962FAEC5
:105670006797212F302F432D522D28966FAD2897F5
:1056800027967FAD27972C968FAD2C9760969FAD70
:1056900060970E94A1E7181664F428961FAF289718
:1056A00027960FAF27972C963FAE2C9760962FAE7C
:1056B0006097A096AFADA0972AA93EA54EAD5AAD72
:1056C000612F702F832D922DAA2309F447C00E94C9
:1056D000A1E718160CF05CC04AA55BA56CA57DA5DA
:1056E000481959096A097B09DB01CA0188589341A5
:1056F000A109B109B7FD4CC08EA99FA9A8ADB9AD4C
:1057000084199509A609B709B595A7959795879521
:105710008093E713A8964CAF5DAF6EAF7FAFA897AD
:10572000BAA96196BFAF6197EEA56596EFAF659791
:10573000FEAD6696FFAF66972AAD67962FAF679767
:105740008AA59BA5ACA5BDA5A4968CAF9DAFAEAF19
:10575000BFAFA497A0961FAEA0971AC00E945AEDA3
:1057600087FF16C08AA59BA5ACA5BDA5A4962CADA8
:105770003DAD4EAD5FADA497821B930BA40BB50B53
:10578000AC01BD01485853416109710977FFBBC2A3
:1057900020E030E040EA51E46AA97EA58EAD9AADE2
:1057A0000E9459E59B01AC01612F702F832D922D32
:1057B0000E94A1E7181664F4E3ECF5E084918F01F0
:1057C0000F5F1F4F882309F487C2C2D6F801F6CFB6
:1057D00080E398EFAFEFBFEFAF962CAD3DAD4EAD90
:1057E0005FADAF97821B930BA40BB50B2AA53BA50E
:1057F0004CA55DA5820F931FA41FB51FB7FD0EC05A
:105800000E949BC88AE0A4D68AA59BA5ACA5BDA58D
:10581000AF968CAF9DAFAEAFBFAFAF978AA59BA53C
:10582000ACA5BDA5880F991FAA1FBB1FA4962CADC0
:105830003DAD4EAD5FADA497821B930BA40BB50B92
:1058400088199909AA09BB0981389F44A241B10569
:1058500060F0E5EAF5E084918F010F5F1F4F882328
:1058600009F43AC275D6F801F6CF24964EAD5FAD75
:105870002497AA968EAD9FADAA97841795070CF032
:1058800062C0E8E4F5E084918F010F5F1F4F882329
:1058900019F05ED6F801F7CFB701A60183E395E0D2
:1058A0000E9427378AE054D66B964CAD5DAD6EAD45
:1058B0007FAD6B978EE195E00E9427378AE048D64E
:1058C0006F964CAD5DAD6EAD7FAD6F9789E095E0A5
:1058D0000E9427378AE03CD6AB969FADAB979923C1
:1058E00009F4FAC1C0922A02D0922B02E0922C0253
:1058F000F0922D022CE933E549E45EE36B966CAD42
:105900007DAD8EAD9FAD6B970E94BFED609332026F
:105910007093330280933402909335022CE933E57F
:1059200049E45EE36F966CAD7DAD8EAD9FAD6F9734
:105930000E9445E660932E0270932F0280933002FE
:1059400090933102C9C10E94795259CE80911C02B4
:105950008111C2C10E94F9B7BFC10E9479B0BCC118
:1059600080E00E94D799B8C183E50AD4882379F0F2
:1059700049D4182F0E94E6A5811110E080912E05D0
:10598000811101C010E0812F0E94AC9701C010E08E
:10599000F0904E09111103C0E1E4F7E118C0F110D5
:1059A000FBCFEAEFF5E184918F010F5F1F4F882352
:1059B00019F0CED5F801F7CFE4E6F6E084918F0137
:1059C0000F5F1F4F882341F3C3D5F801F7CF8491B0
:1059D0008F010F5F1F4F882319F0BAD5F801F7CF59
:1059E000F11003C062E374E002C06EE274E086E589
:1059F00096E0B5D58AE0ACD586E5C2D3882309F414
:105A00006BC18091770690917806892B39F080914F
:105A10002E05882319F00E9406975EC1E7E3F6E0A1
:105A200084918F010F5F1F4F882309F455C190D5D2
:105A3000F801F6CF8FEF282E8EE0382EA2EEBEE0D2
:105A4000BBA7AAA7E5E9FBE0FFABEEAB00E010E0E7
:105A50002EA93FA925593B403BAB2AABAEA9BFA914
:105A60008D91BFABAEAB882309F4ABC0F801EC5FFE
:105A7000FD4F2081318142815381F801E05FFD4F6C
:105A800060817181828193810E9459E520E030E03C
:105A900040E05FE30E94BFED9B01AC01F10160813A
:105AA0007181828193810E94A1E718162CF4C801AC
:105AB0008154994FF2D403C060E070E0CB01D10172
:105AC0004D905D906D907C90EAA5FBA5C080D18043
:105AD000E280F380A70196010E9459E5F801EA529D
:105AE000F14F20813181428153810E9459E59B0110
:105AF000AC01C301B2010E9458E54B015C0120E0FA
:105B000030E040EA51EC0E94A1E718166CF520E065
:105B100030E040EA51E4C501B4010E945AED87FF2C
:105B200023C0A5019401C701B6010E9458E54B01AD
:105B30005C01A70196010E9458E59B01AC01C301DD
:105B4000B2010E9459E5D1016D937D938D939C9391
:105B50001397EAA5FBA580829182A282B3828AA9CB
:105B60009BA90E94CD9B2DC0EAEFF5E184918F01A6
:105B70000F5F1F4F882319F0EBD4F801F7CFE1EA4C
:105B8000F6E084918F010F5F1F4F882319F0E0D456
:105B9000F801F7CF61E083E996E00E9426820E9437
:105BA000607088E290E09A83898388EC90E099A302
:105BB00088A3BE016F5F7F4FCE0180960E9417AA17
:105BC0008BC0F4E02F0E311C0C5F1F4F2AA53BA5A4
:105BD0002C5F3F4F3BA72AA70C30110509F038CFA7
:105BE0001DD40E94B7C760E083E896E00E94268239
:105BF00083E992E099A388A308EC10E01A83098353
:105C0000BE01605E7F4FCE0101960E9417AA8AEB0B
:105C100092E099A388A31A830983BE01605E7F4F37
:105C2000CE0101960E9417AA57C00E94643A0E94B2
:105C3000069752C00E9462D44FC00E9473C74CC0E6
:105C40000E947AC549C0EAEFF5E184918F010F5FA8
:105C50001F4F882319F07CD4F801F7CFEBECF6E066
:105C600084918F010F5F1F4F882309F435C070D4D2
:105C7000F801F6CFF894E0E0F0E019952DC081E04E
:105C80008093AB021092E60883E57AD2882309F468
:105C9000A6C1B8D2811120C0A2C12093EE0EE1E4CA
:105CA000F7E184918F010F5F1F4F882319F050D4C3
:105CB000F801F7CF6091EE0E70E08AED96E0ECD738
:105CC0008AE046D409C06F2D7E2D8CEE96E047D435
:105CD00082E23ED48AE03CD40E94E164BFC1D7D2C4
:105CE000AB01BC014093AC0E5093AD0E6093AE0E71
:105CF0007093AF0E8BEF9DE00E94D673EDCF0E94A4
:105D00008AAA0C94F72224964EAD5FAD2497141600
:105D100015060CF034C1A8968CAC9DACAEACBFACF3
:105D2000A897880E991EAA1EBB1EA8962CAD3DAD45
:105D30004EAD5FADA897281B390B4A0B5B0BCA0110
:105D4000B901A30192010E9426F1A50194010E94CC
:105D500057F14EA85FA868AC79AC420E531E641E82
:105D6000751E34E143165104610471040CF14CEECC
:105D700044165104610471043CF450E84516510482
:105D8000610471041CF105C05BEE452E512C612CA1
:105D9000712C4EAA5FAA68AE79AE8EEF90E0A0E0BB
:105DA000B0E084199509A609B7092C013D0112C07C
:105DB00024E130E040E050E02EAB3FAB48AF59AFBC
:105DC00044E1442E512C612C712C04C04EAA5FAAD0
:105DD00068AE79AE4EA95FA968AD79AD8FE296E065
:105DE0000E949CD8B301A2018AE296E00E949CD84E
:105DF00028964FAD289727965FAD27972C966FADC5
:105E00002C9760967FAD609783E296E00E942737DB
:105E100061964FAD619765965FAD659766966FAD7C
:105E2000669767967FAD67978CE196E00E9427376B
:105E300024964EAD5FAD2497433051050CF49FC0BE
:105E4000C301B2010E9460ED20E030E040E850E480
:105E50000E94BFED6B017C0128962FAD28972796F5
:105E60003FAD27972C964FAD2C9760965FAD60970E
:105E700061966FAD619765967FAD659766968FADBC
:105E8000669767969FAD67970E9458E52BED3FE0B8
:105E900049E450E40E94BFED20E030E040E05FE3E1
:105EA0000E94BFED9B01AC01C701B6010E9445E60F
:105EB0006B017C01C501B4010E9460ED2FE632E167
:105EC00043E85AE30E94BFED4B015C01B701A60114
:105ED00086E196E0BCD7B501A40180E196E0B7D792
:105EE0002AE939E949E15FE3C701B6010E94BFED44
:105EF0006B017C019B01AC010E9459E5A501940155
:105F00000E9445E66B966CAF7DAF8EAF9FAF6B97EF
:105F1000A5019401C701B6010E94BFED20E030E069
:105F200040E05EE30E94BFED6F966CAF7DAF8EAF39
:105F30009FAF6F97E0E0F6E084915F015FEFA51AF5
:105F4000B50A882319F004D3F501F6CFB701A601ED
:105F50008AEF95E07CD76B964CAD5DAD6EAD7FADB5
:105F60006B9784EF95E073D76F964CAD5DAD6EADDA
:105F70007FAD6F978EEE95E06AD78AE0E9D28EA961
:105F80009FA9A8ADB9AD840D951DA61DB71DB595EA
:105F9000A795979587958093E71324968EAD9FAD2F
:105FA0002497019624969FAF8EAF24979AA928969E
:105FB0009FAF2897AEA52796AFAF2797BEAD2C967B
:105FC000BFAF2C97EAAD6096EFAF60978AA49BA411
:105FD000ACA4BDA4F1E0A096FFAFA097D9CB1092DE
:105FE000D7151092D8151092D9151092DA150E9473
:105FF00071D872CEE1E4F7E184918F010F5F1F4FFA
:10600000882309F460CEA4D2F801F6CF0E9479B0BB
:10601000D02E60E0802F0E94497CFFEFEF16FF0634
:1060200059F4802F0E947ADA31E020E0892B09F0C0
:1060300030E0032F122F05C0EA94EF2861F000E052
:1060400010E08D2D0E947ADA8017910709F444CE72
:106050000E949B56F6CF01E010E0F3CFCE58DF4F01
:106060000FB6F894DEBF0FBECDBFDF91CF911F9169
:106070000F91FF90EF90DF90CF90BF90AF909F90E7
:106080008F907F906F905F904F903F902F900895EA
:1060900020912B0530E0F901EE52F94F80832F5FFC
:1060A0003F4F2370332720932B05809175088F5F16
:1060B0008093750808958FB7F8949091D615209124
:1060C000D515291759F0E92FF0E0EB5AFA4E208147
:1060D00030E09F5F9F779093D61502C02FEF3FEF80
:1060E0008FBFC90108950F931F93CF93DF93EC01E6
:1060F0000E94847D0E811F81288539850115110537
:106100002105310559F52C852223A9F13A85215025
:106110002C8721E0230F2A874D85241301C01A867E
:10612000FE0124E0329FE00DF11D11240685178544
:10613000208931890A831B832C833D83DC01CB01B9
:10614000800F911FA11DB11D8E839F83A887B987E2
:106150008C819D81892B79F0409A0DC0DC01CB01A7
:10616000801B910BA20BB30BB7FD05C040981E829C
:106170001F8218861986DF91CF911F910F91089584
:10618000682F880F770B8091BF049091C0040E9404
:1061900085E89C01909322148093211481E0232BA5
:1061A00009F480E0089580912114909122144AE02E
:1061B00050E060E070E001960E947BEA97FD1EC00F
:1061C00080912114909122144AE050E060E070E048
:1061D00001960E947BEA6F3F71058105910509F0E8
:1061E0007CF480912114909122144AE050E060E008
:1061F00070E001960E947BEA862F089580E0089562
:106200008FEF0895E0912114F0912214818121E013
:1062100030E0803239F42F5F3F4FDF01A20FB31F10
:106220008C91F7CF8D3211F08B3231F42F5F3F4FCD
:10623000DF01A20FB31F8C918E3219F4E20FF31F0E
:10624000818180538A3030F4AEDF91E0811103C048
:1062500090E001C091E0892F0895809121149091E0
:1062600022144AE050E060E070E001960E94A3EB47
:10627000CB01089580912114909122144AE050E0BE
:1062800060E070E001960E947BEACB010895809166
:106290002114909122144AE050E060E070E00196F1
:1062A0000C947BEA80912114909122144AE050E0F2
:1062B00060E070E001960C94A3EB0F931F93CF93D3
:1062C000DF93C0912114D091221465E470E0CE01D7
:1062D0000E9485E88C01CE0101960115110541F45B
:1062E00060E070E0DF91CF911F910F910C9415E960
:1062F000F801108260E070E00E9415E925E4F801E1
:106300002083DF91CF911F910F910895D6DF20E078
:1063100030E04AE754E40E94BFED0C94BCE6CF9312
:10632000FC0180818B33A1F080917508843080F46A
:10633000C62FBF0180912B0520E6829FC00111244A
:106340008D50994F0E9499E88C2FA2DE81E001C008
:1063500080E0CF910895DF92EF92FF920F931F9309
:10636000CF93DF93CDB7DEB76E970FB6F894DEBF4D
:106370000FBECDBF6091920B7091930B61157105AB
:1063800009F14DE150E08E010F5F1F4FC8010E94DF
:1063900002ED1E8EF8017F01E01AF10AD190DD2096
:1063A00019F08AE0D812F7CFF801EE0DFF1D108228
:1063B00060E0C801B4DF882329F0C8010E941F569D
:1063C000811109C081E02091920B3091930B232B16
:1063D000B9F480E015C0DD2071F08FEFE81AF80AFB
:1063E0008091920B9091930BE80EF91EF092930B13
:1063F000E092920BE7CF1092930B1092920BE2CFA8
:106400006E960FB6F894DEBF0FBECDBFDF91CF9171
:106410001F910F91FF90EF90DF9008950C944BAA7D
:106420000F931F93CF93DF93CDB7DEB72C970FB6A3
:10643000F894DEBF0FBECDBFEFEFFEE08085918503
:10644000A285B38544815581668177810081118160
:106450002281338109831A832B833C834D835E839E
:106460006F83788789879A87AB87BC872BE03FE06B
:10647000AE01475F5F4FBE016B5F7F4FCE0101965C
:106480000E9403892C960FB6F894DEBF0FBECDBFD5
:10649000DF91CF911F910F910895FC016591759146
:1064A000859194910895FC01238121110C940F751D
:1064B00008950F931F93CF93DF93CDB7DEB72C973B
:1064C0000FB6F894DEBF0FBECDBF20914E09222338
:1064D00049F18C01CE0101962CE0FC0111922A9524
:1064E000E9F7F801408151816281738149835A83C0
:1064F0006B837C8344815581668177814D835E8384
:106500006F8378870E94A75E9B01AC01F8016085CC
:106510007185828593850E9459E5F80160877187AE
:10652000828793872C960FB6F894DEBF0FBECDBF3F
:10653000DF91CF911F910F9108950E94847D609308
:10654000A2067093A3068093A4069093A5060895CF
:106550009091C00095FFFCCF8093C60008950F93E3
:106560001F93CF93DF931F921F92CDB7DEB7FC012D
:1065700084918F010F5F1F4F811102C08B0107C0F3
:1065800069837A83E5DFF80169817A81F1CFF801C7
:1065900081918F01882311F0DBDFF9CF0F900F90ED
:1065A000DF91CF911F910F9108958F929F92AF929B
:1065B000BF92EF92FF921F93CF93DF93CDB7DEB7D9
:1065C000A0970FB6F894DEBF0FBECDBF6115710561
:1065D0008105910579F110E0842E912CA12CB12C2C
:1065E000EE24E394F12CEC0EFD1EE10EF11C17FDE0
:1065F000FA94A50194010E9435F1F7016083B90175
:10660000CA011F5F611571058105910549F7115098
:1066100010F1E1E0F0E0EC0FFD1FE10FF11D17FDBF
:10662000FA9580818A3010F097E301C090E3890FDA
:106630008FDFEDCF80E3A0960FB6F894DEBF0FBEDC
:10664000CDBFDF91CF911F91FF90EF90BF90AF90A2
:106650009F908F907DCFA0960FB6F894DEBF0FBEAF
:10666000CDBFDF91CF911F91FF90EF90BF90AF9082
:106670009F908F900895CF92DF92EF92FF92CF93E9
:10668000DF936A017B01FC018491EF01219688234D
:1066900019F05EDFFE01F8CF4AE0C701B601DF91D5
:1066A000CF91FF90EF90DF90CF907FCFCF92DF928E
:1066B000EF92FF926B017C0197FF0AC08DE248DFE9
:1066C000F094E094D094C094C11CD11CE11CF11C46
:1066D0004AE0C701B601FF90EF90DF90CF9065CF01
:1066E000EF92FF920F931F93CF93DF931F92CDB73B
:1066F000DEB7082F162FEAEFF5E184917F012FEF27
:10670000E21AF20A882329F0998322DFF70199819E
:10671000F4CFE02FF92F84917F019FEFE91AF90A56
:10672000882319F015DFF701F6CF6091D715709126
:10673000D8158091D9159091DA15B8DF8AE008DF75
:1067400011110E9471D810922905109228050F90FE
:10675000DF91CF911F910F91FF90EF9008952F92AD
:106760003F924F925F926F927F928F929F92AF92E1
:10677000BF92CF92DF92EF92FF920F931F93CF932E
:10678000DF931F92CDB7DEB7E6DD811171C2809134
:106790007508843058F42FB7F8948091D5159091EE
:1067A000D6152FBF891B8F7709F03DC18091300C22
:1067B000882309F45DC280917508811102C010928E
:1067C0002D05EE24E3944091AC0E5091AD0E6091F6
:1067D000AE0E7091AF0E8091A80E9091A90EA0916F
:1067E000AA0EB091AB0E481759076A077B0708F449
:1067F000E12C00E010E09924939480E6882E98E341
:10680000C92E98E0D92E24E3A22E28E0B22E3DE82E
:10681000732E80917508843008F02AC2E11028C2D6
:1068200080912D05811124C28091030E9091040E58
:10683000A091050EB091060E8093AC0E9093AD0E14
:10684000A093AE0EB093AF0E41E050E0BE016F5F7B
:106850007F4F8BEF9DE00E947677019719F4898135
:1068600090E002C08FEF9FEFF82EEE24E39420908B
:10687000AC0E3090AD0E4090AE0E5090AF0E4091E9
:10688000A80E5091A90E6091AA0E7091AB0E24161D
:10689000350646065706C8F4E12C8F3FEFEF9E07FA
:1068A00009F475C0FAE08F1709F48EC02DE0821745
:1068B00009F48AC083E2F81619F09AE3F91299C034
:1068C00080912C05811195C07AC0E3E5F8E08491B0
:1068D0002F012FEF421A520A882319F039DEF201F4
:1068E000F6CF0E9479B08BEF9DE00E940F758091EA
:1068F000160E882339F181508093160E789EC001C0
:10690000112441E061E0855E914F0E941EA1E0915B
:10691000160E84E0E89FF0011124E95EF14F4081FA
:106920005181628173814093AC0E5093AD0E6093A0
:10693000AE0E7093AF0E8BEF9DE00E94D6730E9457
:10694000CB9E15C01092300CD092930BC092920B3C
:1069500002DD0E94D1A70E94959E6D3371058105CD
:10696000910528F0B092930BA092920BF4DC109258
:10697000B40E8091310C882319F00E94A6A31FC089
:106980000E94D0A88091310C8111F7CF18C0EAEF96
:10699000F5E184912F019FEF491A590A882319F0D4
:1069A000D7DDF201F6CFE4E4F8E084912F012FEF78
:1069B000421A520A882319F0CBDDF201F6CF83E2A6
:1069C000F81202C090922D0510922C0501151105A8
:1069D00009F41FCF80912B05889E000D111D1124F5
:1069E000F801ED50F94F108280E052DB00E010E03A
:1069F00010CF0F35110508F00CCF9BE3F91202C040
:106A000090922C0580912C05811103CF80912B054C
:106A1000F801889EE00DF11D1124ED50F94FF08230
:106A20000F5F1F4FF6CE47DB2091280530912905D7
:106A30008A3019F08D3009F0EBC010922A0521152B
:106A4000310509F4A4CEF901E853FB4F10821092EE
:106A500029051092280528EC34E06901F9018081AC
:106A60002F5F3F4F8032C9F386018E3411F0C12C65
:106A7000D12C6AE270E0C8010E9485E85C01C11473
:106A8000D10409F475C06FE278E0C8010E9411EDED
:106A9000FF24F394892B11F4F12C09C06EE470E00B
:106AA000C80104960E9485E8009709F06C014AE04D
:106AB00050E060E070E0C60101960E947BEA6093BE
:106AC000C4047093C5048093C6049093C704409097
:106AD000D7155090D8156090D9157090DA15FFEF42
:106AE0004F1A5F0A6F0A7F0A6415750586059705B8
:106AF00031F0F11004C061E08CEF97E026C0A114E2
:106B0000B10401F180E0F12CF801E80FF11D908152
:106B10009A3219F08F5FF926F7CF4AE050E060E033
:106B200070E0C50101960E947BEACF2CD12CE12CAC
:106B3000F12C6C157D058E059F0549F061E08DED0A
:106B400097E003C061E083EB97E0CADD2FCE809130
:106B5000C4049091C504A091C604B091C704809369
:106B6000D7159093D815A093D915B093DA1506C010
:106B7000892B21F060E08FEF96E0E7CF8091AB02A8
:106B8000811122C067E470E0C8010E9485E8009787
:106B9000D9F04AE050E060E070E001960E947BEAA4
:106BA0006430710588F4ECE3F7E084917F012FEF06
:106BB000E21AF20A882319F0CBDCF701F6CF60E085
:106BC00082E397E00E94268263E874E0C8010E9495
:106BD00090E8892B21F410921C021092960668E826
:106BE00074E0C8010E9490E8892B21F489E297E0C3
:106BF0000E9459566DE874E0C8010E9490E8892B04
:106C000011F40E947EC761E088EC94E088DBBFCD80
:106C10002F3531050CF0BBCD8C35A9F42FB7F89486
:106C20008091D5159091D6152FBF891B8F7709F4C8
:106C3000AECD41DA90912A059111A9CD2091280578
:106C40003091290509C08B3319F491E090932A05FE
:106C500090912A0591119BCDA9014F5F5F4F5093F1
:106C6000290540932805F901E853FB4F80838FCD18
:106C70000F90DF91CF911F910F91FF90EF90DF90D8
:106C8000CF90BF90AF909F908F907F906F905F90CC
:106C90004F903F902F9008950F931F93CF93DF93C2
:106CA0008B01FC018491EF012196882319F050DCBF
:106CB000FE01F8CFB801110F880B990BDF91CF912E
:106CC0001F910F91F3CCEF92FF921F93CF93DF931D
:106CD0007C0184E555DA182F882311F164DA8823C2
:106CE000D1F0E1E4F7E18491EF012196882319F0D6
:106CF0002FDCFE01F8CF8DE42BDCB701FF0C880BF5
:106D0000990BD4DC50DA682F70E087E698E0C4DF96
:106D10008AE01EDC09C047DA8093B80410E004C0A2
:106D20008091EE0E8093B804812FDF91CF911F9157
:106D3000FF90EF9008958F929F92AF92BF92CF9263
:106D4000DF92EF92FF92CF936B017C01B42E20E093
:106D500030E0A9010E945AED87FF06C08DE2F8DB02
:106D6000F7FAF094F7F8F094C0E060E070E080E0AB
:106D70009FE3CB1541F02DEC3CEC4CEC5DE30E9425
:106D8000BFEDCF5FF6CF9B01AC01C701B6010E94FA
:106D900059E56B017C010E94BCE64B015C014AE0B5
:106DA00004DCCC2379F1C501B4010E945EED9B01A6
:106DB000AC01C701B6010E9458E56B017C018EE26F
:106DC000C7DB20E030E040E251E4C701B6010E9499
:106DD000BFED4B015C010E94B6E66B01770FEE0838
:106DE000FF08C701B60162DCC701B6010E9460ED71
:106DF0009B01AC01C501B4010E9458E56B017C0107
:106E0000C150F9F6CF91FF90EF90DF90CF90BF90F7
:106E1000AF909F908F900895CF92DF92EF92FF9264
:106E2000CF93DF936A017B01FC018491EF012196EE
:106E3000882319F08DDBFE01F8CF42E0C701B601CF
:106E4000DF91CF91FF90EF90DF90CF9074CFCF92F2
:106E5000DF92EF92FF92CF93DF936A017B01FC01F7
:106E60008491EF012196882319F072DBFE01F8CF9F
:106E700042E0C701B601DF91CF91FF90EF90DF9024
:106E8000CF9059CF1F920F920FB60F9211240BB6CD
:106E90000F922F933F938F939F93EF93FF932091A4
:106EA000C6009FB7F894E091D51581E08E0F8F77DB
:106EB0003091D615831731F0F0E0EB5AFA4E20836B
:106EC0008093D5159FBFFF91EF919F918F913F9137
:106ED0002F910F900BBE0F900FBE0F901F90189523
:106EE000DF92EF92FF920F931F93CF93DF937C017A
:106EF000EB01D0907E068B01040F151FF7018081F6
:106F000091810E9410F1D11001C0888320917C06EC
:106F100030917D06A901480F511D50937D06409385
:106F20007C06F7018081918101969183808321966F
:106F3000C017D10719F7DF91CF911F910F91FF90E3
:106F4000EF90DF900895AF92BF92DF92EF92FF92A1
:106F50000F931F93CF93DF9320917B06211144C0A1
:106F60008A017C01EB01060F171FC017D10709F436
:106F70003BC0F701A080B180D990C5010E9410F1FB
:106F8000D81609F16D2DC5010E9418F1C5010E94A6
:106F900010F18D15C1F0E1E4F7E18491EF01219644
:106FA000882319F0D5DAFE01F8CFEAE7F8E08491FA
:106FB000EF012196882319F0CBDAFE01F8CF81E0AA
:106FC00080937B0611C080917C0690917D068D0D8B
:106FD000911D90937D0680937C06F70180819181BD
:106FE000019691838083C1CFDF91CF911F910F9143
:106FF000FF90EF90DF90BF90AF9008958F929F9297
:10700000AF92BF92CF92DF92EF92FF920F931F93B6
:10701000CF93DF93CDB7DEB764970FB6F894DEBF9A
:107020000FBECDBF1D821E821F82188680E390E3B3
:10703000A0E3B0E089839A83AB83BC8384E690E0CD
:10704000988B8F8710927B0644E050E0BE016F5F03
:107050007F4FCE010F9677DF8F8598890296988BA8
:107060008F8710927D0610927C0681E08C8B41E028
:1070700050E0BE016C5E7F4FCE010F9664DF40E1B1
:1070800050E067EF78E0CE010F965DDF40E150E021
:1070900067E279E0CE010F9656DF40E150E06FE005
:1070A00079E0CE010F964FDF44E050E067E479E0ED
:1070B000CE010F9648DF44E050E06BE079E0CE016E
:1070C0000F9641DF44E050E067E079E0CE010F9693
:1070D0003ADF44E050E063E279E0CE010F9633DF1F
:1070E00044E050E06FE179E0CE010F962CDF44E000
:1070F00050E061E575E1CE010F9625DF40E150E0FB
:1071000067E379E0CE010F961EDF4CE050E062EEBF
:107110007EE0CE010F9617DF1B8A80914E098823EF
:1071200051F080912E05882331F0809144158823F9
:1071300011F084E08B8B1D821E821F82188683E0F3
:107140008A8B898B41E050E0BE016D5E7F4FCE019E
:107150000F96F9DE44E050E0BE016B5F7F4FCE0139
:107160000F96F1DE41E050E0BE016E5E7F4FCE0132
:107170000F96E9DE41E050E0BE016F5E7F4FCE0129
:107180000F96E1DE1AE0115044E050E039F0BE0104
:107190006B5F7F4FCE010F96D6DEF5CF64E472E0D1
:1071A000CE010F96D0DE1D821E821F8218861AE045
:1071B000115049F044E050E0BE016B5F7F4FCE01BB
:1071C0000F96C1DEF5CF80914415882341F189E007
:1071D0008B87898741E050E0BE01655F7F4FCE011C
:1071E0000F96B1DE41E050E0BE01675F7F4FCE01F8
:1071F0000F96A9DE44E050E067E776E0CE010F96F7
:10720000A2DE44E050E063E776E0CE010F969BDE1D
:1072100044E451E06FE275E0CE010F9694DE4CE05D
:1072200050E065E475E1CE010F968DDE44E050E05C
:1072300069E972E0CE010F9686DE44E050E065E930
:1072400072E0CE010F967FDE44E050E06FEE72E018
:10725000CE010F9678DE44E050E06AEE7BE0CE018E
:107260000F9671DE44E050E062EE7BE0CE010F96B7
:107270006ADE44E050E06AED7BE0CE010F9663DE0B
:1072800044E050E066E878E0CE010F965CDE44E032
:1072900050E062E878E0CE010F9655DE44E050E021
:1072A0006AE878E0CE010F964EDE10E0C12C80E84F
:1072B000D82E8BE3E82E85E4F82E812C912C90E8D3
:1072C000A92E9FE3B92E111122C044E050E06AE2DA
:1072D00072E0CE010F9637DE44E050E062E372E0E8
:1072E000CE010F9630DE44E050E06EE272E0CE0157
:1072F0000F9629DE8D829E82AF82B88644E050E0F0
:10730000BE016B5F7F4FCE010F961DDE1CC0CD828C
:10731000DE82EF82F88644E050E0BE016B5F7F4F73
:10732000CE010F9610DE1D821E821F82188604E099
:10733000015049F044E050E0BE016B5F7F4FCE0149
:107340000F9601DEF5CF1F5F143009F0BCCF84E14A
:1073500090E09E878D8742E050E0BE01635F7F4FE3
:10736000CE010F96F0DD80E090E8ABE3B5E48D83CD
:107370009E83AF83B887115049F044E050E0BE01CE
:107380006B5F7F4FCE010F96DEDDF5CF80E290E0A0
:107390009C878B8742E050E0BE01655F7F4FCE0146
:1073A0000F96D1DD41E050E06BE479E0CE010F961D
:1073B000CADD11110CC08091480290914902A09140
:1073C0004A02B0914B028D839E83AF83B88744E01D
:1073D00050E0BE016B5F7F4FCE010F96B4DD1F5FA3
:1073E000143039F780917B06811137C080917C067B
:1073F00090917D069A878987EF84F88884E690E0EB
:10740000988B8F8744E050E063E873E0CE010F96DD
:107410009ADD42E050E0BE01675F7F4FCE010F96DC
:1074200092DDE1E4F7E184918F010F5F1F4F882324
:1074300019F08ED8F801F7CFB701645671098DE9BC
:1074400098E02ADCE4E9F8E084918F010F5F1F4F98
:10745000882319F07DD8F801F7CF64960FB6F89419
:10746000DEBF0FBECDBFDF91CF911F910F91FF9077
:10747000EF90DF90CF90BF90AF909F908F90089546
:107480000E94768820919502309196024091970251
:10749000509198026091990270919A0280919B029A
:1074A00090919C020E94F55D0E94E0880E94E35446
:1074B00080E090E00E94CD9B81E090E00E94CD9B17
:1074C00082E090E00C94CD9B2F923F924F925F927E
:1074D0006F927F928F929F92AF92BF92CF92DF92E4
:1074E000EF92FF920F931F93CF93DF93CDB7DEB749
:1074F000CE54D1090FB6F894DEBF0FBECDBF8DB705
:107500009EB72D969FAF8EAF2D9784E690E025967F
:107510009FAF8EAF259710927E0644E050E0BE01EB
:10752000635C7F4FCE018D5B9F4FDADC42E050E021
:10753000BE016F5B7F4FCE018D5B9F4FD1DC43E07F
:1075400050E0BE01635C7F4F83E893E00E94A0E8B7
:10755000892B19F00E9462D407C36DB67EB619AEAE
:107560001AAE1BAE1CAE10927D0610927C0641E056
:1075700050E0BE01665B7F4FCE018D5B9F4FB0DC5C
:1075800080E1E1E5F3E0DE01919601900D928A95AC
:10759000E1F780E1E1E6F3E0DE01519601900D9222
:1075A0008A95E1F780E1E1E7F3E08E010F5F1F4F7D
:1075B000D80101900D928A95E1F72B96CFAC2B97CD
:1075C000D12C93E0C90ED11CCC0CDD1CCC0CDD1CE5
:1075D000EDB7FEB7EC19FD090FB6F894FEBF0FBE6C
:1075E000EDBF8DB79EB701964C01EC19FD090FB6A2
:1075F000F894FEBF0FBEEDBF8DB79EB701965C013C
:10760000EC19FD090FB6F894FEBF0FBEEDBF8DB7A4
:107610009EB701967C01A601B401CE018D5B9F4F00
:107620005FDCA601B501CE018D5B9F4F59DCA60141
:10763000B701CE018D5B9F4F53DC2B962FAD2B975F
:1076400030E02E5F3F4FEFE0F9E02F96FFAFEEAF57
:107650002F97A7E2B9E067EF78E080E090E040E0A4
:1076600050E02417350714F0640105C0F1E2CF2E75
:10767000D12CCC0EDD1EC80ED91EF6012080318023
:1076800042805380FB012192319241925192BF017D
:107690002417350714F0650105C0E1E1CE2ED12C89
:1076A000CC0EDD1EC80ED91EF6012080318042802E
:1076B00053802D923D924D925D922417350714F020
:1076C000670101C06801C80ED91EF6012080318013
:1076D000428053802F96EEADFFAD2F9721923192CD
:1076E000419251922F96FFAFEEAF2F974F5F5F4FB2
:1076F00004964430510509F0B4CF44E050E067E40B
:1077000079E0CE018D5B9F4FEBDB44E050E06BE016
:1077100079E0CE018D5B9F4FE3DB44E050E067E012
:1077200079E0CE018D5B9F4FDBDB44E050E063E20C
:1077300079E0CE018D5B9F4FD3DB44E050E06FE1F9
:1077400079E0CE018D5B9F4FCBDB44E050E061E5FB
:1077500075E1CE018D5B9F4FC3DB40E150E067E3F5
:1077600079E0CE018D5B9F4FBBDB4CE050E062EED9
:107770007EE0CE018D5B9F4FB3DB41E050E0BE0168
:10778000675B7F4FCE018D5B9F4FAADB44E050E0EB
:10779000BE01675C7F4FCE018D5B9F4FA1DB41E057
:1077A00050E0BE01685B7F4FCE018D5B9F4F98DB41
:1077B00041E050E0BE01695B7F4FCE018D5B9F4F82
:1077C0008FDB29968FAD299728960FAD2897809F3C
:1077D00080011124E12CF12C44E050E0E016F10688
:1077E00059F0BE01675C7F4FCE018D5B9F4F78DB08
:1077F000FFEFEF1AFF0AF0CF64E472E0CE018D5B79
:107800009F4F6EDB1AE0115051F044E050E0BE0192
:10781000675C7F4FCE018D5B9F4F62DBF4CF41E011
:1078200050E0BE016A5B7F4FCE018D5B9F4F58DBFE
:1078300041E050E0BE016B5B7F4FCE018D5B9F4FFF
:107840004FDB27968FAD2797893059F526968FAD58
:107850002697893031F580E00E94AC9744E050E0F3
:1078600067E776E0CE018D5B9F4F3ADB44E050E066
:1078700063E776E0CE018D5B9F4F32DB44E451E05D
:107880006FE275E0CE018D5B9F4F2ADB2A968FADAC
:107890002A97843019F481E080932E0510924415C4
:1078A0002DC044E050E0BE016B5C7F4FCE018D5B8C
:1078B0009F4F16DB44E050E0BE016F5C7F4FCE016E
:1078C0008D5B9F4F0DDB27968FAD279726960FADCB
:1078D0002697809F80011124E12CF12CE016F106FF
:1078E00069F044E050E0BE01675C7F4FCE018D5BE4
:1078F0009F4FF6DA8FEFE81AF80AF0CF4CE050E02D
:1079000065E475E1CE018D5B9F4FEADA44E050E01B
:1079100069E972E0CE018D5B9F4FE2DA44E050E00E
:1079200065E972E0CE018D5B9F4FDADA44E050E00A
:107930006FEE72E0CE018D5B9F4FD2DA44E050E0F3
:107940006AEE7BE0CE018D5B9F4FCADA44E050E0E7
:1079500062EE7BE0CE018D5B9F4FC2DA44E050E0E7
:107960006AED7BE0CE018D5B9F4FBADA44E050E0D8
:1079700066E878E0CE018D5B9F4FB2DA44E050E0DC
:1079800062E878E0CE018D5B9F4FAADA44E050E0D8
:107990006AE878E0CE018D5B9F4FA2DA10E044E008
:1079A00050E0BE01675C7F4FCE018D5B9F4F98DA40
:1079B000111130C0C9ACDAACEBACFCAC20E030E863
:1079C0004BE355E4C701B6010E945AED882311F13B
:1079D000C0922A02D0922B02E0922C02F0922D0249
:1079E00044E050E062E372E0CE018D5B9F4F78DAB5
:1079F00044E050E06EE272E0CE018D5B9F4F70DAA2
:107A000044E050E0BE01675C7F4FCE018D5B9F4F2D
:107A100067DA0DC004E0015051F044E050E0BE01CF
:107A2000675C7F4FCE018D5B9F4F5ADAF4CF1F5FAB
:107A3000143009F0B4CF42E050E0BE016B5C7F4FE0
:107A4000CE018D5B9F4F4CDA115031F044E050E095
:107A5000BE01675C7F4FF4CF42E050E0BE016F5C37
:107A60007F4FCE018D5B9F4F3BDA41E050E06BE4EE
:107A700079E0CE018D5B9F4F33DA44E050E0BE01E8
:107A8000675C7F4FCE018D5B9F4F2ADA11110CC0CE
:107A900089AD9AADABADBCAD8093480290934902DD
:107AA000A0934A02B0934B021F5F143031F720912C
:107AB0007C0630917D0623968EAD9FAD23972817C7
:107AC0003907A1F580917E06882319F00E9462D4BF
:107AD00046C0D6DCE1E4F7E184918F010F5F1F4FD0
:107AE000811103C003E813E004C00E94A832F8012A
:107AF000F3CFF80181918F01882319F00E94A832F9
:107B0000F8CF25966EAD7FAD25976456710982ED4D
:107B100098E0C2D8E9ECF8E084918F010F5F1F4F25
:107B20008823E9F00E94A832F801F6CFEAEFF5E1E8
:107B300084918F010F5F1F4F882321F00E94A8328C
:107B4000F801F6CFEFEAF8E084918F010F5F1F4F45
:107B5000882309F4BBCF0E94A832F801F5CF0FB6F5
:107B6000F8947EBE0FBE6DBE80E00E94F6CF2D96CB
:107B70008EAD9FAD2D970FB6F8949EBF0FBE8DBFF3
:107B8000C25BDF4F0FB6F894DEBF0FBECDBFDF91F3
:107B9000CF911F910F91FF90EF90DF90CF90BF900A
:107BA000AF909F908F907F906F905F904F903F909D
:107BB0002F900895FC0120E03EE2DB014C91403221
:107BC00041F0283011F430833196DB014C91408331
:107BD00031962F5F6F5F7F4F2B3079F710820895BA
:107BE000CF9380918F0B8823B9F14091870B5091EF
:107BF000880B6091890B70918A0B27E839E080919E
:107C0000900B9091910B0E949676C82F811102C023
:107C1000C0E023C040918B0B50918C0B60918D0B79
:107C200070918E0B411551056105710591F027E8A2
:107C300039E08091900B9091910B0E949676882369
:107C400039F310928B0B10928C0B10928D0B1092BB
:107C50008E0B10928F0B01C0C1E08C2FCF91089535
:107C6000CF92DF92EF92FF92CF936B017C01C42FF2
:107C70008091870B9091880BA091890BB0918A0B12
:107C80008C159D05AE05BF05C9F0AADF811102C0A4
:107C900080E018C027E839E0B701A6018091900B79
:107CA0009091910B0E94FA76882391F3C092870BF2
:107CB000D092880BE092890BF0928A0B81E0C1117F
:107CC00080938F0BCF91FF90EF90DF90CF9008952E
:107CD0004F925F926F927F928F929F92AF92BF92DC
:107CE000CF92DF92EF92FF920F931F93CF93DF9388
:107CF000EC016A017B01280139014230510561051F
:107D0000710510F480E064C089859A85AB85BC85D7
:107D10000196A11DB11D84179507A607B70790F31B
:107D20008F89803149F48D2C9E2CAF2CBB248B89FC
:107D30009C89AD89BE890FC0803221F78B889C88D1
:107D4000AD88BE88DB01CA0157E0B695A795979527
:107D500087955A95D1F7880E991EAA1EBB1E41E041
:107D6000C501B4017DDF882369F29F89903161F4F8
:107D7000DD24EE24FF249601220F331FF901E95779
:107D8000F64F5182408211C0E894C7F8DD24EE24FA
:107D9000FF249601220F331F220F331FF901E957E9
:107DA000F64F40825182628273829A89923080F0CB
:107DB0004D815E816F817885840E951EA61EB71E4B
:107DC00080928B0B90928C0BA0928D0BB0928E0BAD
:107DD000DF91CF911F910F91FF90EF90DF90CF90A7
:107DE000BF90AF909F908F907F906F905F904F90DB
:107DF0000895CF92DF92EF92FF920F931F93CF934C
:107E0000DF93FC0181859285A385B4850196A11D30
:107E1000B11D84179507A607B70710F480E061C06D
:107E20008789803149F4BB27A72F962F852FC388D8
:107E3000D488E588F6880FC0803281F783899489D9
:107E4000A589B6896A017B01C7E0F694E794D794C7
:107E5000C794CA95D1F78C0D9D1DAE1DBF1DE901BC
:107E60006A017B018F014091870B5091880B6091D3
:107E7000890B70918A0B84179507A607B70799F4A9
:107E8000F80187898031B1F4B701A601552766272B
:107E90007727440F551FFA01E957F64F80819181EA
:107EA000A0E0B0E019C040E0BC01CD01D9DE8111F5
:107EB000E7CFB4CFB701A6014F77552766277727BD
:107EC000440F551F440F551FFA01E957F64F8081A3
:107ED0009181A281B381BF7088839983AA83BB8378
:107EE00081E0DF91CF911F910F91FF90EF90DF9094
:107EF000CF9008954F925F926F927F92AF92BF9210
:107F0000CF92DF92EF92FF920F931F93CF93DF9365
:107F100000D01F92CDB7DEB78C0149835A836B83A3
:107F20007C835901C12CD12C7601412C82E0582E42
:107F3000612C712C49815A816B817C819E012F5F5C
:107F40003F4FC80156DF882341F1D301C201F80138
:107F5000058404C0880F991FAA1FBB1F0A94D2F77B
:107F6000C80ED91EEA1EFB1E49815A816B817C8195
:107F70008789803139F481E0483F5F4F61057105A1
:107F800038F4D8CF81E0483F5F4F6F4F7F4090F289
:107F9000F501C082D182E282F3820F900F900F90A0
:107FA0000F90DF91CF911F910F91FF90EF90DF9095
:107FB000CF90BF90AF907F906F905F904F9008955B
:107FC000DF92EF92FF920F931F93CF93DF937C0189
:107FD000EB018A018DE0D82E40E250E0BE01C701DE
:107FE0000E9476778032910539F021E0892B09F4DF
:107FF00020E0822F81953EC02881222399F1253EE1
:1080000059F32E3249F30115110541F13B853F73B8
:108010003F3021F54A8D5B8D452B01F52F713FEFE8
:10802000320F3230D8F430E021503109D29EC001F5
:10803000D39E900D1124D801A80FB91FFE0120E096
:10804000AD01253088F431813D932F5F32962D307C
:10805000C1F7288126FF02C0FA0115862B8523FD72
:10806000BBCF08C080E006C02B3010F43481ECCFC9
:108070003681EACFDF91CF911F910F91FF90EF9062
:10808000DF900895CF93DF93EC018B818823A9F1D2
:10809000898187FF2FC06C857D858E859F8541E016
:1080A000DFDD882351F1E88980E2E89FF0011124A7
:1080B000DF01A957B64F109701F18C91853EE9F089
:1080C0008B81823050F449895A896B897C895C960E
:1080D0004D935D936D937C935F978D899E89AF8956
:1080E000B88DE957F64F938F828FB58BA48B89811A
:1080F0008F778983DF91CF9173CD81E0888380E092
:10810000DF91CF9108952F923F924F925F926F929D
:108110007F928F929F92AF92BF92CF92DF92EF9217
:10812000FF920F931F93CF93DF9300D01F92CDB791
:10813000DEB78C014B011A01DC0113968C91139769
:108140008130C9F411968C9181FF15C082FF19C04E
:10815000F801418952896389748980859185A28556
:10816000B38584179507A607B70759F0C8010E9481
:10817000D673811106C081E0F80180838FEF9FEFF5
:108180002CC1610185C0D80159968D919C915A9757
:10819000FC01248121502A013B0139E07694679447
:1081A000579447943A95D1F7722E74207A01F1E0F2
:1081B000FF22772009F478C080E092E08E199F09B1
:1081C00056018C159D0508F45C01D80159962D9136
:1081D0003C915A9714968D919D910D90BC91A02D34
:1081E0000297A109B109F901058404C0880F991FFC
:1081F000AA1FBB1F0A94D2F74685578560897189EB
:10820000840F951FA61FB71F9C01AD01270D311DBF
:10821000411D511D29013A01A11432E0B30609F0B4
:1082200089C08091870B9091880BA091890BB091A8
:108230008A0B84159505A605B70569F410928F0B76
:108240008FEF9FEFDC018093870B9093880BA093B7
:10825000890BB0938A0B9401B301A2018091900B1A
:108260009091910B0E949676882309F484CFF801AF
:1082700080859185A285B3858A0D9B1DA11DB11DA9
:1082800080879187A287B3878A0C9B1CCA18DB085A
:10829000D80118964D915D916D917C911B97C114F9
:1082A000D10409F070CF7AC0E114F10409F084CF51
:1082B00014964D915D916D917C91179741155105E3
:1082C0006105710559F455968D919D910D90BC9164
:1082D000A02D0097A105B10539F520C09E012F5FA3
:1082E0003F4F87DD882309F446CF89819A81AB818E
:1082F000BC81F801218D328DF9012789203139F4B3
:10830000883FFFEF9F07A105B10540F40DC0883FEE
:108310002FEF9207A2072FE0B20730F0C8010E94AA
:108320001875811149CF27CFF80184839583A683DF
:10833000B78342CFE114F10411F5D80118964D919D
:108340005D916D917C911B9751968D919D910D90B2
:10835000BC91A02D481759076A077B0780F040DCC5
:10836000882309F408CF81E080938F0B4092870B1C
:108370005092880B6092890B70928A0B07C041E083
:10838000C301B2016DDC882309F4F5CEA501B40167
:10839000C7018957964F0E945EE869CF51968D912B
:1083A0009D910D90BC91A02D84179507A607B70746
:1083B00040F4F801418B528B638B748B8181806810
:1083C0008183D80111968C9183FD02C0C10105C043
:1083D000C80158DE8111FACFCECE0F900F900F90CA
:1083E0000F90DF91CF911F910F91FF90EF90DF9051
:1083F000CF90BF90AF909F908F907F906F905F9045
:108400004F903F902F900895CF93DF931F92CDB759
:10841000DEB7698341E050E0BE016F5F7F4F049695
:1084200072DE0F90DF91CF910895CF92DF92EF929D
:10843000FF92CF93C82F0E94847D6B017C0124EAB8
:1084400030E74DE75FE3609177087091780880919D
:10845000790890917A080E945AED87FD05C04AEF8D
:1084600050E060E070E003C040E050E0BA01C40EAC
:10847000D51EE61EF71EC0928B06D0928C06E092A7
:108480008D06F0928E06C0931D02CF91FF90EF9063
:10849000DF90CF9008958091950681110C946670BD
:1084A0006091BB0E7091BC0E8091BD0E9091BE0E7E
:1084B000611571058105910571F10E9460ED2091B2
:1084C0007708309178084091790850917A080E9495
:1084D000BFED9B01AC0160910B0F70910C0F80916F
:1084E0000D0F90910E0F0E9459E560930B0F709342
:1084F0000C0F80930D0F90930E0F1092BB0E1092E5
:10850000BC0E1092BD0E1092BE0E83E090E08DDF87
:1085100081E080939D0280919D02882349F08BE049
:108520009FE00E942A80BC018BE49AE00C94917336
:1085300008952F923F924F925F926F927F928F9207
:108540009F92AF92BF92CF92DF92EF92FF920F93E2
:108550001F93CF93DF9300D000D0CDB7DEB720912B
:1085600095062223D1F026960FB6F894DEBF0FBEF3
:10857000CDBFDF91CF911F910F91FF90EF90DF90D2
:10858000CF90BF90AF909F908F907F906F905F90B3
:108590004F903F902F900C9466707E836D831C01EA
:1085A0008091BB0E9091BC0EA091BD0EB091BE0EFD
:1085B000892B8A2B8B2B09F4B3C00E949D320D812D
:1085C0001E81000F111F000F111FC8018150914F14
:1085D0003C01DC01CD90DD90ED90FC908091BB0ED4
:1085E0009091BC0EA091BD0EB091BE0E89839A836E
:1085F000AB83BC83BC01CD010E9460ED2091770864
:10860000309178084091790850917A080E94BFED26
:108610009B01AC01C701B6010E9459E54B015C0109
:10862000D3016D937D938D939C931397ED81FE8180
:108630003297A9F420E030E04AE754E4C701B601DC
:108640000E9458E52B013C0120E030E04AE754E469
:10865000C701B6010E9459E56B017C0126C0E1E02B
:10866000F0E08D819E81E81BF90BEE0FFF1FEE0FEE
:10867000FF1FE150F14F60817181828193819B01E5
:10868000AC010E94BFED9B01AC0160E074E48CE2A0
:1086900096E40E9458E50E94EAE76B017C012B01F9
:1086A0003C0177FA709477F8709489819A81AB8154
:1086B000BC81B7FF10C0A3019201C501B4010E94A3
:1086C0005AED87FF1FC0F801E150F14F40825182FF
:1086D0006282738217C089819A81AB81BC81892BA8
:1086E0008A2B8B2B79F0A7019601C501B4010E945A
:1086F000A1E718163CF4F801E150F14FC082D18295
:10870000E282F3828D819E8190DE1092BB0E1092E8
:10871000BC0E1092BD0E1092BE0E81E080939D02A1
:1087200080919D02882331F18D819E81880F991F50
:10873000880F991F8150914F0E942A80BC01C1016E
:1087400026960FB6F894DEBF0FBECDBFDF91CF9156
:108750001F910F91FF90EF90DF90CF90BF90AF905F
:108760009F908F907F906F905F904F903F902F9051
:108770000C94917326960FB6F894DEBF0FBECDBF52
:10878000DF91CF911F910F91FF90EF90DF90CF90ED
:10879000BF90AF909F908F907F906F905F904F9021
:1087A0003F902F90089560E070E086E39AE0C1CE9C
:1087B00061E070E08DE39AE0BCCE62E070E084E4BA
:1087C0009AE0B7CE8F929F92AF92BF92CF92DF92F4
:1087D000EF92FF920F931F93CF93DF931092940623
:1087E0008091BB0E9091BC0EA091BD0EB091BE0EBB
:1087F00081309048A105B10540F01092BB0E109257
:10880000BC0E1092BD0E1092BE0E6091BB0E709108
:10881000BC0E8091BD0E9091BE0E25E030E040E090
:1088200050E00E9435F1C22F809186061816F4F4AC
:10883000022E000C330B482F082E000C550B415014
:1088400051092417350794F0CFEFC80F25E0C29FD8
:10885000C0011124092E000CAA0BBB0B8093BB0E88
:108860009093BC0EA093BD0EB093BE0E10928A06DC
:1088700080918906C81714F4C093890680918906EF
:10888000082E000C990B03962C2F0C2E000C330B8A
:108890008217930724F48DEF8C0F80938906109133
:1088A0008906D0E0111118C080919D02882351F0F3
:1088B00081E0C11180E003E023E04BED59E06D2F32
:1088C0000E946CB780919506882309F489C0C11174
:1088D00087C00E94667080C0113009F054C080913A
:1088E0009D02882359F081E0C13009F080E000E268
:1088F0002EE34FEC59E06D2F0E946CB780919506E6
:10890000882309F46DC0C13009F06AC0E0908C087A
:10891000F0908D08C0908408D090850860918808F8
:1089200070918908072E000C880B990B0E9460ED4E
:108930004B015C0120E030E0A9010E94A1E718167C
:10894000CCF420E030E849E853E4C501B4010E94CA
:10895000A1E718163CF4812C80E8982E89E8A82E0F
:1089600083E4B82EC501B4010E94B6E67093810875
:1089700060938008D0927F08C0927E08F0927D08B4
:10898000E0927C0827C0123059F580919D0288231F
:1089900059F081E0C23009F080E000E22EE34FEBB5
:1089A00059E06D2F0E946CB7809195068823C1F025
:1089B000C230B1F480918C0890918D082091840888
:1089C0003091850830937F0820937E0890937D082E
:1089D00080937C080E94607080918A06811108C093
:1089E000DF5F1F5FD43009F05DCF83E080938606A0
:1089F000DF91CF911F910F91FF90EF90DF90CF907B
:108A0000BF90AF909F908F9008958F929F92AF925A
:108A1000BF92CF92DF92EF92FF920F931F93CF936B
:108A2000DF93109294068091BB0E9091BC0EA091A2
:108A3000BD0EB091BE0E81309048A105B10540F049
:108A40001092BB0E1092BC0E1092BD0E1092BE0E74
:108A50006091BB0E7091BC0E8091BD0E9091BE0EC8
:108A600025E030E040E050E00E9435F1C22F8091D7
:108A700083061816F4F4022E000C330B482F082E30
:108A8000000C550B415051092417350794F0CFEFD6
:108A9000C80F25E0C29FC0011124092E000CAA0BAB
:108AA000BB0B8093BB0E9093BC0EA093BD0EB093F6
:108AB000BE0E10928A0680918906C81714F4C093DE
:108AC000890680918906082E000C990B03962C2F9D
:108AD0000C2E000C330B8217930724F48DEF8C0FB0
:108AE0008093890610918906D0E0111118C08091F9
:108AF0009D02882351F081E0C11180E003E023E072
:108B00004BE059E06D2F0E946CB780919506882349
:108B100009F489C0C11187C00E94667080C01130FD
:108B200009F054C080919D02882359F081E0C13042
:108B300009F080E000E22EE34FEF58E06D2F0E9435
:108B40006CB780919506882309F46DC0C13009F097
:108B50006AC0E0908A08F0908B08C0908208D0909C
:108B600083086091860870918708072E000C880B97
:108B7000990B0E9460ED4B015C0120E030E0A901FF
:108B80000E94A1E71816CCF420E030E849E853E44D
:108B9000C501B4010E94A1E718163CF4812C80E8BD
:108BA000982E89E8A82E83E4B82EC501B4010E944E
:108BB000B6E67093810860938008D0927F08C092D7
:108BC0007E08F0927D08E0927C0827C0123059F5AB
:108BD00080919D02882359F081E0C23009F080E045
:108BE00000E22EE34FEE58E06D2F0E946CB78091AB
:108BF00095068823C1F0C230B1F480918A08909123
:108C00008B08209182083091830830937F0820934D
:108C10007E0890937D0880937C080E94607080910C
:108C20008A06811108C0DF5F1F5FD43009F05DCF75
:108C300083E080938306DF91CF911F910F91FF9086
:108C4000EF90DF90CF90BF90AF909F908F9008955E
:108C5000CF92DF92EF92FF920F931F93CF93DF9308
:108C6000109294068091BB0E9091BC0EA091BD0E07
:108C7000B091BE0E81309048A105B10540F0109230
:108C8000BB0E1092BC0E1092BD0E1092BE0E6091E3
:108C9000BB0E7091BC0E8091BD0E9091BE0E25E072
:108CA00030E040E050E00E9435F1C22F809187060D
:108CB0001816F4F4022E000C330B482F082E000C6B
:108CC000550B415051092417350794F0CFEFC80FC9
:108CD00025E0C29FC0011124092E000CAA0BBB0B7A
:108CE0008093BB0E9093BC0EA093BD0EB093BE0EAE
:108CF00010928A0680918906C81714F4C0938906D9
:108D000080918906082E000C990B03962C2F0C2EAF
:108D1000000C330B8217930724F48DEF8C0F809394
:108D2000890610918906D0E084E0E82E8AE0F82ECA
:108D300093E2C92E9AE0D92E111118C080919D029C
:108D4000882351F081E0C11180E003E023E041E39A
:108D50005AE06D2F0E946CB780919506882309F424
:108D6000BAC0C111B8C00E946670B1C01130E1F440
:108D700080919D02882359F081E0C13009F080E0A4
:108D800000E22EE347E25AE06D2F0E946CB780911B
:108D90009506882309F49FC0C13009F09CC0D09289
:108DA000930BC092920B39C01230D1F480919D0286
:108DB000882359F081E0C23009F080E00EE32EE311
:108DC00049E15AE06D2F0E946CB780919506882387
:108DD00009F481C0C23009F07EC082E995E655C031
:108DE0001330F1F480919D02882359F081E0C33063
:108DF00009F080E000E22EE348E05AE06D2F0E9487
:108E00006CB780919506882309F465C0C33009F0DA
:108E100062C0F092930BE092920B0E94AB3157C06C
:108E20001430D1F480919D02882359F081E0C43040
:108E300009F080E00EE32EE348EF59E06D2F0E9429
:108E40006CB780919506882309F445C0C43009F0B9
:108E500042C085E095E419C01530D1F480919D029F
:108E6000882359F081E0C53009F080E00EE32EE35D
:108E70004CEE59E06D2F0E946CB7809195068823C7
:108E800051F1C53041F582EE93E40E94CE541FC0EB
:108E9000163009F580919D02882359F081E0C63093
:108EA00009F080E000E22EE343EE59E06D2F0E94CE
:108EB0006CB780919506882371F0C63061F41092EA
:108EC0007D0810927C080E94F9B70E946070809122
:108ED0008A06811108C0DF5F1F5FD43009F02CCFF4
:108EE00087E080938706DF91CF911F910F91FF90CC
:108EF000EF90DF90CF9008958F929F92AF92BF92A4
:108F0000CF92DF92EF92FF920F931F93CF93DF9355
:108F1000109294068091BB0E9091BC0EA091BD0E54
:108F2000B091BE0E81309048A105B10540F010927D
:108F3000BB0E1092BC0E1092BD0E1092BE0E609130
:108F4000BB0E7091BC0E8091BD0E9091BE0E25E0BF
:108F500030E040E050E00E9435F1C22F809184065D
:108F60001816F4F4022E000C330B482F082E000CB8
:108F7000550B415051092417350794F0CFEFC80F16
:108F800025E0C29FC0011124092E000CAA0BBB0BC7
:108F90008093BB0E9093BC0EA093BD0EB093BE0EFB
:108FA00010928A0680918906C81714F4C093890626
:108FB00080918906082E000C990B03962C2F0C2EFD
:108FC000000C330B8217930724F48DEF8C0F8093E2
:108FD000890610918906D0E083E1E82E89E0F82E19
:108FE0009EE1C92E99E0D92E2DE2A22E29E0B22EC3
:108FF0003DE4832E39E0932E111118C080919D021B
:10900000882351F081E0C11180E003E023E04FE5C7
:1090100059E06D2F0E946CB780919506882309F462
:109020009CC0C1119AC00E94667093C01130E1F4D7
:1090300080919D02882359F081E0C13009F080E0E1
:1090400000E22EE341E559E06D2F0E946CB780915C
:109050009506882309F481C0C13009F07EC0909242
:10906000930B8092920B73C01230E1F480919D02B9
:10907000882359F081E0C23009F080E00EE32EE34E
:109080004CE359E06D2F0E946CB7809195068823C0
:1090900009F463C0C23009F060C082EC98E40E9419
:1090A000CE5457C01330E1F480919D02882359F0CB
:1090B00081E0C33009F080E000E22EE344E359E0B0
:1090C0006D2F0E946CB780919506882309F445C0E6
:1090D000C33009F042C0B092930BA092920B37C0FC
:1090E0001430D1F480919D02882359F081E0C4307E
:1090F00009F080E000E22EE345E259E06D2F0E9486
:109100006CB780919506882341F1C43031F5D09237
:10911000930BC092920B1BC01530F9F480919D0205
:10912000882359F081E0C53009F080E000E22EE3A9
:1091300048E159E06D2F0E946CB780919506882315
:1091400061F0C53051F4F092930BE092920B0E94C3
:10915000AB3180918A06811108C0DF5F1F5FD43078
:1091600009F04ACF86E080938406DF91CF911F916A
:109170000F91FF90EF90DF90CF90BF90AF909F90B6
:109180008F9008958F929F92AF92BF92DF92EF924D
:10919000FF920F931F93CF93DF93109294068091C9
:1091A000BB0E9091BC0EA091BD0EB091BE0E813051
:1091B0009048A105B10540F01092BB0E1092BC0E74
:1091C0001092BD0E1092BE0E6091BB0E7091BC0E3F
:1091D0008091BD0E9091BE0E25E030E040E050E061
:1091E0000E9435F1C22F809185061816F4F4022EE4
:1091F000000C330B482F082E000C550B4150510921
:109200002417350794F0CFEFC80F25E0C29FC001A7
:109210001124092E000CAA0BBB0B8093BB0E90935C
:10922000BC0EA093BD0EB093BE0E10928A06809124
:109230008906C81714F4C093890680918906082E00
:10924000000C990B03962C2F0C2E000C330B82175D
:10925000930724F48DEF8C0F80938906D0908906B4
:10926000D0E024E6A22E29E0B22E3AE9832E39E09E
:10927000932ED11018C080919D02882351F081E077
:10928000C11180E003E023E04DEA59E06D2F0E9418
:109290006CB780919506882309F49AC0C11198C0D3
:1092A0000E94667091C081E0D8121CC080919D021E
:1092B000882359F081E0C13009F080E000E22EE31C
:1092C0004EE959E06D2F0E946CB780919506882376
:1092D00009F47EC0C13009F07BC09092930B80925C
:1092E000920B70C022E0D21227C080919D02882389
:1092F00071F08FE796E00E9474809C0181E0C2309B
:1093000009F080E04DE859E06D2F0E94B3E48091B0
:109310009506882309F45CC0C23009F059C0E12CDD
:10932000F12C00EA11E420E030E040E252EC6FE77B
:1093300076E080E899E027C083E0D81227C08091CA
:109340009D02882371F084E492E00E9474809C0165
:1093500081E0C33009F080E047E759E06D2F0E94BB
:10936000B3E480919506882399F1C33089F5E12C07
:10937000F12C00EA11E420E030E040E252EC64E439
:1093800072E08EE699E00E94C3D81EC024E0D2129B
:109390001FC080919D02882359F081E0C43009F0FC
:1093A00080E000E22EE348E659E06D2F0E946CB7A2
:1093B00080919506882361F0C43051F4B092930BEC
:1093C000A092920B0E94AB3180918A06811108C055
:1093D000DF5FD394D43009F04CCF85E080938506CD
:1093E000DF91CF911F910F91FF90EF90DF90BF9091
:1093F000AF909F908F900895FF920F931F93CF93FC
:10940000DF93109294068091BB0E9091BC0EA091B8
:10941000BD0EB091BE0E81309048A105B10540F05F
:109420001092BB0E1092BC0E1092BD0E1092BE0E8A
:109430006091BB0E7091BC0E8091BD0E9091BE0EDE
:1094400025E030E040E050E00E9435F1C22F8091ED
:1094500088061816F4F4022E000C330B482F082E41
:10946000000C550B415051092417350794F0CFEFEC
:10947000C80F25E0C29FC0011124092E000CAA0BC1
:10948000BB0B8093BB0E9093BC0EA093BD0EB0930C
:10949000BE0E10928A0680918906C81714F4C093F4
:1094A000890680918906082E000C990B03962C2FB3
:1094B0000C2E000C330B8217930724F48DEF8C0FC6
:1094C0008093890610918906F12C112329F080914F
:1094D000950B81111CC065C080919D02882351F0BD
:1094E00081E0C11180E003E023E042E75AE06F2D04
:1094F0000E946CB780919506882349F3C111E7CF8C
:109500000E94667080918A06882309F3B3C0809117
:10951000960B882309F445C08091970B882309F4A2
:1095200040C01130D1F480919D02882359F081E030
:10953000C13009F080E00EE32EE34BE65AE06F2DD8
:109540000E946CB780919506882309F491C0C130C0
:1095500009F08EC083ED93E41CC0123009F088C07E
:1095600080919D02882359F081E0C23009F080E0AB
:109570000EE32EE344E65AE06F2D0E946CB7809113
:109580009506882309F474C0C23009F071C088EDD3
:1095900093E40E94CE5480918A06882309F468C01F
:1095A00069C0D1E020E030E040E251E4609177080A
:1095B000709178088091790890917A080E945AED0C
:1095C00087FF4EC08091950B882349F18091960BBF
:1095D000882329F18091970B882309F11D1711F039
:1095E000DF5F1DC080919D02882351F081E0C1138F
:1095F00080E00EE32EE34DE55AE06F2D0E946CB73C
:1096000080919506882361F3C113EACF8DED93E431
:109610000E94CE5480918A06882311F32BC01D1717
:1096200011F0DF5F1DC080919D02882351F081E021
:10963000C11380E00EE32EE344E55AE06F2D0E9453
:109640006CB780919506882361F3C113EACF8BE450
:1096500092E40E94CE5480918A06882311F30AC0B6
:10966000F3941F5F84E0F81230CFD093880602C0D5
:10967000D3E098CFDF91CF911F910F91FF90089584
:10968000CF92DF92EF92FF920F931F93CF93DF93CE
:1096900000D01F92CDB7DEB78091BB0E9091BC0E6B
:1096A000A091BD0EB091BE0EB7FF08C01092BB0EC8
:1096B0001092BC0E1092BD0E1092BE0E8091BF0E85
:1096C0009091C00EA091C10EB091C20E4091BB0E00
:1096D0005091BC0E6091BD0E7091BE0E841795071F
:1096E000A607B70744F48093BB0E9093BC0EA093DB
:1096F000BD0EB093BE0E80919D02882379F14091FA
:10970000BB0E5091BC0E6091BD0E7091BE0E80914B
:10971000C30E9091C40EA091C50EB091C60E6A0101
:109720007B01C80ED91EEA1EFB1EC701B6010E94AE
:109730005EED20E030E048EC52E40E94BFED69832A
:109740007A838B839C83CE0101960E94867FBC0125
:109750008091C90E9091CA0E0E94917380919506D6
:10976000882391F10091C70E1091C80E4091BB0E55
:109770005091BC0E6091BD0E7091BE0E8091C30ED3
:109780009091C40EA091C50EB091C60E6A017B01E6
:10979000C80ED91EEA1EFB1EC701B6010E945EED6F
:1097A00020E030E048EC52E40E94BFED0E94BCE6AD
:1097B000F80160837183828393830E946670E091D5
:1097C000CB0EF091CC0E19950F900F900F900F903B
:1097D000DF91CF911F910F91FF90EF90DF90CF908D
:1097E0000895CF92DF92EF92FF920F931F93CF9342
:1097F000DF9300D01F92CDB7DEB78091BB0E909162
:10980000BC0EA091BD0EB091BE0EB7FF08C0109265
:10981000BB0E1092BC0E1092BD0E1092BE0E809127
:10982000BF0E9091C00EA091C10EB091C20E40919A
:10983000BB0E5091BC0E6091BD0E7091BE0E841790
:109840009507A607B70744F48093BB0E9093BC0E10
:10985000A093BD0EB093BE0E80919D02882379F136
:109860004091BB0E5091BC0E6091BD0E7091BE0E2A
:109870008091C30E9091C40EA091C50EB091C60EFA
:109880006A017B01C80ED91EEA1EFB1EC701B60184
:109890000E9460ED20E030E048EC52E40E94BFED11
:1098A00069837A838B839C83CE0101960E94867F95
:1098B000BC018091C90E9091CA0E0E949173809153
:1098C0009506882359F10091C70E1091C80E40915A
:1098D000BB0E5091BC0E6091BD0E7091BE0E80917A
:1098E000C30E9091C40EA091C50EB091C60E6A0130
:1098F0007B01C80ED91EEA1EFB1EC701B6010E94DD
:1099000060ED20E030E048EC52E40E94BFEDF80149
:1099100060837183828393830E9466700F900F909F
:109920000F900F90DF91CF911F910F91FF90EF90CB
:10993000DF90CF900895CF92DF92EF92FF920F9336
:109940001F93CF93DF9300D01F92CDB7DEB78091E6
:10995000BB0E9091BC0EA091BD0EB091BE0EB7FF94
:1099600008C01092BB0E1092BC0E1092BD0E109249
:10997000BE0E8091BF0E9091C00EA091C10EB0910D
:10998000C20E4091BB0E5091BC0E6091BD0E709105
:10999000BE0E84179507A607B70744F48093BB0E45
:1099A0009093BC0EA093BD0EB093BE0E80919D020D
:1099B000882379F14091BB0E5091BC0E6091BD0E91
:1099C0007091BE0E8091C30E9091C40EA091C50EF1
:1099D000B091C60E6A017B01C80ED91EEA1EFB1E9D
:1099E000C701B6010E9460ED2AE037ED43E25CE377
:1099F0000E94BFED69837A838B839C83CE0101969D
:109A00000E94607EBC018091C90E9091CA0E0E9496
:109A1000917380919506882381F10091C70E109172
:109A2000C80E4091BB0E5091BC0E6091BD0E70915E
:109A3000BE0E8091C30E9091C40EA091C50EB09140
:109A4000C60E6A017B01C80ED91EEA1EFB1EC701A5
:109A5000B6010E9460ED2AE037ED43E25CE30E942C
:109A6000BFEDF80160837183828393830E946670E7
:109A7000E091CB0EF091CC0E19950F900F900F90B6
:109A80000F90DF91CF911F910F91FF90EF90DF909A
:109A9000CF900895AF92BF92CF92DF92FF920F9333
:109AA0001F93CF93DF9300D01F92CDB7DEB7809185
:109AB000BB0E9091BC0EA091BD0EB091BE0EB7FF33
:109AC00008C01092BB0E1092BC0E1092BD0E1092E8
:109AD000BE0E8091BF0E9091C00EA091C10EB091AC
:109AE000C20E4091BB0E5091BC0E6091BD0E7091A4
:109AF000BE0E84179507A607B70744F48093BB0EE4
:109B00009093BC0EA093BD0EB093BE0E80919D02AB
:109B1000882379F14091BB0E5091BC0E6091BD0E2F
:109B20007091BE0E8091C30E9091C40EA091C50E8F
:109B3000B091C60E5A016B01A80EB91ECA1EDB1EDB
:109B4000C601B5010E9460ED2AE037ED43E25CE317
:109B50000E94BFED69837A838B839C83CE0101963B
:109B60000E94037FBC018091C90E9091CA0E0E9491
:109B70009173F0909506FF2059F10091C70E109156
:109B8000C80E8091BB0E9091BC0EA091BD0EB091FD
:109B9000BE0E4091C30E5091C40E6091C50E7091DF
:109BA000C60E5C016D01A40EB51EC61ED71EC601F1
:109BB000B5010E9460ED2AE037ED43E25CE30E94CC
:109BC000BFEDF80160837183828393830E94667086
:109BD0008F2D0F900F900F900F90DF91CF911F91CD
:109BE0000F91FF90DF90CF90BF90AF90089552DF1C
:109BF000882329F0E091CB0EF091CC0E19940895B2
:109C000049CFCF92DF92EF92FF920F931F93CF93A2
:109C1000DF9300D01F92CDB7DEB78091BB0E90913D
:109C2000BC0EA091BD0EB091BE0EB7FF08C0109241
:109C3000BB0E1092BC0E1092BD0E1092BE0E809103
:109C4000BF0E9091C00EA091C10EB091C20E409176
:109C5000BB0E5091BC0E6091BD0E7091BE0E84176C
:109C60009507A607B70744F48093BB0E9093BC0EEC
:109C7000A093BD0EB093BE0E80919D02882379F112
:109C80004091BB0E5091BC0E6091BD0E7091BE0E06
:109C90008091C30E9091C40EA091C50EB091C60ED6
:109CA0006A017B01C80ED91EEA1EFB1EC701B60160
:109CB0000E9460ED2FE632E143E85AE30E94BFEDD7
:109CC00069837A838B839C83CE0101960E94F0AFD7
:109CD000BC018091C90E9091CA0E0E94917380912F
:109CE0009506882381F10091C70E1091C80E40910E
:109CF000BB0E5091BC0E6091BD0E7091BE0E809156
:109D0000C30E9091C40EA091C50EB091C60E6A010B
:109D10007B01C80ED91EEA1EFB1EC701B6010E94B8
:109D200060ED2FE632E143E85AE30E94BFEDF8010F
:109D300060837183828393830E946670E091CB0E6F
:109D4000F091CC0E19950F900F900F900F90DF911E
:109D5000CF911F910F91FF90EF90DF90CF900895DA
:109D6000CF92DF92EF92FF920F931F93CF93DF93E7
:109D700000D01F92CDB7DEB78091BB0E9091BC0E84
:109D8000A091BD0EB091BE0EB7FF08C01092BB0EE1
:109D90001092BC0E1092BD0E1092BE0E8091BF0E9E
:109DA0009091C00EA091C10EB091C20E4091BB0E19
:109DB0005091BC0E6091BD0E7091BE0E8417950738
:109DC000A607B70744F48093BB0E9093BC0EA093F4
:109DD000BD0EB093BE0E80919D02882379F1409113
:109DE000BB0E5091BC0E6091BD0E7091BE0E809165
:109DF000C30E9091C40EA091C50EB091C60E6A011B
:109E00007B01C80ED91EEA1EFB1EC701B6010E94C7
:109E100060ED2AE037ED43E25CE30E94BFED698329
:109E20007A838B839C83CE0101960E947480BC014F
:109E30008091C90E9091CA0E0E94917380919506EF
:109E4000882359F10091C70E1091C80E4091BB0EA6
:109E50005091BC0E6091BD0E7091BE0E8091C30EEC
:109E60009091C40EA091C50EB091C60E6A017B01FF
:109E7000C80ED91EEA1EFB1EC701B6010E9460ED86
:109E80002AE037ED43E25CE30E94BFEDF801608316
:109E90007183828393830E9466700F900F900F905E
:109EA0000F90DF91CF911F910F91FF90EF90DF9076
:109EB000CF900895CF92DF92EF92FF920F931F936E
:109EC000CF93DF931F921F92CDB7DEB78091BB0E69
:109ED0009091BC0EA091BD0EB091BE0EB7FF08C010
:109EE0001092BB0E1092BC0E1092BD0E1092BE0EC0
:109EF0008091BF0E9091C00EA091C10EB091C20E84
:109F00004091BB0E5091BC0E6091BD0E7091BE0E83
:109F100084179507A607B70744F48093BB0E909368
:109F2000BC0EA093BD0EB093BE0E80919D028823FF
:109F300049F14091BB0E5091BC0E6091BD0E7091E5
:109F4000BE0E8091C30E9091C40EA091C50EB0912B
:109F5000C60E6A017B01C80ED91EEA1EFB1EC70190
:109F6000B6010E9460ED0E94B6E67A836983CE0155
:109F700001960E949881BC018091C90E9091CA0EF1
:109F80000E94917380919506882329F10091C70E54
:109F90001091C80E4091BB0E5091BC0E6091BD0E49
:109FA0007091BE0E8091C30E9091C40EA091C50E0B
:109FB000B091C60E6A017B01C80ED91EEA1EFB1EB7
:109FC000C701B6010E9460EDF8016083718382834E
:109FD00093830E9466700F900F90DF91CF911F9135
:109FE0000F91FF90EF90DF90CF900895CF93DF9384
:109FF00000D0CDB7DEB78091BB0E9091BC0EA09182
:10A00000BD0EB091BE0EB7FF08C01092BB0E1092ED
:10A01000BC0E1092BD0E1092BE0E8091BF0E90919C
:10A02000C00EA091C10EB091C20E4091BB0E5091D6
:10A03000BC0E6091BD0E7091BE0E84179507A607E9
:10A04000B70744F48093BB0E9093BC0EA093BD0E53
:10A05000B093BE0E80919D028823B9F02091C30E6B
:10A060003091C40E8091BB0E9091BC0E820F931F55
:10A070009A838983CE0101960E949881BC018091C8
:10A08000C90E9091CA0E0E94917380919506882303
:10A09000A1F0E091C70EF091C80E4091C30E50910F
:10A0A000C40E2091BB0E3091BC0E240F351F31839E
:10A0B00020838B830E9466708B810F900F900F908E
:10A0C000DF91CF91089592CF91DF882329F0E0911D
:10A0D000CB0EF091CC0E19940895AF92BF92CF920F
:10A0E000DF92EF92FF920F931F93CF93DF93CDB741
:10A0F000DEB76F970FB6F894DEBF0FBECDBF80916D
:10A100009D02811105C080919506882309F4E0C164
:10A110008EE79CE090937D0C80937C0C81E090E036
:10A120009093B60E8093B50E1092B80E1092B70EA3
:10A1300040E050E0BA0182E89CE00E94D673809132
:10A140007C0C90917D0C2BE1FC013496DE01159680
:10A1500001900D922A95E1F7FC01828193819C8305
:10A160008B838FED93E09A83898340E050E0BE01BA
:10A170006F5F7F4F83EB94E00E94E99ECE010196D2
:10A180007FD5C090B70ED090B80E109294068091F3
:10A19000BB0E9091BC0EA091BD0EB091BE0E813051
:10A1A0009048A105B10540F01092BB0E1092BC0E74
:10A1B0001092BD0E1092BE0E6091BB0E7091BC0E3F
:10A1C0008091BD0E9091BE0E25E030E040E050E061
:10A1D0000E9435F1122F809197061816F4F4022E82
:10A1E000000C330B482F082E000C550B4150510921
:10A1F0002417350794F01FEF180F25E0129FC001B8
:10A200001124092E000CAA0BBB0B8093BB0E90935C
:10A21000BC0EA093BD0EB093BE0E10928A06809124
:10A220008906181714F41093890680918906082E60
:10A23000000C990B0396212F012E000C330B821773
:10A24000930724F48DEF810F80938906F09089069F
:10A25000E12C560181E0A81AB108FF2059F063E310
:10A260007CE082E89CE00E94BF748091330C8F32C6
:10A27000E1F420C080919D02882351F081E011110A
:10A2800080E003E023E046E95AE06E2D0E946CB7BF
:10A2900080919506882319F31111E1CF0E94667011
:10A2A00080918A068823D9F213C191E0F91639F01A
:10A2B00092E001C091E0650101E00F0D63C0809163
:10A2C0009D02882359F081E0113009F080E000E21E
:10A2D0002EE342E95AE06E2D0E946CB780919506FC
:10A2E000882331F3113021F78091D30D8823D1F0E9
:10A2F00081508093D30DEFE18E9FC0011124FC01AA
:10A30000EF55F34F2BE1A2E8BCE001900D922A95A6
:10A31000E1F7FC01E356F34F828193819093810C26
:10A320008093800C109289060EC08AE00E94A832A9
:10A33000CE010196A5D41092BB0E1092BC0E1092C5
:10A34000BD0E1092BE0E81E080938A0683E080935A
:10A350009D02BEC0F912B3C060E070E0C6010E9469
:10A36000CAA09091320C80919D02992309F48BC070
:10A3700081110DC080919506811111C0902FF1E0DF
:10A38000CF1AD1082FEFC216D20621F79AC081E06A
:10A390001F1180E045E06E2D0E942D65EBCF1F114F
:10A3A000EDCF1D8218861C821B828FED93E09A836D
:10A3B00089838091850C882319F00EE71CE002C088
:10A3C0000DE51CE07801F4E0EF0EF11C21E043E321
:10A3D0005CE0B701CE0105960E949B7A811126C0F0
:10A3E000E1E4F7E184917F012FEFE21AF20A88237A
:10A3F00021F00E94A832F701F5CFECE7FAE0849152
:10A400007F019FEFE91AF90A811103C003E31CE001
:10A4100004C00E94A832F701F2CFF80181918F01A8
:10A42000882309F482CF0E94A832F7CF8091D30D00
:10A430008A30C8F491E0980F9093D30DFFE18F9F7D
:10A44000C0011124DC01AF55B34F2BE1F70101909E
:10A450000D922A95E1F7F80122813381FC01E35640
:10A46000F34F338322838BE1FE013596A2E8BCE0F3
:10A4700001900D928A95E1F78B819C819093810CDC
:10A480008093800C55CF882339F081E01F1180E044
:10A4900040E26E2D0E942D6580919506882309F477
:10A4A0006DCF1F116BCF83E39CE00E9444A30E94F9
:10A4B000607080918A06882309F460CF09C09F5F8D
:10A4C0005ECFE394F39484E0E812C7CE90939706AE
:10A4D0006F960FB6F894DEBF0FBECDBFDF91CF9160
:10A4E0001F910F91FF90EF90DF90CF90BF90AF90B2
:10A4F00008954F925F926F927F928F929F92AF9248
:10A50000BF92CF92DF92EF92FF920F931F93CF9360
:10A51000DF93CDB7DEB72E970FB6F894DEBF0FBE30
:10A52000CDBF10911D021F3FF9F00E94847DC090A5
:10A530008B06D0908C06E0908D06F0908E06DC01A4
:10A54000CB018C199D09AE09BF09B7FD0DC0209143
:10A55000D50B8091D40B30E090E001968F70992755
:10A560002817390709F085C10E94D3818091E80836
:10A5700082FF40C08091A10681113EC081E080939E
:10A58000A1069091960689278093950610929606CB
:10A5900083E080939D021092E8080E94847DDC0194
:10A5A000CB018C509E4FAF4FBF4F8093E9089093E3
:10A5B000EA08A093EB08B093EC0888E893E19E8743
:10A5C0008D8782E090E09A838983BE01635F7F4F2D
:10A5D000CE0101960E9417AA16E0115069F082E0A0
:10A5E0009CE00E94733062E070E080E090E00E94A6
:10A5F0004C7DF3CF1092A1061091090110951170B6
:10A600008091A0061817A9F0112309F481C10E94B6
:10A61000D0A88091A006823029F060E088EA9AE014
:10A620000E9426821093A00683E080939D020E94E0
:10A63000EEB70E94847D6B017C0180919C06909115
:10A640009D06A0919E06B0919F06A7019601281B2A
:10A65000390B4A0B5B0B57FD6DC1D701C6018C59F5
:10A660009F4FAF4FBF4F80939C0690939D06A09342
:10A670009E06B0939F061091E708612F012E000CF3
:10A68000770B77FF03C071956195710961157105AD
:10A6900029F48091950681117BC08BC0809194062E
:10A6A000882309F454C08090900690909106A09061
:10A6B0009206B090930681149104A104B104D1F1E3
:10A6C000072E000C880B990B0E9460ED2B013C01BA
:10A6D000C701B601681979098A099B090E945EEDD4
:10A6E0009B01AC01C301B2010E9445E620E030E0CD
:10A6F0004AE754E40E94BFED4B015C0120E030E0EA
:10A7000040E253E40E94A1E787FF0FC020E030E061
:10A7100046E952E4C501B4010E94A1E787FD0AC0E1
:10A720002AE030E040E050E009C024E630E040E0BC
:10A7300050E004C021E030E040E050E0C0929006DC
:10A74000D0929106E0929206F092930604C021E026
:10A7500030E040E050E0A12F110FBB0B0E947DF1D3
:10A760008090BB0E9090BC0EA090BD0EB090BE0E1F
:10A77000DC01CB01880D991DAA1DBB1D8093BB0E6A
:10A780009093BC0EA093BD0EB093BE0E1092E7083E
:10A79000D701C6018856954CAF4FBF4F809398069E
:10A7A00090939906A0939A06B0939B0681E08093BC
:10A7B0009D02E0919E02F0919F023DE6E535F30790
:10A7C00041F480911E02882309F4ADC0815080932A
:10A7D0001E0280919D02882379F0823050F08430EF
:10A7E00028F0843031F410929D0203C081E0809300
:10A7F0009D0219951092950680919E0290919F025C
:10A8000085559D4621F080918F06882379F058E97F
:10A81000C50E5AE3D51EE11CF11CC0929806D092D9
:10A820009906E0929A06F0929B060FC080919806D6
:10A8300090919906A0919A06B0919B06C81AD90AE0
:10A84000EA0AFB0AF7FE0E94607080919D02823046
:10A8500061F0833031F0813009F06CC010929D02BC
:10A8600069C088E99BE00E94597E81E080939D0247
:10A8700061C084E01802F0011124E957FC4F20E088
:10A8800030E040E752E460817181828193810E94CF
:10A8900045E64B015C018091FF0E9091000FA09165
:10A8A000010FB091020F89839A83AB83BC8380919F
:10A8B000030F9091040FA091050FB091060F8D83A7
:10A8C0009E83AF83B8878091070F9091080FA09166
:10A8D000090FB0910A0F89879A87AB87BC87CE0191
:10A8E00001960E945932CE0101960E948B5CC12CC8
:10A8F000850174012BE03FE047E15FE063E17FE029
:10A900008FE09FE00E94C6898FEF80931D022CCEBE
:10A910001092300C1092310C823009F483CE60E03A
:10A920008BE99AE07DCE89E080931E0281E08093DE
:10A930009D024FCF2E960FB6F894DEBF0FBECDBF4F
:10A94000DF91CF911F910F91FF90EF90DF90CF900B
:10A95000BF90AF909F908F907F906F905F904F903F
:10A9600008950E94EEB73E98469A3C98449A3A98C9
:10A97000429AEAE0F1E080818E7F80839FB7F8946D
:10A98000EBE0F1E08081816080839FBF82E0809373
:10A99000A0060E94D3811092E7080895CF93DF9319
:10A9A0001F921F92CDB7DEB789839A830E94106DE4
:10A9B00040E050E0BA0189819A810F900F90DF91B9
:10A9C000CF910C94306DCF92DF92EF92FF92C090B6
:10A9D0004802D0904902E0904A02F0904B028091E8
:10A9E0004B09882351F120E030E0A901C701B601ED
:10A9F0000E945AED882309F12BED3FE049E450E431
:10AA0000C701B6010E94BFED20E030E040E05FE307
:10AA10000E94BFEDA70196010E94BFED20E030E04B
:10AA200040E05FE30E94BFED9B01AC0160E070E09D
:10AA300080E89FE30E9445E604C060E070E080E8A3
:10AA40009FE360935002709351028093520290935F
:10AA50005302FF90EF90DF90CF9008958FEF8EBD5F
:10AA60000DB407FEFDCF8EB508958CE0EAEAF6E05E
:10AA7000AFEFBEE001900D928A95E1F708954F92F5
:10AA80005F926F927F928F929F92AF92BF92CF927E
:10AA9000DF92EF92FF920F931F93CF93DF9300D03B
:10AAA00000D0CDB7DEB77C01FC01E857F44F14911C
:10AAB0006C01CC0CDD1CCC0CDD1CC6018458944F01
:10AAC0000E944D324B015C01612F110F770B880BF7
:10AAD000990B0E9460ED2B013C0120E030E040EC3E
:10AAE0005FE3C501B4010E94BFEDA30192010E9482
:10AAF000BFEDAB01BC0100E010E09801C7010E946E
:10AB00006C96C6018059944F0E944D329B01AC0156
:10AB1000C301B2010E94BFED4B015C0120E030E0B7
:10AB2000A9010E945AED882309F45AC000E010E000
:10AB30009801B501A4017058C7010E946C9686E087
:10AB4000E7E9F3E0DE01119601900D928A95E1F7B5
:10AB5000F701EE0FFF1F81E090E08C0F9D1FE80FC3
:10AB6000F91F8081918118161906D4F0E1E4F7E10C
:10AB700084918F010F5F1F4F882321F00E94A8321C
:10AB8000F801F6CFEEE4FBE084918F010F5F1F4FD9
:10AB9000882321F00E94A832F801F6CF8AE090E0E5
:10ABA000BC01990F880B990B0E9460ED9B01AC01D1
:10ABB000F601E356FC4F60817181828193810E948E
:10ABC00045E62B013C01A5019401C501B4010E9499
:10ABD00059E5AB01BC0193018201C7010E946C964B
:10ABE000F601EB5BFA4E80809180A280B38020E07A
:10ABF00030E0A901C501B4010E945AED87FF08C0E9
:10AC000000E010E09801B501A401C7010E946C9614
:10AC100026960FB6F894DEBF0FBECDBFDF91CF9161
:10AC20001F910F91FF90EF90DF90CF90BF90AF906A
:10AC30009F908F907F906F905F904F9008950F93AB
:10AC40001F93CF93DF938C01E1E4F7E18491EF014F
:10AC50002196882321F00E94A832FE01F7CFB80187
:10AC600081E49BE00E94AF3282E20E94A8328AE037
:10AC70000E94A83281E0DF91CF911F910F9108953A
:10AC80002FED33E0FC013183208304960C94533282
:10AC90005F9AEEECF6E010828A9A11829FB7F894E0
:10ACA000A8E0B1E08C9181608C939FBF1282129AD0
:10ACB00008958C01EAEFF5E18491EF012196882354
:10ACC00021F00E94A832FE01F7CFE1E2FBE084917F
:10ACD000EF012196882321F00E94A832FE01F7CFD0
:10ACE00040DE61E0C8010E9426820E94607060E040
:10ACF00080E00E94EEA788E592E00E94A1B762E0A2
:10AD000080E00E94EEA782E19BE00E94B6B763E07C
:10AD100080E00E94EEA785E09BE00E94B6B764EF5A
:10AD200071E080E090E00E944C7DF8940E94F9B7B9
:10AD3000AFDFA895FECF4F925F926F927F928F9276
:10AD40009F92AF92BF92CF92DF92EF92FF920F93BA
:10AD50001F93CF93DF93CDDB20E030E040E752E458
:10AD600060919E0870919F088091A0089091A10821
:10AD70000E94A1E79FB718162CF4F89480910B015C
:10AD8000806204C0F89480910B018F7D80930B0149
:10AD90009FBF80917508843010F40E94AF330E94E9
:10ADA000847DC090A606D090A706E090A806F090FB
:10ADB000A906C114D104E104F104B9F00091A2067E
:10ADC0001091A3062091A4063091A5060C0D1D1D1F
:10ADD0002E1D3F1D6B017C01C01AD10AE20AF30A45
:10ADE000F7FC03C08CEF9AE041C0C0901F02D090E6
:10ADF0002002E0902102F0902202C114D104E1046B
:10AE0000F104D9F00091A2061091A3062091A406A6
:10AE10003091A5060C0D1D1D2E1D3F1DDC01CB0123
:10AE2000801B910BA20BB30BB7FD07C09091D40B05
:10AE30008091D50B981709F4A6C18091C606909110
:10AE4000C706909902C0019604C0181619062CF482
:10AE500001979093C7068093C6068091C60690918D
:10AE6000C7068E3E92401CF083EF9AE022DF0E94DC
:10AE7000847D0091C2061091C3062091C4063091D2
:10AE8000C5066B017C01C01AD10AE20AF30AF7FC7D
:10AE900046C08B019C010C53164F2F4F3F4F009320
:10AEA000C2061093C3062093C4063093C5064F9B79
:10AEB0007CC17A9B7AC12091060120FF76C1209146
:10AEC000E613211172C1029B70C10091BE06109160
:10AED000BF062091C0063091C1060115110521055C
:10AEE000310599F0DC01CB01801B910BA20BB30B58
:10AEF00080569A4EA109B1098827B7FD83959927F5
:10AF0000AA27BB27C82FC19501C0C0E06C2F87E0DE
:10AF10000E94077C6C2F70E087E00E94857C609126
:10AF20007C089091D40B8091D50B981791F0E0910B
:10AF3000D50B29E4E29FF0011124EE59F04F608116
:10AF40008091D50B9091D40B891719F08F5F8F707A
:10AF5000F9CF70E089E00E94857C80917B0888238E
:10AF600009F4FBC000913E0210913F02D0914002D3
:10AF7000C09141026091800870918108072E000CF9
:10AF8000880B990B0E9460ED20E030E040E050E437
:10AF90000E9459E598014D2F5C2F0E945AED87FDC4
:10AFA000DCC0F090D50B912CA12CB12CE12C89E4C4
:10AFB000882E8091D40BF81609F45CC08F2D90E098
:10AFC000889EF001899EF00D1124E55EF04F4281CC
:10AFD000538164817581452B462B472B81F4468133
:10AFE000578160857185452B462B472B41F442855F
:10AFF000538564857585452B462B472BB1F1889E7B
:10B000009001899E300D1124C901855E904F6C011D
:10B01000FC0166857785808991890E9460ED2B010E
:10B020003C01F60162897389848995890E945EEDED
:10B030009B01AC01C301B2010E9445E6F60123A1C8
:10B0400034A145A156A10E94BFED3B016C019B01BB
:10B05000AC01692D7A2D8B2D9E2D0E945AED87FF14
:10B0600004C0962CA72CBC2CED2C81E08F0D8F708A
:10B07000F82E9FCF2091360230913702409138024E
:10B0800050913902692D7A2D8B2D9E2D0E94BFED96
:10B090009B01AC01B8018D2F9C2F0E9459E56B01DB
:10B0A0007C0198014D2F5C2F0E945AED87FD14C042
:10B0B00000913A0210913B02D0913C02C0913D02B6
:10B0C00098014D2F5C2FB601C7010E94A1E7181609
:10B0D0001CF08601DE2DCF2DC090BA06D090BB06A5
:10B0E000E090BC06F090BD0698014D2F5C2FC70183
:10B0F000B6010E94A1E71816E4F420E037ED43EA18
:10B100005CE3B8018D2F9C2F0E94BFED4B015C01C9
:10B1100028E431EE4AE75FE3C701B6010E94BFEDC4
:10B120009B01AC01C501B4010E9459E58B01D82FE8
:10B13000C92FC801AD2FBC2F8093BA069093BB06D0
:10B14000A093BC06B093BD06B8018D2F9C2F0E9422
:10B15000B6E670938108609380080E94E5BA82E0A9
:10B160009CE0DF91CF911F910F91FF90EF90DF90C6
:10B17000CF90BF90AF909F908F907F906F905F9097
:10B180004F900C9473305F9A1092CE068A9A109268
:10B19000CF069FB7F89480910801816080930801E1
:10B1A0009FBF1092D006129A48CE6093BE0670934D
:10B1B000BF068093C0069093C10687CE2F923F9220
:10B1C0004F925F926F927F928F929F92AF92BF92B7
:10B1D000CF92DF92EF92FF920F931F93CF93DF9363
:10B1E000CDB7DEB7E0970FB6F894DEBF0FBECDBF88
:10B1F00082E090E00E9497BD69877A878B879C8761
:10B2000081E090E00E9497BD2B013C0180E090E03E
:10B210000E9497BD6D8F7E8F8F8F98A38091FE0BBC
:10B220009091FF0BA091000CB091010C89A39AA3FF
:10B23000ABA3BCA39C01AD016091F60B7091F70B21
:10B240008091F80B9091F90B0E9458E54B015C013D
:10B250008091FA0B9091FB0BA091FC0BB091FD0B30
:10B260008DA39EA3AFA3B8A79C01AD016091F20B83
:10B270007091F30B8091F40B9091F50B0E9458E5BF
:10B280006B017C012D8D3E8D4F8D58A1C301B20104
:10B290000E9458E56D837E838F839887A501940172
:10B2A000C501B4010E94BFED2B013C01A70196012D
:10B2B000C701B6010E94BFED9B01AC01C301B20101
:10B2C0000E9459E52B013C012D813E814F8158851B
:10B2D000CA01B9010E94BFED9B01AC01C301B201DB
:10B2E0000E9459E50E94EAE769837A838B839C83F5
:10B2F0009B01AC01C501B4010E9445E6698B7A8BC4
:10B300008B8B9C8B29813A814B815C81C701B60173
:10B310000E9445E66D8B7E8B8F8B988F29813A81B9
:10B320004B815C816D817E818F8198850E9445E68D
:10B33000698F7A8F8B8F9C8F29A13AA14BA15CA139
:10B340006091B6067091B7068091B8069091B906E3
:10B350000E9458E54B015C012DA13EA14FA158A5CB
:10B360006091EE0B7091EF0B8091F00B9091F10BCF
:10B370000E9458E56B017C012D8D3E8D4F8D58A1AB
:10B3800069857A858B859C850E9458E56D877E87C7
:10B390008F87988BA501940169897A898B899C890B
:10B3A0000E94BFED2B013C01A70196016D897E89AA
:10B3B0008F89988D0E94BFED9B01AC01C301B20142
:10B3C0000E9459E52B013C012D853E854F8558890A
:10B3D000698D7A8D8B8D9C8D0E94BFED9B01AC0198
:10B3E000C301B2010E9459E56D837E838F839887E4
:10B3F0009B01AC0169897A898B899C890E94BFED88
:10B400009B01AC01C501B4010E9458E569877A87A8
:10B410008B879C872D813E814F8158856D897E89E0
:10B420008F89988D0E94BFED9B01AC01C701B601C9
:10B430000E9458E54B015C012D813E814F8158856A
:10B44000698D7A8D8B8D9C8D0E94BFED9B01AC0127
:10B450006D857E858F8598890E9458E56B017C01FA
:10B4600029853A854B855C85CA01B9010E94BFEDEB
:10B470002B013C01A5019401C501B4010E94BFED5F
:10B480009B01AC01C301B2010E9459E52B013C01B3
:10B49000A7019601C701B6010E94BFED9B01AC0157
:10B4A000C301B2010E9459E50E94EAE72B013C0169
:10B4B0009B01AC0169857A858B859C850E9445E658
:10B4C0006D877E878F87988BA3019201C501B40198
:10B4D0000E9445E669A77AA78BA79CA7A3019201C2
:10B4E000C701B6010E9445E66DA77EA78FA798AB5E
:10B4F0008091E60B9091E70BA091E80BB091E90BDE
:10B5000089879A87AB87BC872091DE0B3091DF0B50
:10B510004091E00B5091E10BBC01CD010E9458E538
:10B520006B017C0129813A814B815C81CA01B9019F
:10B530000E94BFED9B01AC01C701B6010E9459E515
:10B540006B017C0129813A814B815C81CA01B9017F
:10B550000E9459E59B01AC01C701B6010E9445E676
:10B5600069837A838B839C832091D60B3091D70B90
:10B570004091D80B5091D90B69857A858B859C8534
:10B580000E9458E56B017C012D813E814F815885D9
:10B59000CA01B9010E94BFED4B015C01A3019201F8
:10B5A000C301B2010E94BFED9B01AC01C501B40112
:10B5B0000E9459E59B01AC01C701B6010E9459E503
:10B5C00020E030E040E05FE30E94BFED6B017C01D2
:10B5D00029813A814B815C816D817E818F81988543
:10B5E0000E94BFED9B01AC01C701B6010E9458E566
:10B5F000A30192010E9445E66B017C0129813A81F9
:10B600004B815C81CA01B9010E94BFED4B015C0115
:10B61000A7019601C701B6010E94BFED9B01AC01D5
:10B62000C501B4010E9459E59B01AC0169857A8589
:10B630008B859C850E9458E50E94EAE76D837E8396
:10B640008F8398878AEA282E86E0382E29813A81CE
:10B650004B815C8169897A898B899C890E94BFEDC5
:10B660009B01AC0169A17AA18BA19CA10E9459E523
:10B670004B015C01A70196016D857E858F859889B8
:10B680000E94BFED9B01AC01C501B4010E9459E5C8
:10B690004B015C012DA53EA54FA558A96D897E895A
:10B6A0008F89988D0E94BFED2B013C0129A53AA5F9
:10B6B0004BA55CA5698D7A8D8B8D9C8D0E94BFED0D
:10B6C0009B01AC01C301B2010E9458E52D813E816E
:10B6D0004F8158850E94BFED9B01AC01C501B401AB
:10B6E0000E9458E54B015C0102EE1EE020E030E0D4
:10B6F000A901D8016D917D918D919C910E9459E590
:10B70000E6EDFEE020813181428153810E9459E5BE
:10B710009B01AC01C501B4010E9459E5D1016D93B3
:10B720007D938D939C93139729813A814B815C8102
:10B730006D897E898F89988D0E94BFED9B01AC0138
:10B740006DA17EA18FA198A50E9459E54B015C01D6
:10B75000A701960169A57AA58BA59CA50E94BFEDBE
:10B760009B01AC01C501B4010E9459E54B015C018C
:10B770002D853E854F855889698D7A8D8B8D9C8D61
:10B780000E94BFED2B013C012DA53EA54FA558A958
:10B7900069897A898B899C890E94BFED9B01AC01E4
:10B7A000C301B2010E9458E52D813E814F81588529
:10B7B0000E94BFED9B01AC01C501B4010E9458E598
:10B7C0004B015C0120E030E0A901F8016481758142
:10B7D000868197810E9459E52091DA0E3091DB0E27
:10B7E0004091DC0E5091DD0E0E9459E59B01AC01A9
:10B7F000C501B4010E9459E5D10114966D937D9362
:10B800008D939C93179729813A814B815C81698D37
:10B810007A8D8B8D9C8D0E94BFED9B01AC016D8D4F
:10B820007E8D8F8D98A10E9459E54B015C01A70187
:10B8300096016DA57EA58FA598A90E94BFED9B01DD
:10B84000AC01C501B4010E9459E56B017C0129A539
:10B850003AA54BA55CA569897A898B899C890E9448
:10B86000BFED4B015C012D853E854F8558896D8963
:10B870007E898F89988D0E94BFED9B01AC01C50127
:10B88000B4010E9458E52D813E814F8158850E9468
:10B89000BFED9B01AC01C701B6010E9458E56B01E9
:10B8A0007C0120E030E0A901F80160857185828586
:10B8B00093850E9459E52091DE0E3091DF0E409174
:10B8C000E00E5091E10E0E9459E59B01AC01C701C9
:10B8D000B6010E9459E5D10118966D937D938D9321
:10B8E0009C931B97E0960FB6F894DEBF0FBECDBFBA
:10B8F000DF91CF911F910F91FF90EF90DF90CF904C
:10B90000BF90AF909F908F907F906F905F904F907F
:10B910003F902F9008954F925F926F927F928F92F7
:10B920009F92AF92BF92CF92DF92EF92FF920F93CE
:10B930001F93CF93DF93CDB7DEB728970FB6F89458
:10B94000DEBF0FBECDBF7C0182EEC82E8EE0D82EAA
:10B95000F6012081318142815381F701608171813B
:10B96000828193810E9458E506ED1EE0F801208156
:10B970003181428153810E9458E52B013C01F6013F
:10B980002481358146815781F701648175818681E3
:10B9900097810E9458E5F8012481358146815781BD
:10B9A0000E9458E54B015C01F601208531854285F6
:10B9B0005385F70160857185828593850E9458E5DE
:10B9C000F80120853185428553850E9458E56B0139
:10B9D0007C01A30192016091FE0B7091FF0B80919D
:10B9E000000C9091010C0E9458E569837A838B8347
:10B9F0009C83A50194016091FA0B7091FB0B8091DF
:10BA0000FC0B9091FD0B0E9458E56D837E838F8324
:10BA1000988729813A814B815C81CA01B9010E94D2
:10BA2000BFED69837A838B839C832D813E814F8117
:10BA30005885CA01B9010E94BFED9B01AC01698123
:10BA40007A818B819C810E9459E59B01AC016091B8
:10BA5000E60B7091E70B8091E80B9091E90B0E9447
:10BA600058E50E94EAE79B01AC010FE01FE0C70127
:10BA7000B6010E9459E5F801608371838283938344
:10BA8000A30192016091F60B7091F70B8091F80B76
:10BA90009091F90B0E9458E569837A838B839C838C
:10BAA000A50194016091F20B7091F30B8091F40B5E
:10BAB0009091F50B0E9458E56D837E838F83988764
:10BAC00029813A814B815C81CA01B9010E94BFED95
:10BAD00069837A838B839C832D813E814F81588536
:10BAE000CA01B9010E94BFED9B01AC0169817A8155
:10BAF0008B819C810E9459E59B01AC016091DE0B1A
:10BB00007091DF0B8091E00B9091E10B0E9458E562
:10BB10000E94EAE79B01AC01C701B6010E9459E50A
:10BB2000F8016483758386839783A30192016091F2
:10BB3000B6067091B7068091B8069091B9060E943A
:10BB400058E52B013C01A50194016091EE0B709129
:10BB5000EF0B8091F00B9091F10B0E9458E54B0197
:10BB60005C01A3019201C301B2010E94BFED2B0150
:10BB70003C01A5019401C501B4010E94BFED9B01E8
:10BB8000AC01C301B2010E9459E59B01AC01609177
:10BB9000D60B7091D70B8091D80B9091D90B0E9446
:10BBA00058E50E94EAE79B01AC01C701B6010E947B
:10BBB00059E5F801608771878287938728960FB6C9
:10BBC000F894DEBF0FBECDBFDF91CF911F910F91D3
:10BBD000FF90EF90DF90CF90BF90AF909F908F90AD
:10BBE0007F906F905F904F9008954F925F926F9209
:10BBF0007F928F929F92AF92BF92CF92DF92EF92FD
:10BC0000FF9249015A0120E030E0A9010E9459E564
:10BC10006B017C0127ED33EB4DE55FEB0E94BFED3F
:10BC20006093FE0B7093FF0B8093000C9093010CBC
:10BC300020E030E040E05FEBC701B6010E94BFEDBD
:10BC40002B013C016093FA0B7093FB0B8093FC0B70
:10BC50009093FD0B27ED33EB4DE55FE3C701B60194
:10BC60000E94BFED6093F60B7093F70B8093F80B77
:10BC70009093F90B4092F20B5092F30B6092F40BFD
:10BC80007092F50B1092B6061092B7061092B80695
:10BC90001092B906C092EE0BD092EF0BE092F00B2F
:10BCA000F092F10B2091EA0B3091EB0B4091EC0BF1
:10BCB0005091ED0BC501B4010E9459E59B01AC0107
:10BCC0000E94BFED6093E60B7093E70B8093E80B47
:10BCD0009093E90B2091E20B3091E30B4091E40B40
:10BCE0005091E50BC501B4010E9459E59B01AC01DF
:10BCF0000E94BFED6093DE0B7093DF0B8093E00B2F
:10BD00009093E10B2091DA0B3091DB0B4091DC0B2F
:10BD10005091DD0BC501B4010E9459E59B01AC01B6
:10BD20000E94BFED6093D60B7093D70B8093D80B16
:10BD30009093D90BFF90EF90DF90CF90BF90AF9092
:10BD40009F908F907F906F905F904F9008952F926B
:10BD50003F924F925F926F927F928F929F92AF929B
:10BD6000BF92CF92DF92EF92FF920F931F93CF93E8
:10BD7000DF9300D000D0CDB7DEB78C012091E20E6A
:10BD80003091E30E4091E40E5091E50EDC016D918F
:10BD90007D918D919C910E9458E52091D60E309115
:10BDA000D70E4091D80E5091D90E0E9458E56B01E4
:10BDB0007C018091730690917406BC01990F880BE9
:10BDC000990B0E9460ED9B01AC01C701B6010E9476
:10BDD00058E56B017C014091770650917806BA01D5
:10BDE000550F880B990B0E9460ED9B01AC01C701B8
:10BDF000B6010E9445E64B015C012091E60E3091B0
:10BE0000E70E4091E80E5091E90EF80164817581CA
:10BE1000868197810E9458E52091DA0E3091DB0EE1
:10BE20004091DC0E5091DD0E0E9458E56B017C01C3
:10BE30008091750690917606BC01990F880B990B3D
:10BE40000E9460ED9B01AC01C701B6010E9458E55C
:10BE50006B017C018091790690917A06BC01990F63
:10BE6000880B990B0E9460ED9B01AC01C701B601E4
:10BE70000E9445E66B017C01C501B4010E94EBE61E
:10BE80002B013C0120E030E0A9010E945AED87FD22
:10BE900010C020E030E040E051E4C301B2010E9454
:10BEA000A1E718164CF0C301B2010E94B6E68B015F
:10BEB00005C000E010E002C008E010E0C701B601D4
:10BEC0000E94EBE62B013C0120E030E0A9010E943A
:10BED0005AED87FD15C020E030E040E051E4C30199
:10BEE000B2010E94A1E718160CF400C1C301B2010F
:10BEF0000E94B6E67E836D83073011056CF406C0A0
:10BF0000073011050CF0EBC01E821D82A8014F5FA7
:10BF10005F4F5A83498304C088E090E09A83898305
:10BF2000AD81BE81179774F42D803E80BFEF2B1A30
:10BF30003B0A0BC088E090E09A838983A8E0B0E0D8
:10BF4000BE83AD8378E0272E312CB801012E000C82
:10BF5000880B990B0E9460ED9B01AC01C501B401F7
:10BF60000E9458E54B015C01ED81FE81BF01FF0F8E
:10BF7000880B990B0E9460ED9B01AC01C701B601D3
:10BF80000E9458E56B017C0120E030E0A901C50169
:10BF9000B4010E945AED87FF03C0812C912C5401FB
:10BFA00020E030E0A901C701B6010E945AED87FFE9
:10BFB00003C0C12CD12C760129E0209FC001219F14
:10BFC000900D1124ED81FE81E80FF91FEE0FFF1F88
:10BFD000EE0FFF1FE15DFA4F408051806280738059
:10BFE00049815A81249F8001259F100D11242D81A4
:10BFF0003E81200F311F220F331F220F331FD90123
:10C00000A15DBA4F2D913D914D915C9129833A8369
:10C010004B835C83FC01E20DF31DEE0FFF1FEE0F5F
:10C02000FF1FE15DFA4FA30192016081718182815E
:10C0300093810E9458E5A70196010E94BFED9B01E4
:10C04000AC01C301B2010E9459E52B013C01F8018A
:10C05000E20DF31DEE0FFF1FEE0FFF1FE15DFA4F24
:10C0600029813A814B815C816081718182819381D8
:10C070000E9458E5A70196010E94BFED9B01AC010B
:10C0800069817A818B819C810E9459E5A30192018B
:10C090000E9458E59B01AC01C501B4010E94BFEDAF
:10C0A0009B01AC01C301B2010E9459E526960FB66F
:10C0B000F894DEBF0FBECDBFDF91CF911F910F91DE
:10C0C000FF90EF90DF90CF90BF90AF909F908F90B8
:10C0D0007F906F905F904F903F902F90089548E031
:10C0E00050E05A8349831E821D821ECF07301105FE
:10C0F0000CF020CF28E030E03E832D8307CF2F9235
:10C100003F924F925F926F927F928F929F92AF92E7
:10C11000BF92CF92DF92EF92FF920F931F93CF9334
:10C12000DF93CDB7DEB7CC55D1090FB6F894DEBF9B
:10C130000FBECDBF0E949D328091E41383FD97C056
:10C14000C090FB0ED090FC0EE090FD0EF090FE0E25
:10C1500020910B0F30910C0F40910D0F50910E0F4D
:10C16000C701B6010E945AED882309F480C080916E
:10C170004F09811136C020914C0230914D024091FF
:10C180004E0250914F0260919E0870919F088091DD
:10C19000A0089091A1080E945AED87FF22C0C0928A
:10C1A0000B0FD0920C0FE0920D0FF0920E0FE1E406
:10C1B000F7E184917F012FEFE21AF20A882321F040
:10C1C0000E94A832F701F5CFE8EDFAE084917F01F3
:10C1D0003FEFE31AF30A882321F00E94A832F70107
:10C1E000F5CFC090FB0ED090FC0EE090FD0EF090CD
:10C1F000FE0E20910B0F30910C0F40910D0F5091BE
:10C200000E0FC701B6010E9458E50E94B6E697FFDF
:10C2100007C090958095709561957F4F8F4F9F4F88
:10C22000693C71058105910514F1C0920B0FD09204
:10C230000C0FE0920D0FF0920E0FE1E4F7E1849104
:10C240007F019FEFE91AF90A882321F00E94A832A2
:10C25000F701F5CFE9EBFAE084917F01AFEFEA1A3D
:10C26000FA0A882321F00E94A832F701F5CF6091E5
:10C27000A0027091A102072E000C880B990B0E945E
:10C2800060ED2091A2023091A3024091A40250914E
:10C29000A5020E94BFED2AE037ED43E25CE30E9475
:10C2A000BFED63966CAF7DAF8EAF9FAF639740904D
:10C2B000EF0E5090F00E6090F10E7090F20E209103
:10C2C000FF0E3091000F4091010F5091020FC301FA
:10C2D000B2010E945AED811133C08090F30E90900C
:10C2E000F40EA090F50EB090F60E2091030F309151
:10C2F000040F4091050F5091060FC501B4010E9433
:10C300005AED81111DC0C090EE0E49825A826B8297
:10C310007C828D829E82AF82B8868091F70E90914A
:10C32000F80EA091F90EB091FA0E89879A87AB8723
:10C33000BC87CE0101960E945932CE01019613C3EB
:10C340000FEE1EE09FEFC92E9EE0D92E7E01B1E2D6
:10C35000EB0EF11CF80161917191819191918F0126
:10C36000D6012D913D914D915D916D010E9458E551
:10C37000F70161937193819391937F01FEE00F3FE9
:10C380001F0741F749A05AA06BA07CA08DA09EA0DA
:10C39000AFA0B8A489A59AA5ABA5BCA52F968CAFD4
:10C3A0009DAFAEAFBFAF2F97A3019201C301B20102
:10C3B0000E94BFED6B017C01A5019401C501B40190
:10C3C0000E94BFED9B01AC01C701B6010E9459E577
:10C3D0006B017C012F962CAD3DAD4EAD5FAD2F971F
:10C3E000CA01B9010E94BFED9B01AC01C701B601B2
:10C3F0000E9459E50E94EAE76B017C012DEB37E3CF
:10C4000046E855E30E945AED87FF11C0CDA4DEA493
:10C41000EFA4F8A820E030E0A901C701B6010E940E
:10C42000A1E7181624F0F7FAF094F7F8F0942DEB42
:10C4300037E346E855E3C701B6010E945AED87FD90
:10C44000A6C263962CAD3DAD4EAD5FAD6397C701FF
:10C45000B6010E9445E62091EF023091F002409132
:10C46000F1025091F2020E94BFED0E94BCE61B0156
:10C47000672B19F422242394312CB10180E090E041
:10C480000E945EED6B017C019B01AC01C301B20116
:10C490000E9445E6698B7A8B8B8B9C8BA70196015A
:10C4A000C501B4010E9445E66D8B7E8B8F8B988F02
:10C4B000A70196012F966CAD7DAD8EAD9FAD2F97E8
:10C4C0000E9445E6698F7A8F8B8F9C8FA70196011A
:10C4D0006DA57EA58FA598A90E9445E66D8F7E8FDC
:10C4E0008F8F98A320E1EFEFFEE0CE010196DC01F3
:10C4F00001900D922A95E1F7DE0151962B96BFAF80
:10C50000AEAF2B976C968FAF6C976D969FAF6D9774
:10C5100031E0231A310809F4FAC18E010F5E1F4F72
:10C520006C96EFAC6C976D96FFAC6D97F80121910E
:10C530003191419151918F01D7016D917D918D91F3
:10C540009C910E9459E5F7016193719381939193B6
:10C550007F012B962EAD3FAD2B97E217F30731F7F6
:10C560002091E20E3091E30E4091E40E5091E50EE1
:10C5700069817A818B819C810E9458E52091D60E39
:10C580003091D70E4091D80E5091D90E0E9458E5A7
:10C590002B013C012091E60E3091E70E4091E80E10
:10C5A0005091E90E6D817E818F8198850E9458E5BA
:10C5B0002091DA0E3091DB0E4091DC0E5091DD0EB1
:10C5C0000E9458E52F966CAF7DAF8EAF9FAF2F972F
:10C5D0002091EA0E3091EB0E4091EC0E5091ED0E51
:10C5E00069857A858B859C850E9458E52091DE0EB1
:10C5F0003091DF0E4091E00E5091E10E0E9458E51F
:10C6000067966CAF7DAF8EAF9FAF6797A301920126
:10C610006091FE0B7091FF0B8091000C9091010CCA
:10C620000E9458E54B015C012F962CAD3DAD4EADFF
:10C630005FAD2F976091FA0B7091FB0B8091FC0B13
:10C640009091FD0B0E9458E56B017C01A5019401BE
:10C65000C501B4010E94BFED4B015C01A701960129
:10C66000C701B6010E94BFED9B01AC01C501B40139
:10C670000E9459E59B01AC016091E60B7091E70BBC
:10C680008091E80B9091E90B0E9458E50E94EAE73F
:10C690009B01AC0167966CAD7DAD8EAD9FAD67978C
:10C6A0000E9459E56B966CAF7DAF8EAF9FAF6B97D5
:10C6B00060930F0F7093100F8093110F9093120FD0
:10C6C000A30192016091F60B7091F70B8091F80B2A
:10C6D0009091F90B0E9458E54B015C012F962CAD0F
:10C6E0003DAD4EAD5FAD2F976091F20B7091F30BA6
:10C6F0008091F40B9091F50B0E9458E56B017C0141
:10C70000A5019401C501B4010E94BFED4B015C017C
:10C71000A7019601C701B6010E94BFED9B01AC01C4
:10C72000C501B4010E9459E59B01AC016091DE0B8B
:10C730007091DF0B8091E00B9091E10B0E9458E526
:10C740000E94EAE79B01AC0167966CAD7DAD8EADB2
:10C750009FAD67970E9459E56B017C016093130FB1
:10C760007093140F8093150F9093160FA3019201ED
:10C770006091B6067091B7068091B8069091B9069F
:10C780000E9458E52B013C012F962CAD3DAD4EADDE
:10C790005FAD2F976091EE0B7091EF0B8091F00BD6
:10C7A0009091F10B0E9458E54B015C01A3019201AD
:10C7B000C301B2010E94BFED2B013C01A501940110
:10C7C000C501B4010E94BFED9B01AC01C301B201E0
:10C7D0000E9459E59B01AC016091D60B7091D70B7B
:10C7E0008091D80B9091D90B0E9458E50E94EAE7FE
:10C7F0009B01AC0167966CAD7DAD8EAD9FAD67972B
:10C800000E9459E52B013C016093170F7093180F9C
:10C810008093190F90931A0F80914E098823B9F1D4
:10C820006C968FAD6C976D969FAD6D9790DA4B01BE
:10C830005C019B01AC016B966CAD7DAD8EAD9FAD87
:10C840006B970E9459E560930F0F7093100F8093C0
:10C85000110F9093120FA5019401C701B6010E9418
:10C8600059E56093130F7093140F8093150F9093F5
:10C87000160FA5019401C301B2010E9459E560930E
:10C88000170F7093180F8093190F90931A0FC09081
:10C89000EE0E8091170F9091180FA091190FB09183
:10C8A0001A0F4091130F5091140F6091150F709152
:10C8B000160F00910F0F1091100F2091110F309152
:10C8C000120F21960CAF1DAF2EAF3FAF21972596CB
:10C8D0004CAF5DAF6EAF7FAF259729968CAF9DAF04
:10C8E000AEAFBFAF29976396ECACFDAC0EAD1FADFC
:10C8F00063979E01235F3F4FAE014B5B5F4FBE01CD
:10C900006F5B7F4FCE01CD960E94C68901CEC0904D
:10C91000EE0E8091EF0E9091F00EA091F10EB0917D
:10C92000F20E89AB9AABABABBCAB8091F30E90919E
:10C93000F40EA091F50EB091F60E8DAB9EABAFABA1
:10C94000B8AF8091F70E9091F80EA091F90EB091CA
:10C95000FA0E89AF9AAFABAFBCAFCE01C1960E94C1
:10C960005932CE01C1960E948B5C6396ECACFDAC53
:10C970000EAD1FAD63972BEF3EE047E15FE063E153
:10C980007FE08FE09FE00E94C6890E94C39BC45A4B
:10C99000DF4F0FB6F894DEBF0FBECDBFDF91CF9152
:10C9A0001F910F91FF90EF90DF90CF90BF90AF90CD
:10C9B0009F908F907F906F905F904F903F902F90BF
:10C9C0000895CF93DF930E949D32E0917308F0E0C9
:10C9D000EE52F94F8081882381F0E6EBFAE08491F2
:10C9E000EF012196882321F00E94A832FE01F7CFA3
:10C9F0008AE0DF91CF910C94A832DF91CF91089516
:10CA0000CF92DF92EF92FF920F931F93CF93DF931A
:10CA10006C017A018B01C0E0D0E0CE15DF0589F012
:10CA2000D8016D918D01D601ED91FC910190F081BD
:10CA3000E02DC6011995892B11F47E0102C02196C3
:10CA4000ECCFC701DF91CF911F910F91FF90EF9035
:10CA5000DF90CF9008950E9444E80F931F93CF93E7
:10CA6000DF93C82FD42F80E00E94EEA7C11102C02F
:10CA700080E201C08EE30E94E5AF8091400C8823E4
:10CA800029F01092520C00E41CE002C003E31CE009
:10CA9000C2E1F80161918F01662311F0C1110EC04E
:10CAA000CC2329F080E20E94E5AFC150F9CF8D2F51
:10CAB000DF91CF911F910F910C94E5AF88E99BE036
:10CAC0000E94527EC150E5CF2CE933E549E45EE394
:10CAD00060919008709191088091920890919308CC
:10CAE0000E9445E660932E0270932F0280933002DD
:10CAF0009093310208952CE933E549E45EE36091B7
:10CB000094087091950880919608909197080E94DA
:10CB1000BFED60933202709333028093340290939E
:10CB200035020895FF920F931F93CF93DF931092D6
:10CB300094068091BB0E9091BC0EA091BD0EB09159
:10CB4000BE0E81309048A105B10540F01092BB0E99
:10CB50001092BC0E1092BD0E1092BE0E6091BB0ED4
:10CB60007091BC0E8091BD0E9091BE0E25E030E01C
:10CB700040E050E00E9435F1C22F80918E081816D7
:10CB8000F4F4022E000C330B482F082E000C550B2A
:10CB9000415051092417350794F0CFEFC80F25E015
:10CBA000C29FC0011124092E000CAA0BBB0B80935D
:10CBB000BB0E9093BC0EA093BD0EB093BE0E109210
:10CBC0008A0680918906C81714F4C093890680915B
:10CBD0008906082E000C990B03962C2F0C2E000CA6
:10CBE000330B8217930724F48DEF8C0F8093890603
:10CBF00010918906F12C112329F08091950B811158
:10CC00001CC046C080919D02882351F081E0C11173
:10CC100080E003E023E047E35EE06F2D0E946CB705
:10CC200080919506882349F3C111E7CF0E94667071
:10CC300080918A06882309F37BC08091960B882314
:10CC400039F18091970B882319F1113019F58091F2
:10CC50009D02882359F081E0C13009F080E00EE3A5
:10CC60002EE34DE25EE06F2D0E946CB78091950639
:10CC7000882309F45BC0C13009F058C08DE89BE6F9
:10CC80000E94CE5480918A06882309F44FC050C078
:10CC9000D1E001C0D2E01D131FC080919D02882306
:10CCA00051F081E0C11380E00EE32EE344E25EE048
:10CCB0006F2D0E946CB780919506882361F0C11397
:10CCC0000AC08BE99BE60E94CE5480918A068111AE
:10CCD0002FC0DC2F01C0D12F81E08D0F181749F034
:10CCE000F3941F5F84E0F81286CFDE5FD0938E0846
:10CCF0001FC080919D02882351F081E0C11380E024
:10CD00000EE32EE349E15EE06F2D0E946CB7809147
:10CD10009506882329F3C113E3CF89EA9BE60E9495
:10CD2000CE5480918A068823D9F202C0D2E0D4CFB3
:10CD3000DF91CF911F910F91FF9008952F923F9215
:10CD40004F925F926F927F928F929F92AF92BF921B
:10CD5000CF92DF92EF92FF920F931F93CF93DF93C7
:10CD600000D0CDB7DEB7109294068091BB0E9091A3
:10CD7000BC0EA091BD0EB091BE0E81309048A105B1
:10CD8000B10540F01092BB0E1092BC0E1092BD0E79
:10CD90001092BE0E6091BB0E7091BC0E8091BD0EC4
:10CDA0009091BE0E25E030E040E050E00E9435F169
:10CDB000D22E809198081816FCF4022E000C330B2A
:10CDC000482F082E000C550B4150510924173507E8
:10CDD0009CF0DD24DA94D80EA5E0DA9EC00111247F
:10CDE000092E000CAA0BBB0B8093BB0E9093BC0EBC
:10CDF000A093BD0EB093BE0E10928A068091890654
:10CE0000D81614F4D092890680918906082E000C59
:10CE1000990B03962D2D0D2C000C330B82179307C5
:10CE200024F48DEF8D0D80938906B0918906BB8324
:10CE3000C12C34E6432E512C612C712C44EF842EEE
:10CE40004DE3942E4FE0A42EB12C57EF252E5DE438
:10CE5000352E2B81211118C080919D02882351F01D
:10CE600081E0D11080E003E023E047E35FE06C2D38
:10CE70000E946CB780919506882309F45BC1D1109C
:10CE800059C10E94667052C18B81813061F58091D9
:10CE90009D02882369F080E898E00E9498819C01B7
:10CEA00081E0D81280E040E35FE06C2D0E94B3E4A3
:10CEB00080919506882309F43DC191E0D9123AC1C9
:10CEC000D0929406109290061092910610929206BB
:10CED0001092930628EE3CE644E051E060E878E0EA
:10CEE00089E29FE030C0AB81A23081F580919D0244
:10CEF000882371F08EE798E00E9498819C0181E080
:10CF0000B2E0DB1280E045E25FE06C2D0E94B3E40A
:10CF100080919506882309F40DC122E0D2120AC13E
:10CF200081E08093940610929006109291061092E0
:10CF300092061092930629EE3CE647E850E06EE731
:10CF400078E081E29FE00E9422E3F0C08B81833091
:10CF500081F580919D02882371F08CE798E00E9412
:10CF600098819C0181E093E0D91280E047E15FE085
:10CF70006C2D0E94B3E480919506882309F4DAC0F1
:10CF8000A3E0DA12D7C081E0809394061092900655
:10CF90001092910610929206109293062FEF30E0B5
:10CFA00040E050E06CE778E08DE09FE00E94C3D95C
:10CFB000BDC0BB81B43029F580919D02882391F0DA
:10CFC00080917B08811103C02CEF3EE002C020E07D
:10CFD0003FE081E094E0D91280E044E05FE06C2D16
:10CFE0000E943ADA80919506882309F4A3C0A4E050
:10CFF000DA12A0C090917B0881E0892780937B089A
:10D0000095C0BB81B53091F580919D028823D1F008
:10D0100060913E0270913F028091400290914102E6
:10D020000E94B6E67A836983CE0101960E949881B8
:10D030009C0181E095E0D91280E045EF5EE06C2D27
:10D040000E94B3E480919506882309F473C0A5E09B
:10D05000DA1270C0E12CF12C02E813E420E030E099
:10D06000A9016EE372E08EEE9EE034C0BB81B63063
:10D07000A1F580919D028823D1F060913A027091D0
:10D080003B0280913C0290913D020E94B6E67A8379
:10D090006983CE0101960E9498819C0181E096E00F
:10D0A000D91280E047EE5EE06C2D0E94B3E48091DF
:10D0B0009506882309F43EC0A6E0DA123BC0E12CB5
:10D0C000F12C02E813E420E030E0A9016AE372E009
:10D0D00080EE9EE00E944CD929C0BB81B73051F54B
:10D0E00080919D02882371F086E392E00E94748013
:10D0F0009C0181E097E0D91280E048ED5EE06C2D64
:10D100000E94B3E4809195068823A1F0A7E0DA128B
:10D1100011C0E12CF12C00E81FE320E030E0A90170
:10D1200066E372E080ED9EE00E94C3D880918A069B
:10D130008111A8C12CE933E549E45EE36091320234
:10D140007091330280913402909135020E9445E63D
:10D15000609394087093950880939608909397082D
:10D160002CE933E549E45EE360912E0270912F02D1
:10D1700080913002909131020E94BFED609390083F
:10D18000709391088093920890939308BB81B83074
:10D1900009F05FC080919D02882371F08AE292E0DD
:10D1A0000E94037F9C0181E098E0D91280E04AEC64
:10D1B0005EE06C2D0E94B3E480919506882309F40B
:10D1C00057C1A8E0DA1254C12BD483E080939D02AA
:10D1D00084EC9EE09093CA0E8093C90E8AE292E09E
:10D1E0009093C80E8093C70E4092C30E5092C40E07
:10D1F0006092C50E7092C60E8092BF0E9092C00EC5
:10D20000A092C10EB092C20E20E030E048EC52E491
:10D2100060912A0270912B0280912C0290912D0234
:10D220000E94BFED20E030E048EC52E40E9458E557
:10D230000E94BCE66093BB0E7093BC0E8093BD0E43
:10D240009093BE0E80E09EE490939F0280939E0296
:10D250000BC1BB81B93009F067C080919D02882362
:10D2600071F084E998E00E94037F9C0181E099E0DD
:10D27000D91280E04EEB5EE06C2D0E94B3E4809109
:10D280009506882309F4F4C0A9E0DA12F1C0C8D3E6
:10D2900083E080939D0288EB9EE09093CA0E80937A
:10D2A000C90EA4E9B8E0B093C80EA093C70E81E000
:10D2B00090E0A0E0B0E08093C30E9093C40EA093E2
:10D2C000C50EB093C60E87E59EE3AFE0B0E0809355
:10D2D000BF0E9093C00EA093C10EB093C20E20E07B
:10D2E00030E048EC52E46091940870919508809188
:10D2F0009608909197080E94BFED20E030E040E84A
:10D300005FE30E9458E50E94BCE66093BB0E7093F9
:10D31000BC0E8093BD0E9093BE0E30929F02209261
:10D320009E028BE795E662C09B819A3009F063C04C
:10D3300080919D02882371F080E998E00E94037F2C
:10D340009C0181E0AAE0DA1280E042EB5EE06C2D05
:10D350000E94B3E480919506882309F489C0BAE05D
:10D36000DB1286C05DD383E080939D028CEA9EE051
:10D370009093CA0E8093C90EA0E9B8E0B093C80E8E
:10D38000A093C70E4092C30E5092C40E6092C50E79
:10D390007092C60E8092BF0E9092C00EA092C10EE7
:10D3A000B092C20E20E030E048EC52E46091900868
:10D3B0007091910880919208909193080E94BFED1E
:10D3C00020E030E048EC52E40E9458E50E94BCE6C0
:10D3D0006093BB0E7093BC0E8093BD0E9093BE0EF7
:10D3E00030929F0220929E0284E695E69093CC0EA6
:10D3F0008093CB0E39C09B819B30C9F480919D02F4
:10D40000882359F081E0ABE0DA1280E00EE32EE3EE
:10D410004BE95EE06C2D0E946CB7809195068823E5
:10D4200039F1BBE0DB1224C086E698E81BC02B81F3
:10D430002C30F1F480919D02882359F081E09CE02A
:10D44000D91280E00EE32EE34AE85EE06C2D0E94E4
:10D450006CB780919506882359F0ACE0DA1208C0C9
:10D4600083E698E80E94CE5480918A0681110AC012
:10D47000C394BB81BF5FBB8324E0C212EACC8DE0C2
:10D48000809398080F900F900F90DF91CF911F918C
:10D490000F91FF90EF90DF90CF90BF90AF909F9053
:10D4A0008F907F906F905F904F903F902F90089556
:10D4B0000F931F93CF93DF93109294068091BB0E2E
:10D4C0009091BC0EA091BD0EB091BE0E81309048DF
:10D4D000A105B10540F01092BB0E1092BC0E109247
:10D4E000BD0E1092BE0E6091BB0E7091BC0E80916D
:10D4F000BD0E9091BE0E25E030E040E050E00E946D
:10D5000035F1C22F80918F081816F4F4022E000C0A
:10D51000330B482F082E000C550B4150510924178E
:10D52000350794F0CFEFC80F25E0C29FC00111244A
:10D53000092E000CAA0BBB0B8093BB0E9093BC0E64
:10D54000A093BD0EB093BE0E10928A0680918906FC
:10D55000C81714F4C093890680918906082E000C20
:10D56000990B03962C2F0C2E000C330B821793076C
:10D5700024F48DEF8C0F8093890610918906D0E0FA
:10D58000111117C080919D02882351F081E0C111D3
:10D5900080E003E023E045E85EE06D2F0E946CB779
:10D5A00080919506882309F4ABC0C111A9C08ED51E
:10D5B000A3C01130D1F480919D02882359F081E0FD
:10D5C000C13009F080E00EE32EE349E75EE06D2F05
:10D5D0000E946CB780919506882309F491C0C130F0
:10D5E00009F08EC08EE996E637C01230D1F48091F2
:10D5F0009D02882359F081E0C23009F080E00EE3FB
:10D600002EE342E75EE06D2F0E946CB78091950695
:10D61000882309F475C0C23009F072C08EEA93E81D
:10D620001BC01330E1F480919D02882359F081E002
:10D63000C33009F080E00EE32EE349E65EE06D2F93
:10D640000E946CB780919506882309F459C0C330B5
:10D6500009F056C08CE492E80E94CE544DC01430BC
:10D66000C1F480919D02882359F081E0C43009F013
:10D6700080E000E22EE34CE55EE06D2F0E946CB787
:10D68000809195068823E1F1C430D1F50E94FE37E0
:10D6900033C01530C1F480919D02882359F081E098
:10D6A000C53009F080E000E22EE340E55EE06D2F3A
:10D6B0000E946CB780919506882311F1C53001F561
:10D6C0000E94643A19C01630D9F480919D028823D3
:10D6D00059F081E0C63009F080E000E22EE34FE32C
:10D6E0005EE06D2F0E946CB780919506882341F013
:10D6F000C63031F40E9462D480918A06811108C03C
:10D70000DF5F1F5FD43009F03BCF87E080938F0845
:10D71000DF91CF911F910F91089580E090E0A0E2FA
:10D72000B1E48093770890937808A0937908B09338
:10D730007A080C94FC4980E090E0A0E8BFE3809375
:10D74000770890937808A0937908B0937A080C949E
:10D75000FC498DEC9CECACECBDE380937708909396
:10D760007808A0937908B0937A080C94FC49AF929A
:10D77000BF92CF92DF92EF92FF920F931F93CF93BE
:10D78000DF93F82E109294068091BB0E9091BC0E00
:10D79000A091BD0EB091BE0E81309048A105B1059B
:10D7A00040F01092BB0E1092BC0E1092BD0E109263
:10D7B000BE0E6091BB0E7091BC0E8091BD0E90911B
:10D7C000BE0E25E030E040E050E00E9435F1C22F6F
:10D7D000809199081816F4F4022E000C330B482F90
:10D7E000082E000C550B415051092417350794F0B1
:10D7F000CFEFC80F25E0C29FC0011124092E000CF5
:10D80000AA0BBB0B8093BB0E9093BC0EA093BD0ED6
:10D81000B093BE0E10928A0680918906C81714F440
:10D82000C093890680918906082E000C990B0396F7
:10D830002C2F0C2E000C330B8217930724F48DEF42
:10D840008C0F8093890610918906D0E02F2D30E04F
:10D85000220F331FC9018E57974F7C01C9018A5788
:10D86000974F6C01C9018657974F5C01111117C082
:10D8700080919D02882351F081E0C11180E003E096
:10D8800023E046E75FE06D2F0E946CB7809195061C
:10D89000882309F48AC0C11188C018D482C011300D
:10D8A00009F580919D02882369F0C5010E94988145
:10D8B0009C0181E0C13009F080E04CE65FE06D2F13
:10D8C0000E94B3E480919506882309F46EC0C130AC
:10D8D00009F06BC02FEF30E040E050E0B50182E688
:10D8E0009FE022C0123019F580919D02882369F0D3
:10D8F000C6010E9498819C0181E0C23009F080E05D
:10D900004BE55FE06D2F0E94B3E48091950688237C
:10D9100009F44BC0C23009F048C024E031E045E0D2
:10D9200050E0B60184E59FE00E94C3D93AC01330AD
:10D93000F9F480919D02882369F0C7010E949881C3
:10D940009C0181E0C33009F080E040E55FE06D2F8D
:10D950000E94B3E480919506882339F1C33029F5FC
:10D9600027E830E045E050E0B7018CE49FE0DCCFF1
:10D970001430D9F480919D02882359F081E0C4309D
:10D9800009F080E000E22EE34FE35FE06D2F0E949C
:10D990006CB780919506882341F0C43031F40E9421
:10D9A000FE3780918A06811108C0DF5F1F5FD43087
:10D9B00009F05CCF85E080939908DF91CF911F91AA
:10D9C0000F91FF90EF90DF90CF90BF90AF900895B0
:10D9D000089508950E94CB9E0C948AAA81E08093BA
:10D9E00074088093940B1092300C87EA9FE00E9499
:10D9F000DFBC8091200C9091210C019781F482E092
:10DA000090E09093210C8093200C0E94847D609381
:10DA10002A0C70932B0C80932C0C90932D0C089552
:10DA20008091DE088A30D8F496E0899FF0011124B5
:10DA3000EE55F74F20919E0230919F023183208353
:10DA40004091BB0E5091BC0E6091BD0E7091BE0E08
:10DA500042835383648375838F5F8093DE080895C8
:10DA600020919E0230919F0228173907E9F0909388
:10DA70009F0280939E024093BB0E5093BC0E609316
:10DA8000BD0E7093BE0E85559D4621F410928F06F3
:10DA90001092DE0888E99BE00E94597E82E0809324
:10DAA0009D0281E080938A0608958F929F92AF92A3
:10DAB000BF92CF92DF92EF92FF920F931F93CF937B
:10DAC000DF93CDB7DEB72A970FB6F894DEBF0FBE4F
:10DAD000CDBF1092940660E080E00E94EEA782E045
:10DAE0000E94E5AF20E030E040E05FE360919E08F7
:10DAF00070919F088091A0089091A1080E9459E51B
:10DB00000E94B6E67A8369838E010F5F1F4FC801BA
:10DB10000E9498810E9467B08FE20E94E5AF6091F9
:10DB2000800870918108072E000C880B990B0E94C9
:10DB300060ED20E030E040E05FE30E9459E50E94A4
:10DB4000B6E67A836983C8010E9463810E9467B048
:10DB500084EA9FE00E94B6B76091800870918108C6
:10DB6000072E000C880B990B0E9460ED20E030E03E
:10DB700040E251E40E945AED87FF03C080E20E9418
:10DB8000E5AF60E08AE00E94EEA780E00E94E5AF8A
:10DB900020E030E040E05FE360919A0870919B08DC
:10DBA00080919C0890919D080E9459E50E94B6E6DC
:10DBB0007A836983C8010E9498810E9467B08FE2CE
:10DBC0000E94E5AF60917E0870917F08072E000CDF
:10DBD000880B990B0E9460ED20E030E040E05FE3AD
:10DBE0000E9459E50E94B6E67A836983C8010E94C3
:10DBF00063810E9467B081EA9FE00E94B6B760919E
:10DC00007E0870917F08072E000C880B990B0E94EC
:10DC100060ED20E030E040E251E40E945AED87FFE1
:10DC200003C080E20E94E5AF0E94847DC090E008BE
:10DC3000D090E108E090E208F090E3089B01AC018D
:10DC40002C193D094E095F0957FD13C02091DF08CB
:10DC500020952093DF08DC01CB018A549C4FAF4F05
:10DC6000BF4F8093E0089093E108A093E208B0933F
:10DC7000E308FF24F3948091DF08811101C0F12CA7
:10DC800061E080E00E94EEA7FF2029F08FE99FE08D
:10DC90000E94B6B70DC08091950B811102C08FE331
:10DCA00005C08091CE068111F1CF80E20E94E5AFE0
:10DCB0006091FF0E7091000F8091010F9091020F03
:10DCC0000E94B6E67A836983C8010E94F4800E94AC
:10DCD00067B080E20E94E5AFFF2029F08DE99FE068
:10DCE0000E94B6B70DC08091960B811102C08FE3E0
:10DCF00005C08091CF068111F1CF80E20E94E5AF8F
:10DD00006091030F7091040F8091050F9091060FA1
:10DD10000E94B6E67A836983C8010E94F4800E945B
:10DD200067B061E08CE00E94EEA7FF2029F08BE94C
:10DD30009FE00E94B6B70DC08091970B811102C081
:10DD40008FE305C08091D0068111F1CF80E20E945F
:10DD5000E5AF2CEA35EC47E257E36091070F70918D
:10DD6000080F8091090F90910A0F0E9459E520E059
:10DD700030E048EC52E40E94BFED0E94B6E66B0131
:10DD80007C0197FD16C0603137E27307810591056C
:10DD9000D4F020E137E240E050E00E9457F1CA01A0
:10DDA000B9012AE030E040E050E00E9457F1605DA8
:10DDB0000BC0F094E094D094C094C11CD11CE11C21
:10DDC000F11C6DE201C060E26093CD0E48EEC41616
:10DDD00043E0D406E104F10494F0C701B60128EE53
:10DDE00033E040E050E00E9457F1CA01B9012AE057
:10DDF00030E040E050E00E9457F1605D01C060E219
:10DE00006093CE0EC701B60124E630E040E050E05A
:10DE10000E9457F16AE0862E912CA12CB12CCA01E8
:10DE2000B901A50194010E9457F1605D6093CF0E86
:10DE3000C701B601A50194010E9457F16B017C0155
:10DE4000672B682B692B79F08EE28093D00ECA0184
:10DE5000B901A50194010E9457F1605D6093D10E54
:10DE600080E38C0D15C0CA01B901A50194010E947F
:10DE700057F1662339F08EE28093D00E605D609397
:10DE8000D10E05C080E28093D10E8093D00E80E247
:10DE90008093D20E1092D30E8DEC9EE00E9467B05C
:10DEA00062E080E00E94EEA786E00E94E5AF80EA93
:10DEB00092E00E9498810E9467B085E20E94E5AFDF
:10DEC00062E087E00E94EEA788E99FE00E94B6B773
:10DED0008091300C882389F12091FE0D222321F1BD
:10DEE0008091A80E9091A90EA091AA0EB091AB0EB0
:10DEF0000097A105B105B9F0BC01CD016D597F4F67
:10DF00008F4F9F4F24E630E040E050E00E9435F113
:10DF10006091AC0E7091AD0E8091AE0E9091AF0EEF
:10DF20000E9435F101C020E030E03A832983C80126
:10DF30000E9498810E9467B004C084E99FE00E941B
:10DF4000B6B785E20E94E5AF0E94959E2CE3C22EF3
:10DF5000D12CE12CF12CA70196010E9435F1CA01C8
:10DF6000B901A70196010E9435F1C9012436310596
:10DF7000B8F47F936F9368E170E00E9429E59F9366
:10DF80008F938AE89FE09F938F931F930F930E9434
:10DF90002BED0FB6F894DEBF0FBECDBF95E012C0DB
:10DFA0007F936F933F932F9382E89FE09F938F938C
:10DFB0001F930F930E942BED0FB6F894DEBF0FBE98
:10DFC000CDBF96E062E083E1891B0E94EEA787E067
:10DFD0000E94E5AFC8010E94A1B763E080E00E9403
:10DFE000EEA788E592E00E94A1B78091950688236C
:10DFF00041F00E94EEB740E050E0BA0187EE91E7B1
:10E000002FDD2091A0023091A1024091BB0E5091D2
:10E01000BC0E6091BD0E7091BE0EC901840F951F9C
:10E020002436310524F4853691053CF416C0243697
:10E03000310531F08436910584F484E690E00DC01A
:10E040004B3051056105710514F00A9706C0463F33
:10E050005F4F6F4F7F4F6CF40A969093A1028093AD
:10E06000A0021092BB0E1092BC0E1092BD0E109228
:10E07000BE0E8091A0029091A1028A3091053CF0E1
:10E08000883E43E094072CF087EE93E002C08AE0DC
:10E0900090E09093A1028093A0022A960FB6F89484
:10E0A000DEBF0FBECDBFDF91CF911F910F91FF90CB
:10E0B000EF90DF90CF90BF90AF909F908F9008959A
:10E0C00040E050E0BA0185E59DE6CACCE091DE086B
:10E0D000EE2381F0E150E093DE0886E0E89FF00156
:10E0E0001124EE55F74F42815381648175818081FF
:10E0F0009181B6CCE5CFFF920F931F93CF93DF931F
:10E10000109294068091BB0E9091BC0EA091BD0E12
:10E11000B091BE0E81309048A105B10540F010923B
:10E12000BB0E1092BC0E1092BD0E1092BE0E6091EE
:10E13000BB0E7091BC0E8091BD0E9091BE0E25E07D
:10E1400030E040E050E00E9435F1C22F8091E508B8
:10E150001816F4F4022E000C330B482F082E000C76
:10E16000550B415051092417350794F0CFEFC80FD4
:10E1700025E0C29FC0011124092E000CAA0BBB0B85
:10E180008093BB0E9093BC0EA093BD0EB093BE0EB9
:10E1900010928A0680918906C81714F4C0938906E4
:10E1A00080918906082E000C990B03962C2F0C2EBB
:10E1B000000C330B8217930724F48DEF8C0F8093A0
:10E1C000890610918906D0E0FF24F394111117C03D
:10E1D00080919D02882351F081E0C11180E003E02D
:10E1E00023E04DE550E16D2F0E946CB780919506BC
:10E1F000882309F4DEC0C111DCC068DFD6C011304D
:10E2000019F580919D02882371F080EA92E00E94C6
:10E2100098819C0181E0C13009F080E047E550E140
:10E220006D2F0E94B3E480919506882309F4C1C044
:10E23000C13009F0BEC027EE33E04AE050E060EAAA
:10E2400072E081E590E1AFC0123069F580919D02E6
:10E25000882371F080E898E00E9498819C0181E019
:10E26000C23009F080E04AE450E16D2F0E94B3E42F
:10E2700080919506882309F49CC0C23009F099C0AA
:10E28000F0929406109290061092910610929206C7
:10E290001092930628EE3CE644E051E060E878E016
:10E2A00083E490E12EC0133079F580919D0288239C
:10E2B00071F08EE798E00E9498819C0181E0C33064
:10E2C00009F080E04FE350E16D2F0E94B3E48091AC
:10E2D0009506882309F46DC0C33009F06AC0F09236
:10E2E0009406109290061092910610929206109247
:10E2F000930629EE3CE647E850E06EE778E08BE3D2
:10E3000090E10E9422E351C0143059F580919D02A2
:10E31000882371F08CE798E00E9498819C0181E04D
:10E32000C43009F080E041E350E16D2F0E94B3E476
:10E33000809195068823E9F1C430D9F5F0929406CE
:10E3400010929006109291061092920610929306E7
:10E350002FEF30E040E050E06CE778E087E290E1BA
:10E3600022C0153031F580919D02882371F082E43E
:10E3700092E00E9498819C0181E0C53009F080E024
:10E3800042E250E16D2F0E94B3E48091950688230C
:10E3900081F0C53071F427EE33E04AE050E062E4EA
:10E3A00072E08DE190E10E94C3D980918A068111CB
:10E3B00008C0DF5F1F5FD43009F008CF86E080938C
:10E3C000E508DF91CF911F910F91FF900895EF9293
:10E3D000FF920F931F93CF93DF9310929406809137
:10E3E000BB0E9091BC0EA091BD0EB091BE0E8130BF
:10E3F0009048A105B10540F01092BB0E1092BC0EE2
:10E400001092BD0E1092BE0E6091BB0E7091BC0EAC
:10E410008091BD0E9091BE0E25E030E040E050E0CE
:10E420000E9435F1C22F8091E4081816F4F4022EF0
:10E43000000C330B482F082E000C550B415051098E
:10E440002417350794F0CFEFC80FE5E0CE9FC00149
:10E450001124092E000CAA0BBB0B8093BB0E9093CA
:10E46000BC0EA093BD0EB093BE0E10928A06809192
:10E470008906C81714F4C093890680918906082E6E
:10E48000000C990B03962C2F0C2E000C330B8217CB
:10E49000930724F48DEF8C0F8093890610918906E1
:10E4A000D0E0E12CF12C112341F08091D40B90911C
:10E4B000D50B891B8F70D9F51AC080919D028823D6
:10E4C00051F081E0C11180E003E023E041E150E13F
:10E4D0006D2F0E946CB780919506882331F3C1118E
:10E4E000E4CFF4DD80918A068823F9F213C180918C
:10E4F000300C81111CC01130E9F480919D028823F9
:10E5000059F081E0C13009F080E00EE32EE344E0F1
:10E5100050E16D2F0E946CB780919506882309F415
:10E5200042C0C13009F03FC088E296E436C01130E5
:10E5300009F4D6C01230C1F480919D02882359F0AD
:10E5400081E0C23009F080E00EE32EE342EF5FE0AD
:10E550006D2F0E946CB780919506882321F1C230FF
:10E5600011F58CE797E419C01330E9F480919D020E
:10E57000882359F081E0C33009F080E00EE32EE3F8
:10E580004AEE5FE06D2F0E946CB78091950688235C
:10E5900051F0C33041F488E59AE60E94CE54809150
:10E5A0008A068111B7C08091310C882309F46FC0AD
:10E5B0008091FE0D882309F459C08091300C882386
:10E5C000D9F01430A1F580919D02882359F081E0A3
:10E5D000C43009F080E000E22EE34EED5FE06D2FE5
:10E5E0000E946CB780919506882309F470C0C430EE
:10E5F00009F06DC0F3D935C01430C9F480919D0283
:10E60000882359F081E0C43009F080E000E22EE375
:10E6100041ED5FE06D2F0E946CB7809195068823D5
:10E6200009F455C0C43009F052C0D4D91AC015300D
:10E6300009F04DC080919D02882359F081E0C530DA
:10E6400009F080E000E22EE346EC5FE06D2F0E94CF
:10E650006CB7809195068823D1F1C530C1F5F701DB
:10E66000199580918A06882391F154C0143011F0D5
:10E6700085E02EC080919D028823D1F081E0C430D6
:10E6800009F080E00EE32EE348EB5FE00EC01430AB
:10E6900079F780919D02882359F081E0C43009F018
:10E6A00080E00EE32EE34DEA5FE06D2F0E946CB731
:10E6B000809195068823E1F2C430D1F68DE690E58D
:10E6C0000E94CE5480918A06882391F223C086E06E
:10E6D000DF5F1F5FD43009F0E6CE8093E4081AC0F4
:10E6E00080919D02882359F081E0C13009F080E0DB
:10E6F0000EE32EE34CE050E16D2F0E946CB7809149
:10E700009506882309F44FCFC13009F04CCF8BE731
:10E7100090E743CFDF91CF911F910F91FF90EF9042
:10E7200008950F931F93CF93DF938C01EB0161E06A
:10E7300081E00E94EEA7C8010E94B6B72097B1F011
:10E740008AE30E94E5AFFE019F012C1B3D0B8191E6
:10E750008111FACF61E084E1821B0E94EEA7CE0115
:10E76000DF91CF911F910F910C94A1B7DF91CF91C1
:10E770001F910F9108950F931F93CF93DF938B01F8
:10E780000E94847DEB010E942E558F3F49F00E942C
:10E79000847D6C1B7D0B60177107A8F380E001C0BE
:10E7A00081E0DF91CF911F910F9108958F929F92F9
:10E7B000AF92BF92CF92DF92EF92FF920F931F938F
:10E7C000CF93DF93EC018B81811102C080E077C091
:10E7D00009891A892B893C890417150726073707E9
:10E7E000A8F36A017B01823029F4C886D986EA86BB
:10E7F000FB860DC0C114D104E104F10451F41C8264
:10E800001D821E821F82188619861A861B8681E049
:10E8100056C088849984AA84BB84E98DFA8D2585A5
:10E8200030E0275F3F4FB501A40141505109610914
:10E830007109022E04C076956795579547950A94FD
:10E84000D2F7D701C6010197A109B10904C0B69555
:10E85000A795979587952A95D2F784179507A607C8
:10E86000B70720F089288A288B2849F44D895E89CA
:10E870006F89788D4C835D836E837F8304C0841B96
:10E88000950BA60BB70B4C015D018E010C5F1F4F62
:10E8900081149104A104B10409F4A7CF4C815D81D6
:10E8A0006E817F819801898D9A8D0E94F93E91E059
:10E8B000891A9108A108B1088111EACF87CFDF91A9
:10E8C000CF911F910F91FF90EF90DF90CF90BF906D
:10E8D000AF909F908F9008950F931F93CF93DF93E6
:10E8E000FC012381222311F080E044C08B01EC0164
:10E8F000FB018789803139F18032B1F783E08B8366
:10E90000F801428D538D648D758D4D8B5E8B6F8BB1
:10E91000788F9E012F5E3F4FC8010E947A3F882367
:10E9200019F31A8F098F81E089831C821D821E8250
:10E930001F82188619861A861B861C861D861E86CF
:10E940001F86188A17C082E08B831D8A1E8A1F8A41
:10E95000188EFB01808D918DA0E0B0E025E0880F3E
:10E96000991FAA1FBB1F2A95D1F7898B9A8BAB8B56
:10E97000BC8BD7CFDF91CF911F910F9108950F934B
:10E980001F93CF93DF93EB01FC012381211102C080
:10E9900080E040C02250223028F48FE28883198220
:10E9A00081E038C08C01FC0164857585868597857A
:10E9B00040E00E94303E882359F3F8014089F0E29C
:10E9C0004F9FA00111249A012957364F232B01F3A1
:10E9D00020E030E090E06EE2F901E40FF51FE95726
:10E9E000F64F7081703271F02830310529F4DE0164
:10E9F000A90FB11D6C939F5FDE01A90FB11D70813E
:10EA00007C939F5F2F5F3F4F2B30310529F7C90F54
:10EA1000D11D1882DF91CF911F910F910895CF934F
:10EA2000DF93EC010E9442401B82DF91CF91089559
:10EA30003F924F925F926F927F928F929F92AF928E
:10EA4000BF92CF92DF92EF92FF920F931F93CF93DB
:10EA5000DF93CDB7DEB72C970FB6F894DEBF0FBEAD
:10EA6000CDBF5C01DC0159968D909C905A97F401C2
:10EA700081859285A385B4859C01AD012F5F3F4FB1
:10EA80004F4F5F4F29873A874B875C87D501149694
:10EA9000CD90DD90ED90FC901797C114D104E10466
:10EAA000F10439F0BFEFCB1ADB0AEB0AFB0A312C79
:10EAB00007C0F401C080D180E280F3803324339416
:10EAC000260137011D821E821F821886F40181856E
:10EAD0009285A385B4852D813E814F815885281765
:10EAE00039074A075B0708F064C089859A85AB85BA
:10EAF000BC858C159D05AE05BF0550F482E0C82E7F
:10EB0000D12CE12CF12C92E0492E512C612C712C4E
:10EB10009E012F5F3F4FB701A601C4010E94F93E3D
:10EB2000882309F446C089819A81AB81BC81892BF5
:10EB30008A2B8B2B41F0260137019FEF491A590A86
:10EB4000690A790A05C0C414D504E604F70491F0F3
:10EB50002D813E814F8158852F5F3F4F4F4F5F4F33
:10EB60002D833E834F8358873FEFC31AD30AE30AAE
:10EB7000F30AACCF0FEF1FEF2FEF3FE0B301A2017D
:10EB8000C4010E94683EF82E882399F0D50114969E
:10EB90004D915D916D917C911797411551056105DE
:10EBA000710549F093018201C4010E94683E811100
:10EBB00002C0F12C29C0D50114964D925D926D9240
:10EBC0007C921797332051F0D301C2010196A11D09
:10EBD000B11DF40180839183A283B383F5018589FC
:10EBE0009689A789B08D892B8A2B8B2B69F4D50147
:10EBF00055964D925D926D927C92589711968C919C
:10EC00001197806811968C938F2D2C960FB6F894DF
:10EC1000DEBF0FBECDBFDF91CF911F910F91FF904F
:10EC2000EF90DF90CF90BF90AF909F908F907F90AC
:10EC30006F905F904F903F90089561E0FC0180815C
:10EC4000E6C58EBD0DB407FEFDCF0895CF92DF92CD
:10EC5000EF92FF921F93CF93DF9300D01F92CDB717
:10EC6000DEB76C01162FFC019281892F806A869590
:10EC70008CBD90FD03C081E0963009F480E08DBD2D
:10EC800060E0F601808129833A834B835C83BFD5A2
:10EC90006CE271E0C6016FDD812F8064D2DF88E114
:10ECA000E82EF12C5C814B813A812981DA01C9017E
:10ECB0000E2C04C0B695A795979587950A94D2F720
:10ECC00029833A834B835C83BCDFF8E0EF1AF108B9
:10ECD00029813A814B815C8188EFE8168FEFF80635
:10ECE00029F7112321F0183021F08FEF03C085E9B7
:10ECF00001C087E8A6DF1C3011F40E942E5510E0F9
:10ED00000E942E55F601838387FF04C01F3F11F038
:10ED10001F5FF6CF0F900F900F900F90DF91CF9164
:10ED20001F91FF90EF90DF90CF9008950F931F9366
:10ED3000CF93DF93EC0189018C81833039F089E036
:10ED4000440F551F661F771F8A95D1F79A01AB01B3
:10ED500068E1CE017BDF882311F086E030C08EEFC2
:10ED60008EBD80E090E00DB407FEFDCFF801E80F06
:10ED7000F91F20812EBD0DB407FEFDCF21812EBDD0
:10ED80000296811522E0920771F70DB407FEFDCFC0
:10ED90008FEF57DF8FEF55DF0E942E558B838F71DA
:10EDA000853029F083E18983CE0147DF09C068E51A
:10EDB00072E0CE01E0DC182F811106C087E1898363
:10EDC000CE013BDF10E010C020E030E0A9016DE093
:10EDD000CE013CDF811104C00E942E55882311F022
:10EDE00086E1EDCFCE0129DF812FDF91CF911F91F9
:10EDF0000F910895EF92FF920F931F93CF93DF939C
:10EE0000EC0189018C81833039F0E9E0440F551F12
:10EE1000661F771FEA95D1F79A01AB0161E1CE0138
:10EE200015DF811157C070D67B010E942E558B8350
:10EE30008F3F41F469D66E197F096D327140A8F396
:10EE400081E13CC08E3F11F08FE038C08FEF8EBD66
:10EE5000D801C80181509E4FF8012FEF0DB407FE75
:10EE6000FDCF3EB531932EBDE817F907B9F70DB4C4
:10EE700007FEFDCF2EB5FC0120831E5FE12CF12C97
:10EE80008D91EF2DFF27E827EE0FFF1FEE59FF4E64
:10EE900085919491FE2CEE24E826F926A017B1075F
:10EEA00079F70E942E55082F10E0102F00270E949E
:10EEB0002E55082BE016F10639F080E28983CE0149
:10EEC000BCDE8FEFBEDE08C0CE01B7DE8FEFB9DE4D
:10EED00081E005C084E08983CE01AFDE80E0DF9170
:10EEE000CF911F910F91FF90EF9008952F923F9235
:10EEF0004F925F926F927F928F929F92AF92BF924A
:10EF0000CF92DF92EF92FF920F931F93CF93DF93F5
:10EF100000D01F92CDB7DEB79C838B834B015A0183
:10EF2000DC0113968C91811103C08FEF9FEFEAC033
:10EF3000EB81FC81818180FFF8CFAB81BC81519650
:10EF40000D911D912D913C91549718964D915D9185
:10EF50006D917C911B97C501A0E0B0E0680179013B
:10EF6000C41AD50AE60AF70AC816D906EA06FB0645
:10EF700018F45801A41AB50A75018B819C81049676
:10EF80009A838983612C92E0792EE114F10409F4CB
:10EF90008BC0AB81BC8118964D915D916D917C9138
:10EFA0001B976A01B1E0DB22EB81FC8123811A010E
:10EFB0002B0189E056944794379427948A95D1F78A
:10EFC000818D928D223061F4FC01828D938DA48D10
:10EFD000B58DBC01CD01620D731D841D951D4AC008
:10EFE000DC0114961C9111501221C114D10401F5B9
:10EFF00011111EC0452B462B472B59F4EB81FC8188
:10F0000085899689A789B08D84839583A683B783E4
:10F010000FC0AB81BC8114964D915D916D917C9137
:10F02000179729813A810E94F93E882309F47DCF00
:10F03000EB81FC81218D328D84819581A681B78100
:10F040000297A109B109F901058404C0880F991F2D
:10F05000AA1FBB1F0A94D2F746855785608971891C
:10F06000840F951FA61FB71FBC01CD01610F711D35
:10F07000811D911D93012C193D0987012E153F0516
:10F0800008F489010115F2E01F0771F52091870B43
:10F090003091880B4091890B50918A0B621773074E
:10F0A0008407950719F420C0C5012CC09401AB0159
:10F0B000BC018091900B9091910B9CDE882309F408
:10F0C00034CF800E911EEB81FC8180859185A285D5
:10F0D000B385800F911FA11DB11D80879187A287E5
:10F0E000B387E01AF10A51CF40E00E94303E8823F6
:10F0F00009F41BCFB6016957764FA801C4010E94DD
:10F100005EE8DFCF0F900F900F900F90DF91CF91BF
:10F110001F910F91FF90EF90DF90CF90BF90AF9035
:10F120009F908F907F906F905F904F903F902F9027
:10F1300008954F925F926F927F929F92AF92BF928B
:10F14000CF92DF92EF92FF920F931F93CF93DF93B3
:10F150001F92CDB7DEB78C017B016A01A22EDB01C5
:10F1600059968D919C915A97F801928F818F40E02A
:10F1700050E0BA01C7011ADB912CF7018085918517
:10F18000A285B3854189528963897489841795075B
:10F19000A607B70708F063C025E0B695A795979531
:10F1A00087952A95D1F7F82FFF70BF2ED7011396B8
:10F1B0008C91823008F469C041E050E0BE016F5F7D
:10F1C0007F4FC70193DE019719F4898190E002C057
:10F1D0008FEF9FEF019609F458C0F7018085918564
:10F1E000A285B3854F96A11DB11D80879187A28707
:10F1F000B387F0E2BF9EC0011124BC016957764F6E
:10F200006115710509F441C0DB012C91222319F02D
:10F21000253ED1F47CC191100EC04091870B5091D6
:10F22000880B6091890B70918A0BF8014487558790
:10F2300066877787B08AFC01E957F64F808188237B
:10F2400061F09924939499CF4BE050E0C6010E945D
:10F2500051E8892B09F091CF1AC0992493948A2DF3
:10F260008274823491F4992009F49CC0D80150969C
:10F27000BC9050971C966D917D918D919C911F979C
:10F2800041E00E94303E811180C080E043C1A7FC74
:10F29000FCCFF0E2BF9EA00111249A012957364FFE
:10F2A000D9011B968C91817121F08A2D827109F010
:10F2B00068C08091870B9091880BA091890BB091C9
:10F2C0008A0BF80184879587A687B787B08AFA01E9
:10F2D000E957F64F4489558960E070E0BA01552737
:10F2E0004427D80155964D935D936D937C93589721
:10F2F000828D938DA0E0B0E0482B592B6A2B7B2B9D
:10F30000D80155964D935D936D937C935897D90191
:10F310001B968C91887159F4848D958DA68DB78D2F
:10F32000F801818B928BA38BB48B81E010C080316C
:10F3300041F598012F5E3F4FD80159968D919C91D0
:10F340005A970E947A3F8823E1F084E0F801838392
:10F350008A2D8F70D80111968C931197F801148221
:10F3600015821682178218961D921D921D921C926C
:10F370001B97A4FEC0C0C8010E94A0A68111BBC0FB
:10F3800084CFD80113961C9280CFF8016089F0E2F7
:10F390006F9FB00111246957764F6115710509F00F
:10F3A0008AC073CFD70113968C911397823009F4DA
:10F3B0006CCF51968D919D910D90BC91A02D803E6A
:10F3C0009F4FAF41B10508F060CFC70131DB882303
:10F3D00009F45BCF0E94F03D882309F456CFD70192
:10F3E00059962D913C915A9714968D919D910D901F
:10F3F000BC91A02D0297A109B109F901058404C0AF
:10F40000880F991FAA1FBB1F0A94D2F746845784FE
:10F4100060887188480E591E6A1E7B1E81E08093A9
:10F420008F0B4092870B5092880B6092890B7092E1
:10F430008A0B80E092E0E7E8F9E0DF019C011D9291
:10F4400021503040E1F7BB24B394D7015996ED9198
:10F45000FC915A978481B81690F427E839E0B301FB
:10F46000A2014B0D511D611D711D8091900B90915A
:10F47000910B5CDC882309F408CFB394E6CF80E0DD
:10F4800092E0A0E0B0E0058404C0880F991FAA1F95
:10F49000BB1F0A94D2F7F7014189528963897489A5
:10F4A000840F951FA61FB71F818B928BA38BB48BE4
:10F4B00067E879E0B12C80E2DB011D928A95E9F7DB
:10F4C0008BE0F601DB0101900D928A95E1F781E274
:10F4D00098E2FB01918B808B20E038E0378726870C
:10F4E000938B828B918F808F378B268B0E94F03D80
:10F4F0008111CFCECACEA5FE08C0F801418952893C
:10F5000063897489C80152D905C081E003C0911094
:10F5100098CE83CE0F90DF91CF911F910F91FF90E6
:10F52000EF90DF90CF90BF90AF909F907F906F90C3
:10F530005F904F9008952F923F924F925F926F92FB
:10F540007F928F929F92AF92BF92CF92DF92EF9273
:10F55000FF920F931F93CF93DF93CDB7DEB7C554C0
:10F56000D1090FB6F894DEBF0FBECDBF3C015B01E1
:10F570008A01322E1C8E1F8E19821C82672B11F479
:10F5800010E0A7C0FC0183818111FACFFA018081CC
:10F590008F3261F4CA018C010196F80120812F326B
:10F5A000D1F3F50183818250823010F475010AC0D5
:10F5B000618D728DCE0101968FD9882309F3CE011A
:10F5C00001967C016E019CE1C90ED11C26014E0101
:10F5D000E7E38E0E911CFBE0F80D2596FFAF259713
:10F5E000CE01019624969FAF8EAF24972696CFAE7C
:10F5F00026972D2C35C080E2819325969FAD2597C7
:10F600009E13F9CFD80190E027E04A2F3B2F8D9130
:10F61000811128C08FA9803209F4B2CF842F932F93
:10F620008C01FC01208101962F32D1F3222309F4B1
:10F630004AC021E0A401B701C6017BDD882309F49B
:10F640009FCFEA14FB0411F0C701E9D9C414D50413
:10F6500099F126969FAD2697822D7601C92ED82E38
:10F66000F401C9CF8F32B1F28E3219F0E2E6F2E145
:10F670000AC02A3009F484CF98E02AE0C6CF319638
:10F68000381709F47DCF34913111F9CF291708F4D7
:10F6900077CF813208F474CF8F3709F471CF31E01E
:10F6A000390FF401E90FF11D9FE9980F9A3108F421
:10F6B00080528083932FA9CF23969FAD23972496C2
:10F6C0008FAD2497CACF232DA401B701C30131DD2B
:10F6D000182FCE0101960E945332CE014C960E9403
:10F6E0005332812FCB5BDF4F0FB6F894DEBF0FBED6
:10F6F000CDBFDF91CF911F910F91FF90EF90DF90E1
:10F70000CF90BF90AF909F908F907F906F905F90C1
:10F710004F903F902F9008953FB7F8948091F30851
:10F720009091F408A091F508B091F60826B5A89B31
:10F7300005C02F3F19F00196A11DB11D3FBFBA2F83
:10F74000A92F982F8827820F911DA11DB11DBC01E3
:10F75000CD0142E0660F771F881F991F4A95D1F7A8
:10F76000089590E0FC013197E231F10508F04EC0B8
:10F770008827EE58FF4F8F4F0C9450E58091800002
:10F780008F7703C0809180008F7D809380000895E3
:10F7900080918000877FF9CF84B58F7702C084B5D0
:10F7A0008F7D84BD08958091B0008F7703C08091D4
:10F7B000B0008F7D8093B0000895809190008F7786
:10F7C00007C0809190008F7D03C080919000877F5B
:10F7D0008093900008958091A0008F7707C080915A
:10F7E000A0008F7D03C08091A000877F8093A00040
:10F7F0000895809120018F7707C0809120018F7D2F
:10F8000003C080912001877F8093200108951F937A
:10F81000CF93DF93282F30E0F901EF5CF34F849111
:10F82000F901E551F44FD491F901EB55F44FC4912E
:10F83000CC23C1F0162F811194DFEC2FF0E0EE0FF6
:10F84000FF1FE457FD4EA591B4918FB7F8941111A5
:10F8500005C09C91ED2FE095E92302C0EC91ED2BC2
:10F86000EC938FBFDF91CF911F910895CF93DF93DA
:10F87000EC0160E08E81CBDF61E08E81C8DF60E06B
:10F880008E81C5DF8BE891E00197F1F7DF91CF9191
:10F890000895CF93DF9390E0FC01E551F44F24915C
:10F8A000FC01EB55F44F8491882361F190E0880FBF
:10F8B000991FFC01EE58FD4EC591D491FC01E4570F
:10F8C000FD4EA591B491611109C09FB7F89488814C
:10F8D000209582238883EC912E230BC0623061F443
:10F8E0009FB7F8943881822F809583238883EC9189
:10F8F0002E2B2C939FBF06C08FB7F894E8812E2B38
:10F9000028838FBFDF91CF9108951F93CF93DF930B
:10F91000182FEB0161E0BDDF209711F460E004C017
:10F92000CF3FD10531F461E0812FDF91CF911F915D
:10F930006ECFE12FF0E0EF5CF34FE4914E2F50E0FB
:10F94000FA013197E231F10508F09DC08827EC57A4
:10F95000FF4F8F4F0C9450E584B5806884BDC7BDC0
:10F9600097C084B5806284BDC8BD92C0809180007C
:10F97000806880938000D0938900C093880088C0FD
:10F9800080918000806280938000D0938B00C09330
:10F990008A007EC080918000886080938000D09330
:10F9A0008D00C0938C0074C08091B00080688093FB
:10F9B000B000C093B3006CC08091B00080628093AF
:10F9C000B000C093B40064C08091900080688093C0
:10F9D0009000D0939900C09398005AC080919000F5
:10F9E000806280939000D0939B00C0939A0050C097
:10F9F00080919000886080939000D0939D00C09388
:10FA00009C0046C08091A00080688093A0008091F7
:10FA1000A0008F7B8093A000D093A900C093A80082
:10FA200037C08091A00080628093A000D093AB008B
:10FA3000C093AA002DC08091A00088608093A00090
:10FA4000D093AD00C093AC0023C0809120018068AA
:10FA500080932001D0932901C093280119C080917F
:10FA60002001806280932001D0932B01C0932A0152
:10FA70000FC080912001886080932001D0932D01D8
:10FA8000C0932C0105C0C038D1050CF04CCF46CF37
:10FA9000DF91CF911F9108958F929F92AF92BF9265
:10FAA000CF92DF92EF92FF926B017C0135DE4B012A
:10FAB0005C01C114D104E104F104E9F02DDEDC01A4
:10FAC000CB0188199909AA09BB09883E9340A10571
:10FAD000B10578F321E0C21AD108E108F10888EEF7
:10FAE000880E83E0981EA11CB11CC114D104E1044E
:10FAF000F10421F7DECFFF90EF90DF90CF90BF9021
:10FB0000AF909F908F9008952FB7F8946091EF0871
:10FB10007091F0088091F1089091F2082FBF08953C
:10FB20001F920F920FB60F9211242F933F938F9332
:10FB30009F93AF93BF938091EF089091F008A091AD
:10FB4000F108B091F2083091EE0823E0230F2D3731
:10FB500020F40196A11DB11D05C026E8230F0296D1
:10FB6000A11DB11D2093EE088093EF089093F0083B
:10FB7000A093F108B093F2088091F3089091F408F3
:10FB8000A091F508B091F6080196A11DB11D8093D2
:10FB9000F3089093F408A093F508B093F608BF918A
:10FBA000AF919F918F913F912F910F900FBE0F902A
:10FBB0001F901895CF92DF92EF92FF920F931F93B1
:10FBC000CF93DF937C016C0187E0C80ED11CC0E0AD
:10FBD000D0E0062F10E0B8010C2E02C07595679595
:10FBE0000A94E2F76170F60181916F0110DE2196AF
:10FBF000C430D10581F7C701DF91CF911F910F91DB
:10FC0000FF90EF90DF90CF9031CECF92DF92EF92C6
:10FC1000FF920F931F93CF93DF93EC01F62E642F87
:10FC20008C81F5DD8D818F3F11F060E0F0DD8F85F7
:10FC30000F2D10E084FF23C06E0187E0C80ED11C99
:10FC4000E12CF12CB8010E2C02C0759567950A9431
:10FC5000E2F76170F60181916F01D9DDFFEFEF1AD4
:10FC6000FF0A88E0E816F10469F7CE01DF91CF9131
:10FC70001F910F91FF90EF90DF90CF90F7CDB801DB
:10FC800084E0759567958A95E1F7CE0193DF6F2D36
:10FC9000CE01DF91CF911F910F91FF90EF90DF90F8
:10FCA000CF9088CF41E0B1DF81E090E0089540E05F
:10FCB000ACCF61E0FCDF8BE39FE10197F1F70895A2
:10FCC0008F929F92AF92BF92CF92DF92EF92FF926C
:10FCD000CF9320E030E048EC52E4FC016081718178
:10FCE000828193810E94BFED6B017C0120E030E0B6
:10FCF000A9010E94A1E718161CF4C701B60103C0B0
:10FD0000C701B60190580E94B6E66B017C0197FFCF
:10FD10000AC0F094E094D094C094C11CD11CE11CA2
:10FD2000F11C8DE201C08BE28093CD0EC701B601BC
:10FD300020EA36E841E050E00E9457F18AE0882E40
:10FD4000912CA12CB12CCA01B901A50194010E94EA
:10FD500057F1605D6093CE0EC701B60120E137E236
:10FD600040E050E00E9457F1CA01B901A501940199
:10FD70000E9457F1605D6093CF0EC701B60128EE77
:10FD800033E040E050E00E9457F1CA01B901A501FB
:10FD900094010E9457F1605D6093D00EC701B601D7
:10FDA00024E630E040E050E00E9457F1CA01B9017A
:10FDB000A50194010E9457F1605D6093D10E8EE21F
:10FDC0008093D20EC701B601A50194010E9457F19C
:10FDD000C62FCA01B901A50194010E9457F1605DC7
:10FDE0006093D30EC05DC093D40E1092D50E8DECEF
:10FDF0009EE0CF91FF90EF90DF90CF90BF90AF90BB
:10FE00009F908F9008958F929F92AF92BF92CF92C2
:10FE1000DF92EF92FF92CF9320E030E048EC52E483
:10FE2000FC0160817181828193810E94BFED0E94FB
:10FE3000B6E66B017C0197FF0AC0F094E094D09481
:10FE4000C094C11CD11CE11CF11C8DE201C08BE2ED
:10FE50008093CD0EC701B60120E137E240E050E0CB
:10FE60000E9457F18AE0882E912CA12CB12CCA0156
:10FE7000B901A50194010E9457F1605D6093CE0E17
:10FE8000C701B60128EE33E040E050E00E9457F190
:10FE9000CA01B901A50194010E9457F1605D609308
:10FEA000CF0EC701B60124E630E040E050E00E94EA
:10FEB00057F1CA01B901A50194010E9457F1605D93
:10FEC0006093D00E8EE28093D10EC701B601A501DA
:10FED00094010E9457F1C62FCA01B901A5019401EE
:10FEE0000E9457F1605D6093D20EC05DC093D30E47
:10FEF0001092D40E8DEC9EE0CF91FF90EF90DF90AA
:10FF0000CF90BF90AF909F908F9008958F929F92C7
:10FF1000AF92BF92CF92DF92EF92FF92FC01C0802E
:10FF2000D180E280F38020E030E0A901C701B60172
:10FF30000E94A1E718161CF4C701B60103C0C7014F
:10FF4000B60190580E94B6E66B017C016031F7E281
:10FF50007F078105910584F020E137E240E050E021
:10FF60000E9457F1CA01B9012AE030E040E050E0B8
:10FF70000E9457F1605D01C060E26093CD0E88EE93
:10FF8000C81683E0D806E104F10494F0C701B60175
:10FF900028EE33E040E050E00E9457F1CA01B90179
:10FFA0002AE030E040E050E00E9457F1605D01C07F
:10FFB00060E26093CE0EE4E6CE16D104E104F104D3
:10FFC00094F0C701B60124E630E040E050E00E9422
:10FFD00057F1CA01B9012AE030E040E050E00E9448
:10FFE00057F1605D01C060E26093CF0EFAE0CF167A
:10FFF000D104E104F1049CF08AE0882E912CA12C1C
:020000021000EC
:10000000B12CC701B601A50194010E9457F1CA01A4
:10001000B901A50194010E9457F1605D01C060E241
:100020006093D00EC701B6012AE030E040E050E016
:100030000E9457F1605D6093D10E1092D20E8DEC4C
:100040009EE0FF90EF90DF90CF90BF90AF909F9099
:100050008F90089520E030E040E251E4FC0160819F
:100060007181828193810E94BFED0E94B6E69B015F
:1000700077FF06C022273327261B370B8DE201C0EE
:100080008BE28093CD0EC90168EE73E00E943DE5DE
:10009000CB01EAE0F0E0BF010E943DE5805D809386
:1000A000CE0EC90164E670E00E943DE5CB01BF01C0
:1000B0000E943DE5805D8093CF0EC901BF010E9483
:1000C0003DE5282FCB01BF010E943DE5805D809377
:1000D000D00E8EE28093D10E205D2093D20E10922E
:1000E000D30E8DEC9EE008958F929F92AF92BF92B7
:1000F000CF92DF92EF92FF92CF9320E030E048EC76
:1001000052E4FC0160817181828193810E94BFED84
:100110000E94B6E66B017C0197FD10C020E137E23A
:1001200040E050E00E9457F1CA01B9012AE030E0F6
:1001300040E050E00E9457F1605D09C0F094E09407
:10014000D094C094C11CD11CE11CF11C6DE26093E1
:10015000CD0EC701B60128EE33E040E050E00E942A
:1001600057F18AE0882E912CA12CB12CCA01B9013B
:10017000A50194010E9457F1605D6093CE0EC70106
:10018000B60124E630E040E050E00E9457F1CA0199
:10019000B901A50194010E9457F1605D6093CF0EF3
:1001A0008EE28093D00EC701B601A50194010E9492
:1001B00057F1C62FCA01B901A50194010E9457F158
:1001C000605D6093D10EC05DC093D20E1092D30ECD
:1001D0008DEC9EE0CF91FF90EF90DF90CF90BF909D
:1001E000AF909F908F900895FC01408151819A01BA
:1001F00057FF04C022273327241B350B483E83E0DA
:100200005807ACF0C90168EE73E00E943DE5CB01F0
:10021000EAE0F0E0BF010E943DE5805D8093CD0EF5
:10022000C90164E670E00E943DE5CB0112C02436AE
:100230003105B4F057FD02C080E201C08DE2809329
:10024000CD0EC90164E670E00E943DE5CB01EAE015
:10025000F0E0BF010E943DE5805D8093CE0E11C0AD
:1002600080E28093CD0E2A303105ACF080819181FF
:1002700097FD02C080E201C08DE28093CE0EEAE0DD
:10028000F0E0C901BF010E943DE5CB01BF010E9422
:100290003DE5805D09C08093CE0E8081918197FD00
:1002A00002C080E201C08DE28093CF0EC9016AE0F6
:1002B00070E00E943DE5805D8093D00E1092D10EDB
:1002C0008DEC9EE00895FC011092D00E808191810A
:1002D0002AE030E0B9010E943DE5805D8093CF0EB9
:1002E000808191818A309105ECF0B9010E943DE551
:1002F000CB01B9010E943DE5805D8093CE0E8081E7
:100300009181843691058CF064E670E00E943DE5B1
:10031000CB01B9010E943DE5805D8093CD0E8DEC4F
:100320009EE008958FEC9EE008958EEC9EE0089587
:10033000FC012081318137FD0FC0243631058CF05E
:10034000C90164E670E00E943DE5CB016AE070E01F
:100350000E943DE5805D06C03195219531098DE211
:1003600001C080E28093CD0E2A30310564F0EAE0CE
:10037000F0E0C901BF010E943DE5CB01BF010E9431
:100380003DE5805D01C080E28093CE0EC9016AE048
:1003900070E00E943DE5805D8093CF0E1092D00EFC
:1003A0008DEC9EE008950F931F93AEDB0091E9085A
:1003B0001091EA082091EB083091EC08DC01CB01A8
:1003C000801B910BA20BB30BB7FD0CC086B186FB53
:1003D000992790F981E08927349B8260329B846061
:1003E0008093E8088091E80881709091E80891FD79
:1003F00082609091ED08891721F18130A9F028F0F1
:10040000823041F0833059F01CC0913089F0923035
:1004100099F017C0992361F0933071F012C09130B8
:1004200059F0923071F404C0992331F0933049F4BB
:100430009091E7089F5F03C09091E70891509093D7
:10044000E7088093ED081F910F9108959C0180911A
:10045000E608681778F0962FB9019093E6084CE308
:1004600050E088E592E00E9402ED0E94C7A583E07B
:1004700080939D0208952091E60821110CC0BC01D3
:100480004CE350E088E592E00E94AEE80E94C7A5E8
:1004900083E080939D0208952F923F924F925F9246
:1004A0006F927F928F929F92AF92BF92CF92DF9284
:1004B000EF92FF920F931F93CF93DF9310929406C6
:1004C0008091BB0E9091BC0EA091BD0EB091BE0E5E
:1004D00081309048A105B10540F01092BB0E1092FA
:1004E000BC0E1092BD0E1092BE0E6091BB0E7091AC
:1004F000BC0E8091BD0E9091BE0E25E030E040E034
:1005000050E00E9435F1C22F80914D091816F4F485
:10051000022E000C330B482F082E000C550B4150B7
:1005200051092417350794F0CFEFC80F25E0C29F7B
:10053000C0011124092E000CAA0BBB0B8093BB0E2B
:100540009093BC0EA093BD0EB093BE0E10928A067F
:1005500080918906C81714F4C09389068091890692
:10056000082E000C990B03962C2F0C2E000C330B2D
:100570008217930724F48DEF8C0F809389061091D6
:100580008906D0E088E4282E82E0382E9CED892E62
:1005900095E0992EA12CB12C26ED422E26E0522E6C
:1005A000612C712C31E0E32E3EE4F32E43EEC42E99
:1005B00044E5D42E111117C080919D02882351F07B
:1005C00081E0C11180E003E023E045E354E16D2FB9
:1005D0000E946CB780919506882371F1C1112CC0DF
:1005E0000E94667025C0113039F580919D028823E4
:1005F00091F080914B09811103C024E234E102C0E3
:1006000028E234E181E0C13009F080E04CE254E1BD
:100610006D2F0E943ADA80919506882369F0C130E7
:1006200059F480914B098C2780934B090E94E35425
:1006300080918A0681117FC080914B09882309F43B
:1006400072C0123011F083E06FC080919D02882348
:1006500071F088E492E00E94F0AF9C0181E0C2302A
:1006600009F080E04AE154E16D2F0E94B3E48091EB
:100670009506882341F3C23031F781E080939406D8
:100680001092900610929106109292061092930684
:100690000E94106D83E080939D0280E194E190932D
:1006A000CA0E8093C90E3092C80E2092C70E809257
:1006B000C30E9092C40EA092C50EB092C60E409288
:1006C000BF0E5092C00E6092C10E7092C20E20E01A
:1006D00030E04AE754E46091480270914902809109
:1006E0004A0290914B020E94BFED20E030E84BEBB4
:1006F00054E40E9458E50E94BCE66093BB0E7093E0
:10070000BC0E8093BD0E9093BE0EF0929F02E092BD
:100710009E02D092CC0EC092CB0E80918A06882386
:1007200009F491CF08C082E0DF5F1F5FD43009F089
:1007300041CF80934D09DF91CF911F910F91FF9091
:10074000EF90DF90CF90BF90AF909F908F907F9071
:100750006F905F904F903F902F900895BF92CF92EF
:10076000DF92EF92FF920F931F93CF93DF9300D00E
:100770001F92CDB7DEB7109294068091BB0E909178
:10078000BC0EA091BD0EB091BE0E81309048A10567
:10079000B10540F01092BB0E1092BC0E1092BD0E2F
:1007A0001092BE0E6091BB0E7091BC0E8091BD0E7A
:1007B0009091BE0E25E030E040E050E00E9435F11F
:1007C000D22E80914C091816FCF4022E000C330B2B
:1007D000482F082E000C550B41505109241735079E
:1007E0009CF0DD24DA94D80E25E0D29EC0011124BD
:1007F000092E000CAA0BBB0B8093BB0E9093BC0E72
:10080000A093BD0EB093BE0E10928A068091890609
:10081000D81614F4D092890680918906082E000C0F
:10082000990B03962D2D0D2C000C330B821793077B
:1008300024F48DEF8D0D80938906B0908906C12C2C
:10084000B11018C080919D02882351F081E0D11031
:1008500080E003E023E048E054E16C2D0E946CB797
:1008600080919506882309F416C4D11014C40E94FF
:1008700066700DC481E0B81227C080919D02882364
:1008800061F084E492E030DC9C0181E0D81280E0E9
:100890004FEF53E16C2D0E94B3E4809195068823BD
:1008A00009F4F9C391E0D912F6C3E12CF12C00EA66
:1008B00011E420E030E040E252EC64E472E086EFC4
:1008C00093E10E94C3D8E3C322E0B21222C0809118
:1008D0009D02882369F087E499E018DB9C0181E0A0
:1008E00092E0D91280E040EF53E16C2D0E94B3E416
:1008F00080919506882309F4CEC322E0D212CBC39F
:1009000020E030E040E251E467E479E08AEE93E1F0
:1009100034C383E0B81233C080919D028823C9F0AC
:1009200060913709709138098091390990913A099D
:100930000E94B6E67A836983CE010196F9DC9C01B8
:1009400081E093E0D91280E042EE53E16C2D0E94E9
:10095000B3E480919506882309F49DC323E0D21265
:100960009AC3E12C10E8F12E07E714E420E030E010
:1009700040E85FE367E379E08AED93E1E3C184E077
:10098000B81233C080919D028823C9F060913B0961
:1009900070913C0980913D0990913E090E94B6E614
:1009A0007A836983CE010196C3DC9C0181E094E0E7
:1009B000D91280E042ED53E16C2D0E94B3E48091A6
:1009C0009506882309F467C324E0D21264C3E12C9E
:1009D00010E8F12E07E714E420E030E040E85FE3A0
:1009E0006BE379E08AEC93E1ADC185E0B81233C0E6
:1009F00080919D028823C9F060913F097091400960
:100A000080914109909142090E94B6E67A836983F8
:100A1000CE0101968DDC9C0181E095E0D91280E049
:100A200042EC53E16C2D0E94B3E48091950688233B
:100A300009F431C325E0D2122EC3E12C10E8F12EC7
:100A400007E714E420E030E040E85FE36FE379E09B
:100A50008AEB93E177C186E0B81233C080919D02A2
:100A60008823C9F060914309709144098091450938
:100A7000909146090E94B6E67A836983CE01019679
:100A800057DC9C0181E096E0D91280E042EB53E113
:100A90006C2D0E94B3E480919506882309F4FBC273
:100AA00026E0D212F8C2E12C10E8F12E07E714E498
:100AB00020E030E040E85FE363E479E08AEA93E134
:100AC00041C187E0B81233C080919D028823C9F0EC
:100AD00060912709709128098091290990912A092C
:100AE0000E94B6E67A836983CE01019621DC9C01DF
:100AF00081E097E0D91280E043EA53E16C2D0E9437
:100B0000B3E480919506882309F4C5C227E0D21288
:100B1000C2C2E12C10ECF12E09E714E420E030E031
:100B200040E85FE367E279E08CE993E10BC188E09C
:100B3000B81233C080919D028823C9F060912B09BF
:100B400070912C0980912D0990912E090E94B6E692
:100B50007A836983CE010196EBDB9C0181E098E00A
:100B6000D91280E045E953E16C2D0E94B3E48091F5
:100B70009506882309F48FC228E0D2128CC2E12C9A
:100B800010ECF12E09E714E420E030E040E85FE3E8
:100B90006BE279E08EE893E1D5C089E0B81233C00A
:100BA00080919D028823C9F060912F0970913009CE
:100BB00080913109909132090E94B6E67A83698367
:100BC000CE010196B5DB9C0181E099E0D91280E06D
:100BD00047E853E16C2D0E94B3E480919506882389
:100BE00009F459C229E0D21256C2E12C10ECF12EC0
:100BF00009E714E420E030E040E85FE36FE279E0E9
:100C000080E893E19FC08AE0B81233C080919D02D2
:100C10008823C9F0609133097091340980913509B6
:100C2000909136090E94B6E67A836983CE010196D7
:100C30007FDB9C0181E09AE0D91280E049E753E133
:100C40006C2D0E94B3E480919506882309F423C299
:100C50002AE0D21220C2E12C10ECF12E09E714E4B4
:100C600020E030E040E85FE363E379E082E793E18E
:100C700069C08BE0B81232C080919D028823C9F010
:100C8000609123097091240980912509909126098A
:100C90000E94B6E67A836983CE01019649DB9C0106
:100CA00081E09BE0D91280E04DE653E16C2D0E947B
:100CB000B3E480919506882309F4EDC12BE0D212AC
:100CC000EAC1E12C10ECF12E09E714E420E030E059
:100CD000A90163E279E088E693E134C08CE0B812C0
:100CE00034C080919D028823C9F060911F097091E2
:100CF000200980912109909122090E94B6E67A8309
:100D00006983CE01019614DB9C0181E09CE0D9123D
:100D100080E04EE553E16C2D0E94B3E4809195068E
:100D2000882309F4B8C12CE0D212B5C1E12C10EC33
:100D3000F12E09E714E420E030E0A9016FE179E049
:100D400084E593E10E944CD9A2C18DE0B81230C075
:100D500080919D028823D9F060910F09709110094C
:100D600080911109909112090E945EED69837A8346
:100D70008B839C83CE010196C9D89C0181E09DE0C4
:100D8000D91280E04DE453E16C2D0E94B3E48091D0
:100D90009506882309F47FC12DE0D2127CC124E698
:100DA00030E040E050E06FE079E086E493E198C005
:100DB0008EE0B81230C080919D028823D9F06091F6
:100DC00013097091140980911509909116090E94D8
:100DD0005EED69837A838B839C83CE01019696D8DE
:100DE0009C0181E09EE0D91280E04FE353E16C2D3D
:100DF0000E94B3E480919506882309F44CC12EE04B
:100E0000D21249C124E630E040E050E063E179E0ED
:100E100088E393E165C08FE0B81230C080919D02F5
:100E20008823D9F0609117097091180980911909E8
:100E300090911A090E945EED69837A838B839C836B
:100E4000CE01019663D89C0181E09FE0D91280E039
:100E500041E353E16C2D0E94B3E480919506882311
:100E600009F419C12FE0D21216C12AE030E040E0A7
:100E700050E067E179E08AE293E132C080E1B812A4
:100E800032C080919D028823D9F060911B09709136
:100E90001C0980911D0990911E090E945EED6983D5
:100EA0007A838B839C83CE01019630D89C0181E0AC
:100EB00090E1D91280E043E253E16C2D0E94B3E44B
:100EC00080919506882309F4E6C020E1D212E3C0A0
:100ED00024E630E040E050E06BE179E08CE193E122
:100EE0000E9437E4D4C081E1B81222C080919D02F3
:100EF000882369F08BE099E009D89C0181E091E1B9
:100F0000D91280E042E153E16C2D0E94B3E480915C
:100F10009506882309F4BFC021E1D212BCC020E0AD
:100F200030E048EC52E46BE079E088E093E125C0E2
:100F300082E1B81225C080919D02882371F087E07C
:100F400099E00E94867F9C0181E092E1D91280E0C5
:100F50004FEF52E16C2D0E94B3E4809195068823F7
:100F600009F499C022E1D21296C020E030E048ECAA
:100F700052E467E079E086EF92E10E9471E387C076
:100F800083E1B8121FC080919D02882371F087EF22
:100F900098E00E94607E9C0181E093E1D91280E09C
:100FA0004CEE52E16C2D0E94B3E4809195068823AB
:100FB00009F471C023E1D2126EC067EF78E082EECF
:100FC00092E163C084E1B8121FC080919D02882322
:100FD00071F08BEF98E00E94607E9C0181E094E1CB
:100FE000D91280E048ED52E16C2D0E94B3E480916B
:100FF0009506882309F44FC024E1D2124CC06BEF50
:1010000078E08EEC92E141C085E1B8121EC080917B
:101010009D02882371F08FEF98E00E94607E9C0112
:1010200081E095E1D91280E044EC52E16C2D0E9400
:10103000B3E480919506882371F125E1D2122BC08B
:101040006FEF78E08AEB92E120C086E1B81223C00E
:1010500080919D02882371F083E099E00E94607E78
:101060009C0181E096E1D91280E040EB52E16C2DC9
:101070000E94B3E480919506882369F026E1D2129C
:101080000AC063E079E086EA92E10E94E3E380919E
:101090008A06811108C0C394B39484E0C812D0CBEF
:1010A00087E180934C090F900F900F900F90DF9184
:1010B000CF911F910F91FF90EF90DF90CF90BF9055
:1010C000089514C07DC081E00C94B76B80E00C944F
:1010D000B76B9091D40B8091D50B981731F080911C
:1010E000D50B8F5F8F708093D50B08958F929F9251
:1010F000AF92BF92CF92DF92EF92FF920F931F9326
:10110000CF93DF9300D01F92CDB7DEB78FE0882E4C
:1011100089E0982E97EFA92E98E0B92E00E519E006
:10112000C12CD12C7601C394F4016191719181910C
:1011300091914F01F50121913191419151915F01BF
:1011400029833A834B835C830E945EED29813A8137
:101150004B815C810E94BFED0E94BCE6F801619367
:101160007193819391938F01C616D706E806F9060D
:1011700010F46B017C01FFE18F16F9E09F06A1F6E8
:101180006FEF7FEFCB01A70196010E9435F120930D
:1011900065093093660940936709509368090F9079
:1011A0000F900F900F90DF91CF911F910F91FF90B3
:1011B000EF90DF90CF90BF90AF909F908F90089569
:1011C0000F931F93CF93DF93C7EFD8E006ED16E0A0
:1011D000299139914991599160E070E080E89FE34D
:1011E0000E9445E6F80161937193819391938F0179
:1011F000F9E0C730DF0761F70E944BAADF91CF917A
:101200001F910F9173CF2F923F924F925F926F92E7
:101210007F928F929F92AF92BF92CF92DF92EF9286
:10122000FF920F931F93CF93DF9300D01F92CDB700
:10123000DEB77B016A011901A7EFB8E02D913D915E
:101240004D915C91FC0160817181828193810E944A
:10125000BFED0E94ACE72B013C0104EC1BE0D80180
:101260006D937D938D939C9313972091FB08309100
:10127000FC084091FD085091FE08F70160817181E2
:10128000828193810E94BFED0E94ACE74B015C011B
:10129000D80114966D937D938D939C93179720910D
:1012A000FF08309100094091010950910209F601AF
:1012B00060817181828193810E94BFED0E94ACE7C1
:1012C0006B017C01D80118966D937D938D939C934F
:1012D0001B97209103093091040940910509509111
:1012E0000609F10160817181828193810E94BFEDC5
:1012F0000E94ACE7D8011C966D937D938D939C93CF
:101300001F9769837A838B839C830E9479B02FB760
:10131000F894E4EDF3E14082518262827382848228
:101320009582A682B782C086D186E286F3866981DD
:101330007A818B819C8164877587868797872FBF89
:101340001092B00B1092B10B1092B20B1092B30B23
:1013500080E1E4EBFBE0DF011D928A95E9F70F9055
:101360000F900F900F90DF91CF911F910F91FF90F1
:10137000EF90DF90CF90BF90AF909F908F907F9035
:101380006F905F904F903F902F9008952F923F92D3
:101390004F925F926F927F928F929F92AF92BF9285
:1013A000CF92DF92EF92FF920F931F93CF93DF9331
:1013B000CDB7DEB7C057D1090FB6F894DEBF0FBE68
:1013C000CDBF3B014A015901EBA6F9AE0EAF219604
:1013D0001FAF21973C2C2091F7083091F8084091DD
:1013E000F9085091FA08DC016D917D918D919C91E5
:1013F0000E94BFED0E94ACE7A9966CAF7DAF8EAFA7
:101400009FAFA9972091FB083091FC084091FD08FF
:101410005091FE08F30160817181828193810E9465
:10142000BFED0E94ACE7AD966CAF7DAF8EAF9FAFC6
:10143000AD972091FF08309100094091010950912A
:101440000209D4016D917D918D919C910E94BFED17
:101450000E94ACE7E1966CAF7DAF8EAF9FAFE19796
:101460002091030930910409409105095091060922
:10147000F50160817181828193810E94BFED0E949C
:10148000ACE764966CAF7DAF8EAF9FAF64978091F1
:10149000C40B9091C50BA091C60BB091C70BA99638
:1014A000CCACDDACEEACFFACA997C81AD90AEA0AFD
:1014B000FB0A8091C80B9091C90BA091CA0BB09107
:1014C000CB0BAD960CAD1DAD2EAD3FADAD97081B52
:1014D000190B2A0B3B0B09AB1AAB2BAB3CAB809126
:1014E000CC0B9091CD0BA091CE0BB091CF0BE19690
:1014F0002CAD3DAD4EAD5FADE197281B390B4A0BCE
:101500005B0B2DAB3EAB4FAB58AF8091E41383FF29
:101510000EC064968CAD9DADAEADBFAD64978093AB
:10152000D00B9093D10BA093D20BB093D30B80919F
:10153000D00B9091D10BA091D20BB091D30B6496AC
:101540008CAC9DACAEACBFAC6497881A990AAA0A61
:10155000BB0A09F487C080914F0981113DC02091D9
:101560004C0230914D0240914E0250914F026091D9
:101570009E0870919F088091A0089091A1080E94F8
:101580005AED87FF29C064960CAD1DAD2EAD3FAD61
:1015900064970093D00B1093D10B2093D20B309310
:1015A000D30BE1E4F7E184918F010F5F1F4F882394
:1015B00021F00E94A832F801F6CFECE5F4E1849125
:1015C0008F010F5F1F4F882321F00E94A832F8017E
:1015D000F6CF812C912C540124013501B7FE07C0B0
:1015E000442455243201481859086A087B08609140
:1015F00003097091040980910509909106090E94E0
:10160000B6E69B01AC01A8ECB0E00E9473F1641552
:101610007505860597054CF564962CAD3DAD4EAD30
:101620005FAD64972093D00B3093D10B4093D20BD6
:101630005093D30BE1E4F7E184918F010F5F1F4FCB
:10164000882321F00E94A832F801F6CFEDE3F4E1FF
:1016500084918F010F5F1F4F882321F00E94A832D1
:10166000F801F6CF812C912C5401D701C6018827AF
:10167000B7FD83959927AA27BB27182F29A93AA92F
:101680004BA95CA957FD12608DA99EA9AFA9B8AD61
:10169000B7FD1460B7FC1860A32DB0E02696BFAF6D
:1016A000AEAF2697C501B4010E9460ED2696EEAD5F
:1016B000FFAD2697EE0FFF1FEE0FFF1FE05BFD4F04
:1016C00020813181428153810E94BFED4B015C0139
:1016D0002696EEADFFAD2697EE0FFF1FEE5BFD4F9A
:1016E00060817181072E000C880B990B0E9460EDC0
:1016F0009B01AC01C501B4010E94BFED2AE037EDAA
:1017000043E25CE30E94BFED2B013C0120E030E0AE
:10171000A9010E94A1E718164CF420E030E040E057
:101720005FE3C301B2010E9459E508C0A301920121
:1017300060E070E080E09FE30E9458E50E94B6E61A
:101740006AAF7BAF8CAF9DAF8091D40B8F5F8F70F2
:10175000A5968FAFA597A82E880FBB088091D50BB3
:1017600090E08A159B0519F40E949B56F7CFE091F3
:10177000D40B2E2F30E038AB2FA739E4E39FF001D4
:101780001124E55EF04F108212A3D701C601F7FEC7
:1017900007C088279927DC018C199D09AE09BF096C
:1017A00082839383A483B58389E40FA518A9809FBE
:1017B000F001819FF00D1124E55EF04F89A99AA9EF
:1017C000ABA9BCA9B7FF07C0B095A095909581952E
:1017D0009F4FAF4FBF4F86839783A087B18789E420
:1017E0000FA518A9809FF001819FF00D1124E55EDF
:1017F000F04F8DA99EA9AFA9B8ADB7FF07C0B095AE
:10180000A095909581959F4FAF4FBF4F828793874B
:10181000A487B58789E40FA518A9809FF001819F4F
:10182000F00D1124E55EF04F2AAD3BAD4CAD5DAD42
:1018300026873787408B518B428153816481758124
:1018400086819781A085B18584179507A607B7077C
:1018500014F4DB01CA0129E40FA518A9209FF001A7
:10186000219FF00D1124E55EF04F0285138524853C
:10187000358580179107A207B30714F4D901C80171
:101880000AAD1BAD2CAD3DAD80179107A207B30784
:1018900014F4D901C80129E40FA518A9209FF0016B
:1018A000219FF00D1124E55EF04F828B938BA48B6A
:1018B000B58B0697A105B10510F40C94C695DF0110
:1018C000A95BBF4F80917C0890917D088D939C937C
:1018D0003182452B462B472B09F05F9889E40FA5F1
:1018E00018A9809FF001819FF00D1124E55EF04F53
:1018F00086819781A085B185892B8A2B8B2B09F056
:101900008A9889E40FA518A9809FF001819FF00DA6
:101910001124E55EF04F82859385A485B585892BDA
:101920008A2B8B2B41F09FB7F894809108018E7F12
:10193000809308019FBF2AAD3BAD4CAD5DAD232B1D
:10194000242B252B71F080916409882319F0815094
:101950008093640931100EC0129880E2809364096C
:1019600009C020901F093090200900912109109191
:10197000220908C0209023093090240900912509EC
:10198000109126099101A8016BA579AD8EAD219624
:101990009FAD21970E945AED87FD02C00C94BE9521
:1019A000C701B6010E9460ED2091D6063091D7069E
:1019B0004091D8065091D9060E94BFED6BA77CA735
:1019C0008DA79EA7698B7A8B8B8B9C8B69A97AA933
:1019D0008BA99CA90E9460ED2091DA063091DB066C
:1019E0004091DC065091DD060E94BFED4B015C0189
:1019F0006D8B7E8B8F8B988F6DA97EA98FA998ADEB
:101A00000E9460ED2091DE063091DF064091E006F5
:101A10005091E1060E94BFED6B017C01698F7A8FC6
:101A20008B8F9C8F2091E2063091E3064091E40673
:101A30005091E506C301B2010E94BFED6D8F7E8F0C
:101A40008F8F98A329E44FA558A9249FF001259FC3
:101A5000F00D1124E55EF04F428053806480758064
:101A600056E04516510461047104D4F4268137818F
:101A70004085518526303105410551058CF422857C
:101A8000338544855585263031054105510544F49B
:101A9000DC01CB01BF7787A790ABA1ABB2AB38C05D
:101AA0002BA53CA54DA55EA5CA01B9010E94BFEDBD
:101AB00069AB7AAB8BAB9CABA5019401C501B401BA
:101AC0000E94BFED9B01AC0169A97AA98BA99CA9D1
:101AD0000E9459E54B015C01A7019601C701B601BF
:101AE0000E94BFED9B01AC01C501B4010E9459E504
:101AF0000E94EAE729E4AFA5B8A92A9FF0012B9F2D
:101B0000F00D1124E55EF04F67A770AB81AB92AB8F
:101B100029E4EFA5F8A92E9FC0012F9F900D112455
:101B20009C01255E304F7901D9019F968D919D9141
:101B30000D90BC91A02DA4968CAF9DAFAEAFBFAF62
:101B4000A4979C01AD0160E070E080E89FE30E94F3
:101B500045E624966CAF7DAF8EAF9FAF24979B0177
:101B6000AC01B101C8010E94BFED4B015C01809145
:101B7000D40B9091D50B891B8F706D968FAF6D979D
:101B8000A5019401A4966CAD7DAD8EAD9FADA497DB
:101B90000E94BFED2A966CAF7DAF8EAF9FAF2A97A4
:101BA000F70163A374A385A396A3028913892489EB
:101BB000358909AB1AAB2BAB3CABC901B8010E940C
:101BC0005EED6DAB7EAB8FAB98AFA50194010E942B
:101BD000BFED0E942EE60E94BCE62E966CAF7DAF54
:101BE0008EAF9FAF2E97F70167AB70AF81AF92AF0B
:101BF0008E010F5E1F4F1FAF0EAF0051110960968F
:101C00001FAF0EAF609707E219E06C961FAF0EAFE3
